:109C6A00414952434F544543004256332E33342020
:109C7A005455520050494C2000532F4E2146414919
:109C8A004C555245005245454E54455221532F4E8C
:109C9A0000434F4E5441435420414952434F544587
:109CAA004300475053004032444000403344400090
:109CBA0059454E214D454E75404B5054000A1600E9
:109CCA000180000300007E0000FE00001E00003636
:109CDA000003E60001C4000000000FFFE020555910
:109CEA00445540415241200059754B53404B414C19
:109CFA00202300504943545552450052414E4B4986
:109D0A004E47004D415020202020200043454E540C
:109D1A004552202000564152594F202020004241EE
:109D2A00534E65204B5900524F54414C415220002A
:109D3A00454E2059414B494E00594F4C4E4F4B54BA
:109D4A004C004962415245544C52004445464155E3
:109D5A004C5400202020214F525421202020204DF5
:109D6A0053460020545241434B214F4E202000209D
:109D7A00545241434B214F464620004D41524B001D
:109D8A0020545241434B2D5550212000204E4F5212
:109D9A0054482D55502120002165494B01524F54FA
:109DAA004140534565200159754B534B2053456536
:109DBA002001556555624C415220686901464C495B
:109DCA0047485420414C4C01594F4C4E4F4B544C30
:109DDA00686901524F54414C415220686901414916
:109DEA00525350414345686901415941524C4152CD
:109DFA002068690059754B534B214159524C410017
:109E0A004241524F4059754B534B20004750532003
:109E1A0059754B534B4C2000514E4820202020406E
:109E2A002148504100464C004B5954204445465461
:109E3A0020424F622020003E2143494B200021430B
:109E4A00494B200154454B52415201474F4E44451C
:109E5A00520153494C202020002165494B200143DF
:109E6A004F4D3A20202020202001544E43203123F8
:109E7A002035374B01544E4320312320392E3601E9
:109E8A0001505743403130234035374B0150574337
:109E9A00403130234031394B01014D585040313067
:109EAA00234035374B014D58502034232035374B4A
:109EBA00014D58502031232035374B014D58504021
:109ECA003130234031394B014D5850203123203154
:109EDA00394B002165494B0159454E4920594F4C90
:109EEA004E4B01594F4C4E4F4B2044454701594F59
:109EFA004C4E4F4B2053494C0101434F4D3A0159A7
:109F0A004F4C4E4F4B20414C2001594F4C4E4F4B1A
:109F1A0020474E440154594C4E4F4B20474E440162
:109F2A0001594F4C4E4B54204D53460154594C4EF7
:109F3A004B542053494C0042524720214449535420
:109F4A00004B4159440047554E434C40504F5A53D9
:109F5A002020004B41594445542020202000205302
:109F6A00544F52452157505420002046554C4C20FE
:109F7A000020204053494C20200053455220004BDA
:109F8A00495A4C00555342200055534220004C492F
:109F9A00535400476F4E4400204241474C204841E9
:109FAA005453492020202020002165494B2001528A
:109FBA004F5441405345652001594E20524F542079
:109FCA004E4F4B01524F544120445A4E4C2001549B
:0D9FDA0045525320524F54412001524F5424
:109FE7004E4F4B2053494C01524F54412053494C3B
:109FF70020200143594C2052414449555301434FB6
:10A007004D3A01524F544120414C20202001524FDC
:10A01700544120476F4E445201434845434B205219
:10A027004F00524F5441205345430059454E490074
:10A0370059454E49404B4F4E0021405445525320FD
:10A04700202040005445525320004E4F4B544C5251
:10A057002153494C0021524F54412053494C00424F
:10A067004F53414C544D4120200021524F54412120
:10A07700476F4E4452002020524144495553002116
:10A0870065494B014C4F41444043545221504301D1
:10A0970056494557404354520144454C40414C4C66
:10A0A700214354520101434F4D3A01524543562033
:10A0B700204354520153454E4420204354520056E6
:10A0C700494557204354520020204D4F5645002004
:10A0D700204D4F564520544F005343414C452020B7
:10A0E700582F5920204558495400434C5220444981
:10A0F7005354004155544F43454E54004155544F16
:10A10700204F4646002020205343414C45004449F8
:10A117005354204B4D0044495354204E4D00216564
:10A12700494B2001594152594F2020206869015855
:10A13700432D41594152206869015254452D5345D9
:10A14700542068690147454E454C20202068690125
:10A1570050494354555245536869010101454153DC
:10A16700592D5345540146414220415941524C52C1
:10A1770001544553542055655562200144454C21EF
:10A18700414C4C21464C49002165494B200153491C
:10A197004E4B544F4E4501656F4B75622D01656FF0
:10A1A7004B62404D4F4401656F4B6240494E56012B
:10A1B700564152205443402020402301564F4C55CE
:10A1C7004D4501564152494F204E554C4C0150497F
:10A1D70054434801504552494F440156415220418A
:10A1E7005640203040230154454320202040303042
:10A1F700402501534F554E44434845434B0053496F
:10A207004E4B21544F4E450053494E4B54214F4618
:10A21700460065465453454E53594F4B00564152DD
:10A22700594F2053465220004031304044414B2E75
:10A237004053455353495A00534946495244414EA6
:10A24700204F4E43452020002165494B20015441B2
:10A257004B4950202020014F544F21476F4E445205
:10A2670001014F52542F4D4553460153755A4C62C5
:10A2770021594F4C014C2F44010157494E44215459
:10A287002D55500143454E5421542D5550015741EA
:10A2970059505421425247002165494B20015354DC
:10A2A7004152544054494D45014649525354014483
:10A2B700454C544120203A014D554C5449504C458A
:10A2C700014C4153540143594C53494740202040C6
:10A2D700230153454C40524F555445010101014359
:10A2E700594C520143594C20542D55500021654972
:10A2F7004B200101554E4954014B4C494B40302CE2
:10A3070040202320014B4F4E5452415354014E4D90
:10A3170045412131383301494D502F4147505301B1
:10A3270001432D564152494F014D454D4F52594416
:10A33700554D50004D454D4F525944554D500040D5
:10A34700594F4C4E4F4B654B622020204000594FD0
:0DA357004C4E4F4B544100202043494B20F9
:10A3640020202100414C202020202000424F532057
:10A3740040003C2D204C495354202D3E202045586C
:10A3840049540053454C004E455854004E455854CA
:10A394002054505400505245562054505400434CBD
:10A3A4005220404C454700434C52204053554D00E9
:10A3B4004B4150415420202020202000204B41506C
:10A3C40000475053204841544120004B41594445D3
:10A3D400542000524F54412000454E2159414B49CD
:10A3E4004E004C495354450045544500414C54409B
:10A3F4003000424F6220524F544120200020544FDD
:10A404004F404D5543482000214C49535445405337
:10A414004543004E4F4B5441405345430021404176
:10A424004C202020202040002020404F204B402062
:10A434002021004F4B0056415200464958004741E5
:10A4440054452158004241624C414E474965200021
:10A45400535443594C2000404F464600545020006A
:10A46400406A40494E20004067404F555400202028
:10A4740048415441202021002043494B20004445B9
:10A48400474900455645540044454749625449529A
:10A49400202059454E492020004E4558542053450C
:10A4A4004C4543542045584954005843542D464C78
:10A4B4004947485420005553454400454E5445529D
:10A4C40020004D4D2E4D4D4D20004D4D2753532E04
:10A4D4005300574753213834002040554054404DD1
:10A4E400402000554054404D002055544320004C1A
:10A4F4004F43414C005357495353474400414C5434
:10A5040000535549405800415647402030402300ED
:10A51400353030003136343000205D203130404B4E
:10A52400632F70005D2020203140632F2300205DC5
:10A53400202035404B5453005D203230304046508B
:10A544004D00406340204B63004654204B63004061
:10A554006340204E4D004654204E4D004D2F530075
:10A564003230305E003530305E003122003222005D
:10A57400332200352200382200464C3700464C3145
:10A584003600464C333300464C36350046313030C5
:10A5940000463136300046323630005E25264053C0
:10A5A4004F47005E25264054415300414C54005609
:10A5B400415200225E2F24004B545300532F4E006F
:10A5C4002224004B5400225E004E4D00302C3500F6
:10A5D400312C3000322C3000302C3600312C32003B
:10A5E400322C3500332C3800372C350040313500FF
:10A5F40040333000403630005441534B00464C2D1C
:10A604004441544500545000544F460053544100B3
:10A6140046494E004C414E00534554204F46465344
:10A624004554004953412048454947485400415541
:10A63400544F2D474F200053544152540020434857
:10A6440045434B40414C4C005241442044495354EF
:10A65400004053454C404845494748543A00475008
:10A6640053404241524F40414C4C0053494E4B40A1
:08A67400312D3221632F230078
:1064F400304D2475A7049005C2E0F51CE0F51DE0BD
:10650400F51EE0F51FE0F56DE0F56EE0F56FE0F5E2
:10651400541270B6126AF42275C70375C6E475B9CD
:1065240001E5BCB481431270B61256DC8E628F63EF
:106534007568F97569001265CA203C2D203B2B1241
:1065440066FF1266D3856D1C856E1D856F1E85548E
:106554001F126636203C12203243201D231266FF90
:10656400126AF4E532242850DC22126636203CF903
:10657400203DF6203205201DBD80EF301DB880EA95
:106584001266FF126AF4856D1C856E1D856F1E856B
:10659400541F1266E9126AF4203DCE8099126922D2
:1065A400201D0D7553107400126885203DBB808634
:1065B400E553540FC553C4540F20350512679A8010
:1065C40003126885808BC23CD23B126686FD12663C
:1065D40086FC126686C39573F565EC9574F564EDD7
:1065E4009575600504600A800EE56424E05011800E
:1065F40006E56424204009126686126686026686D1
:10660400126686FD126686FC126686C39576F56769
:10661400EC9577F566ED9578600904600122E566EE
:10662400F48002E5668562F0A474E025F04002C2BD
:0D6634003B22C23C126686A2E7923DA2E620
:10664100921DA2E592324026A2E492E592E692E7FB
:10665100FC1266862565F565EC3564F5641266867F
:10666100FC1266862567F567EC3566F56622A2E4BD
:106671009235540F79C6F712668609F7301D051257
:106681006686F55322E5697023E56860302404408D
:106691002CE56875F004A485F0C7F5C675B901E568
:1066A100BCB4811985BD68756902801E54037010E0
:1066B10005C675B901E5BC056953690F22D23C22B3
:1066C100147004E5BD80F0147004E5BE80E9E5BFF7
:1066D10080E575A7009006F6E56DF0A3E56EF0A3E1
:1066E100E56FF0A3E554F02275A7009006F6E0F5FA
:1066F1006DA3E0F56EA3E0F56FA3E0F55422E56428
:10670100B2E7F56D85656EAB67E566FC30E707C3FB
:10671100E49BFBE49CFCAA62A9631253DCE56630AE
:10672100E707C3E49DFDE49EFEEEB2E7F56F8D54ED
:106731002275380C12698B1269D6D553012275382E
:106741000C12695C1269CCD55301227538001269AB
:0E6751007412699BD553012275380012695CE1
:10675F0012699BD553012275380312698B126A0790
:10676F00D553012275380312695C1269FDD55301A7
:10677F002275380F126974126A2CD553012275389D
:10678F000F12695C126A2CD553262290679F2373D0
:10679F008091807780688059804A803B802C801D53
:1067AF00800E80DA80CB80BC80AD809E808F808011
:1067BF0075381512698B126A4ED55301227538152B
:1067CF0012695C126A43D553012275380912697434
:1067DF00126A14D553012275380912695C126A14B2
:1067EF00D553012275380612698B1269BED5530134
:1067FF002275380612695C1269B3D55301227538B8
:10680F00121269741269E4D5530122753812126994
:10681F005C1269E4D553012202673275381512698B
:10682F008B126A4ED553012275380F12695C126AAA
:10683F002CD553012275380F126974126A2CD55357
:10684F00012275380312695C1269FDD55301227557
:10685F00380312698B126A07D5530122753800125B
:10686F00695C12699BD55301227538001269741245
:10687F00699BD553262290688A2373809E80A980B6
:10688F00B480BF80CA80D580E08010801B802680B6
:10689F0031803C80478052805D806875380C12696A
:1068AF005C1269CCD553012275380C12698B1269B1
:0E68BF00D6D553012275381212695C1269E4B5
:1068CD00D55301227538121269741269E4D553013A
:1068DD002275380612695C1269B3D55301227538D9
:1068ED000612698B1269BED55301227538091269DA
:1068FD005C126A14D5530122753809126974126A33
:10690D0014D553012275381512695C126A43D5539B
:10691D00012202682A78C686040886037AED12538E
:10692D009A78CAA60408A60378C686040886037A50
:10693D006212539A78CCA60408A60378C68604087A
:10694D0086037AB512539A78C8A60408A603227551
:10695D001A6A751B0A78CA8618088619126B9F78F1
:10696D00CC86060886072278C88618088619E4F5AD
:10697D001AF51B126B9F78C886060886072278C603
:10698D008618088619751A00751B01026B9FE51D87
:10699D002519F51DE51C3518F51CC3E51F9FF51FC1
:1069AD00E51E9EF51E22C3E51F9FF51FE51E9EF5F4
:1069BD001EC3E51D9519F51DE51C9518F51C22E561
:1069CD001D2FF51DE51C3EF51CC3E51F9519F51F83
:1069DD00E51E9518F51E22C3E51D9FF51DE51C9EB0
:0969ED00F51CC3E51F9519F51F07
:1069F600E51E9518F51E22E51F2FF51FE51E3EF52F
:106A06001EE51D2519F51DE51C3518F51C22C3E5E7
:106A16001D9519F51DE51C9518F51CE51F2FF51F8D
:106A2600E51E3EF51E22E51D2FF51DE51C3EF51C57
:106A3600E51F2519F51FE51E3518F51E22C3E51DB0
:106A46009FF51DE51C9EF51CE51F2519F51FE51E86
:106A56003518F51E22E51A7009E51B70058C068DA2
:106A66000722ED851BF0A4A2F792D5ED851AF0A4B6
:106A7600AEF0FFEC851BF0A4A2D53FEE35F0FF92F9
:106A8600D5EC851AF0A42FFFE435F030D50104FECD
:106A960022E4F51AF51BEF4E7003051B22EF65196C
:106AA6007006EE65187001227808C3EF33FFEE33E7
:106AB600FEEF9519F5F0EE95184003FEAFF0E51AD6
:106AC60033F51AD8E5F4F51A751BFF7805C3EF33CD
:106AD600FFEE33FEEF9519F5F0EE95184003FEAF85
:036AE600F0E51BBD
:106AE90033F51BD8E5F4C403F51B22E51D9511E523
:106AF9001C9510500BE56E9511E56D95105001220E
:106B0900E51F9511E51E9510500BE5549511E56F9C
:106B19009510500122E51D9513E51C9512400BE5D2
:106B29006E9513E56D9512400122E51F9513E51E3B
:106B39009512400BE5549513E56F951240012253C8
:106B49002CF8C3E51F9554FFE51E956FFE92605022
:106B590007C3E49FFFE49EFEC3E56E951DF519E5A5
:106B69006D951CF5189261500BC3E49519F519E45C
:106B79009518F518C3E5199FE5189E9262500AE524
:106B890018CEF518E519CFF519126A97E52C5407AF
:106B990075F003A4F538E538906BA573026BBD0257
:106BA9006BD1026BDF026BF7026C0A026C1D026C7F
:106BB9002B026C43851C16851D17C3E4951FF5151B
:106BC900E4951EF514026C56851C16851D17851E45
:106BD90014851F158077C3E4951DF517E4951CF5F9
:106BE90016C3E4951FF515E4951EF514805FC3E4FB
:056BF900951DF517E4F5
:106BFE00951CF516851E14851F15804CC3E4951F34
:106C0E00F517E4951EF516851C14851D158039851E
:106C1E001E16851F17851C14851D15802BC3E49524
:106C2E001FF517E4951EF516C3E4951DF515E495AD
:106C3E001CF5148013851E16851F17C3E4951DF5CC
:106C4E0015E4951CF5148000C3E5179513E516950C
:106C5E001210D70122E5159513E514951210D701E0
:106C6E0022E519F92517FFE518F83516FED3EF952D
:106C7E0011EE9510500122E5119517FDE5109516B0
:106C8E00FC402A4D6027126A5BE5152FF515E514B9
:106C9E003EF514E5159513E514951210D70122E56E
:106CAE00199DF9E5189CF8851016851117E5172919
:106CBE00FFE51638FEE5139FE5129E500BC3E51354
:106CCE009517F9E5129516F8E51A700AE51B700688
:106CDE00AA00AB018013E9851AF0A4E5F0FBE88564
:106CEE001AF0A42BFBE435F0FAE5152BFBE5143A6C
:066CFE00FAE5119BE51010
:106D04009A10D70122EB9515FDEA9514FCC3E515FD
:106D14009511E514951010D717E5139BE5129A50B9
:106D240036E5139515FFE5129514FE126FD38027EF
:106D3400EB9511FFEA9510FEAA00C001126FD3D0A3
:106D440003E5172BFBE5163AFAEB99F517EA98F5E4
:106D540016851115851014C2D5E5466002D2D5AA50
:106D640056E98AF0A4ABF0E88AF0A42B30D5047578
:106D7400F00384F8700122E5172513FDE51635129A
:106D8400FCED8AF0A4ABF0EC8AF0A42B30D50475AA
:106D9400F00384FEE5152513FDE5143512FCED8A98
:106DA400F0A4ABF0EC8AF0A42B30D50475F0038486
:106DB400F9E538906DBB73026DD3026DDF026DE8A7
:106DC400026DF1026DF7026E03026E0A026E0FC3CA
:106DD400743E9EFFC3743E99FE8032C3743E9EFF90
:106DE400AE018029AF06C3743E99FE8020AF06AE83
:0D6DF40001801AC3743E9EFEC3743E99FFD9
:106E0100800EC3743E99FF8007C3743E9EFEAF019E
:106E110008EF2437FFE51B7007E51A700CE8800EB8
:106E2100A2E7E51A50030460F488F0A4E5F06001DC
:106E310004F923FA98FBC3E998C333F9906E43E54B
:106E41003873026E5B026E88026EBD026EEA026FDB
:106E510017026F44026F71026F9E05A7800BEB3022
:106E6100E7032A8002291E1FFBEEC45403F583EEBB
:106E71005408C42FF582EE5407243883F5F0E04519
:106E8100F0F0D8DA05A72205A7800BEB30E7032A3B
:106E91008002290E1FFBEEC45403F583EE5408C48F
:106EA1002FF582EE5407240B83F5F0E045F0F0D87E
:106EB100DA05A722804020100804020105A7800BF3
:106EC100EB30E7032A8002291E0FFBEEC45403F5C1
:106ED10083EE5408C42FF582EE540724EC83F5F0B9
:106EE100E045F0F0D8DA05A72205A7800BEB30E7E3
:056EF100032A800229C4
:106EF6000E0FFBEEC45403F583EE5408C42FF5823F
:106F0600EE540724BF83F5F0E045F0F0D8DA05A784
:106F16002205A7800BEB30E7032A8002291F1EFB00
:106F2600EEC45403F583EE5408C42FF582EE5407DD
:106F3600249283F5F0E045F0F0D8DA05A72205A7FC
:106F4600800BEB30E7032A8002291F0EFBEEC454A8
:106F560003F583EE5408C42FF582EE5407246583A7
:106F6600F5F0E045F0F0D8DA05A72205A7800BEB8F
:106F760030E7032A8002290F1EFBEEC45403F58373
:106F8600EE5408C42FF582EE5407243883F5F0E05A
:106F960045F0F0D8DA05A72205A7800BEB30E7030A
:106FA6002A8002290F0EFBEEC45403F583EE540823
:106FB600C42FF582EE5407240B83F5F0E045F0F07C
:106FC600D8DA05A7228040201008040201EC701FC1
:086FD600ED20E740D2E023CFDB
:106FDE0023CF30E7F980357B08801A7B1080167B33
:106FEE002080127B40800E20E4ED20E3EE20E2EFC5
:106FFE0020E1F07B80EE8BF0A4CF8BF0A4E5F02F98
:10700E00FFEC8BF0A4CD8BF0A4E5F02D2499838FAB
:10701E00F0A433E5F033FBE98BF0A4E5F0C88BF078
:10702E00A428F9E435F0F822FFFEFCFAF8F6F4F2A3
:10703E00F0EFEDEBEAE8E6E5E3E1E0DEDDDBDAD901
:10704E00D7D6D4D3D2D0CFCECCCBCAC9C7C6C5C45F
:10705E00C3C1C0BFBEBDBCBBBAB9B8B7B6B5B4B379
:10706E00B2B1B0AFAEADACABAAA9A8A8A7A6A5A465
:10707E00A3A3A2A1A09F9F9E9D9C9C9B9A99999829
:10708E009797969594949392929190908F8F8E8DD0
:10709E008D8C8C8B8A8A898988878786868585845C
:1070AE00848383828281818075A7009070DCE5469F
:1070BE00FA24FA50027A05EA2323F978107F049312
:1070CE00F60809E9DFF99070F4EA93F556227FC2CB
:1070DE00803E7F4680BA7E8C81747D1882E87A303D
:1070EE0085D074608BA08080402010081271000241
:1070FE007356D215D274D273C219C23A1256DC8E9E
:10710E0047757D0075460575520212914612022191
:10711E00E53524EB500E1291467F1990A0F11276B0
:10712E00F012DD12E55275F016A4F57012730C759F
:10713E007E151271D77F237E0990A0CF127702128F
:10714E00DD1210000810010D10021280E212727F83
:10715E0075330180DA1272C475330180D2757E00E8
:10716E001271D77E0090A0E01277357F237E0590B6
:10717E00A0D612770212722812DD12E55210000FFD
:10718E0010010510028780D5045403F55280CE12EB
:10719E0071D77F237E0B90A10E127702E546600712
:1071AE001460041412411A12DD12E5461000081084
:1071BE00010B10021180D860D6154680D2B405029C
:1071CE0080CD054680C902711B75320012DEE87F44
:1071DE00017E1190A0C61277357E0012D5A9E57EEC
:1071EE00D26612D60075170812DA3312415975712C
:1071FE0000C20612D750741BFFF5177E0F90A11513
:10720E00305D0390A11D127735129189125D0D121A
:10721E0046BFC20612651C021E03E55260141460BE
:10722E001E1460297F647E2D791C1272721E1FD966
:10723E00F9227F6A7E1F79281272721FD9FA227F75
:10724E00487E2D791C1272720F1ED9F9227F567E3E
:10725E003379281F12DE2D0F0F12DE2D1F12DE2D99
:10726E001ED9F0221E12DE2D0E0E12DE2D1E02DE95
:10727E002DE552605514606814606D800075709E27
:10728E001272F98003757000E5732540F573E435CD
:10729E0074F574E43575F575227570161272968054
:1072AE000375702DE5762542F576E5773541F57750
:1072BE00E43578F57822E55260CB1460DC1460E199
:1072CE0080007570441272B2800375705AE5739522
:0972DE0040F573E5749400F574A9
:1072E700E5759400F575227570711272DB80037570
:1072F7007088E5769542F576E5779541F577E578F7
:107307009400F57822E54690732293F540FEAD4749
:10731700E4FFFC12546F8E418F4222020C1830603A
:10732700C07F40120E9E121E1912DD121275D1EB8C
:107337007005909E3A800B1273DF90A42C50039037
:10734700A4727F3F7E0412770212DD1212DDF31260
:10735700DE2375370990A086121CFF9073667302AF
:1073670002930275260270FA0276020273560273BE
:107377007E0273970273287F2E12168680D17F367E
:107387007E0490A40112770212DD1212DDF380BF92
:107397007F37120E9E121E1912DD121275B5124892
:1073A7004FD2AC1000A9306DFA12748F203BCF403A
:1073B700ED7568F97516001274DC40FB1276787F5C
:1073C700367E29E51612D38912DD1205161277A823
:1073D70078C6B6F7E20275AF7C0512484F12DC2C6F
:1073E700744112DC3D745312DBFAEB12DC1B12778B
:1073F700BA5003DCE5227515F975160010000EE585
:1074070015602512743140051274585002D3227F3B
:107417003F7E29E51612D38912DD127F1412DE0A88
:107427000516E51664F870D4C322127D7075B9018C
:10743700E5BCB4811AE5BDF51570037516F778C676
:0B744700A616127EB9127EB1127EB1B3
:10745200C3027EB1D3227F0575F019D5E0FDD5F0C8
:10746200FA12484F12DC2C744112DC3D744212DBDA
:10747200FA7E0F78C6E60812DBFADEF912DC1E127B
:1074820077BA400122DF012275F00080CEC23B12A2
:10749200484FD2AC12DB85204C3CB440F712DB8A59
:1074A200B4400312DB8AB4412DF53812DB8AB4539F
:1074B2002512DB8AFA12DB8AE538701A12DB8AB4EB
:1074C2000D1412DB8AB40A0EC3E5169A4003027742
:1074D2009FC2ACD23B22C2ACD3221277FE12484FDB
:1074E200D2AC1000F112DB85204CEBB440F412DB7D
:1074F2008AB4400312DB8AB441DCF53812DB8AB469
:1075020042D47E1078C612DB8AF608DEF9E53870BE
:10751200C512DB8AB40DBF12DB8AB40AB9C2ACC38E
:10752200220273567F0A120E9E121E1912DD1212C9
:1075320075B5124868D2AC1000E712DB8AB440F588
:10754200F53812DB8AB46EED12DB8AE538600A1276
:107552004868744F12DC0680DC124868744012DC02
:107562003DE51612DC0612DC107568F9751600127C
:107572004868D2AC10003912DB8AB440F7F53812F1
:10758200DB8AB44EC07E1078C612DB8AF608DEF9BA
:10759200124868E5386007744F12DC0680D1127613
:1075A200780516745112DC0678C6B6F7C212761543
:0C75B200027356751500751603127D67F4
:1075BE0075B901E5BC30E70205160515E515242061
:1075CE0050EB227B007515F9127D7075B901E5BC83
:1075DE00B481010B0515E515240450EC7515011247
:1075EE007D6775B901E5BCB481010B0515E5152460
:1075FE002050EC227F1C120E9E121E5C400675154A
:10760E00F9127615027356E51560372404401A24D4
:10761E001E5019E515240740028027127D70127640
:10762E00510515E515240450F2751501127D677587
:10763E00B901E5BC30E7031276510515E515242096
:10764E0050EA22127666124EE605C6124EE605C6C0
:10765E00124EE605C6024EE674FF800574048001E4
:10766E00E4F5BCF5BDF5BEF5BF22E568606AF5151B
:10767E000515E5152404501D751501127D6775B9A4
:10768E0001E5BC30E70280190515E515242050EB05
:10769E00751500800C241C60F750E0E5152406508B
:1076AE0037E56875F004A485F0C7F5C675BC81E5AD
:1076BE0015F5BDF56878C6B6F70375BD00081276E8
:1076CE00DB1276D51276D586BC0886BD0886BE0836
:0976DE0086BF08124EE605C62223
:10C05B0012AE9712C15A12828112C0DF128289125C
:10C06B00C0EC02AE9B12AE9712C15A1282817F5A5C
:10C07B00C23C12816312835F783F79437F607EEA13
:10C08B0012C14E1282897F6512816312835F783DE4
:10C09B0079417F207E4E12C14E303C2012C31012CC
:10C0AB00C16B783F794312C0CA783D794112C0CA3F
:10C0BB0012C31078D7E65480F675370002935BC332
:10C0CB00E796FF1819E796FE0809C3E69FF71819BC
:10C0DB00E69EF7227F5B7E0690A5051277351F80C3
:10C0EB000A7F667E14745912D4A21F127FEC7E391C
:10C0FB00E402D4C17866E620E73418C3E6947208EC
:10C10B00E694045029C318E6941F08E69404401ED5
:10C11B007869E620E71818C3E6940E08E6940150F8
:10C12B000DC318E6947508E694004002D322C3228F
:10C13B00E67D0030E7011D08E62BFB18E63CFCE42E
:0EC14B003DFD22C3EB9FF6F71819EC9EF6F7A8
:10C159002212C0FF400CE47842F608F67840F6084F
:10C16900F6227864C3E6946AF55708E6944CF556C6
:10C179000808C3E69458F55B08E694AEF55A753994
:10C1890000AC56AD57EC12B244784C12B2D2AC5A4C
:10C19900AD5BEC12B244785012B2D27F2B7E867D11
:10C1A900777C1812B209785012B2C612B11512B2C0
:10C1B90009785012B2C612B11512B209785012B2EA
:10C1C900C612B11512B2097F367E847D257C6412B0
:10C1D900B209785012B2C612B11512B209784C12CE
:10C1E900B2C612B11512B2097F3F7EA27D607C8B67
:10C1F90012B209785012B2C612B11512AF0312AFBA
:10C209000312B2DE7F3F7E807D057CE6053912B1DF
:10C2190015784812B2D27F2C7E937D477C7F12B26B
:10C2290009785012B2C612B11512B209785012B279
:10C23900C612B11512B209784C12B2C612B1151252
:10C24900B2097F357EB47DF87CDF12B209785012CD
:10C25900B2C612B11512B209785012B2C612B1158E
:10C2690012B2097F3F7EED7D227CCD12B209784C56
:10C2790012B2C612B11512AF0712AF03784412B247
:10C28900D27F317E397D9D7CE712B209784C12B29A
:10C29900C612B11512B209784C12B2C612B11512F2
:04C2A900B20978441A
:10C2AD0012B2C612AF0712B2097F2C7E377D0C7CFD
:10C2BD00A312B209784C12B2C612B11512B2097896
:10C2CD004C12B2C612B11512B209784C12B2C61286
:10C2DD00B11512AF0712B2DE7F3F7E807D027C9FCB
:10C2ED00053912B115784412B2D2784812B2C6127D
:10C2FD00B27B8E428F43784412B2C612B27B8E400F
:10C30D008F4122753900AC42AD43EC12B2447848EE
:10C31D0012B2D2AC40AD41EC12B244784412B2D25A
:10C32D007F2B7E537D507C0912B209784812B2C61C
:10C33D0012B11512B209784812B2C612B11512B265
:10C34D0009784412B2C612B11512B2097F347EF2C9
:10C35D007DCD7CA312B209784812B2C612B1151266
:10C36D00B209784812B2C612B11512B2097F3F7EDA
:10C37D000A7D2E7CAE12B209784412B2C612B115E6
:10C38D0012AF0312AF03784C12B2D27F2B7E4F7DCA
:10C39D00AF7CB212B209784812B2C612B11512B200
:10C3AD0009784812B2C612B11512B209784812B204
:10C3BD00C612B11512B2097F357EB17D4B7C951237
:10C3CD00B209784812B2C612B11512B209784412E8
:10C3DD00B2C612B11512B2097F3F7E497DCD7C45A3
:10C3ED0012B209784812B2C612B11512AF0712AFC8
:10C3FD0003785012B2D2784C12B2C612B27B8D5560
:10C40D008E568F57785012B2C612B27B8D598E5AF6
:04C41D008F5B786455
:10C42100E557246AF608E556344CF608E555340418
:10C43100F608E55B2458F608E55A34AEF608E4350B
:03C4410059F62287
:1091A90012AE9712983A12AE9B7F6690A4E7127797
:1091B900331292177F5A78C41291F31291FB78C631
:1091C9001291F31291DE7F6578C81291F31291FB27
:1091D90078CA1291F37E2DE51B12D4C17E33E51AAC
:1091E90012D4C17E39E51902D4C186040886030266
:1091F90053397E15E51C12D4C17E1BE51B12D4C15F
:109209007E21E51A12D4C17E27E51902D4C17F5AFD
:109219007E01E53A12D3D77E0B909C2EE53B930253
:10922900D4D4E6FF08E6FE08E6FD339217E45001C0
:10923900F4FC12B2EF75130A75390112B4ED78D73F
:10924900E6C2E775F00A84F9303D02A9F012B2EFDF
:109259008913053912B4C630170A053912B4D9056C
:109269003912B4D9A80302B2D212AE9712983AC2EF
:109279003C7F5A7E0312851012921712DD121000DC
:109289000810011510022080EFE53A146004153A20
:109299008003753A3CD23C80DFE53AB43C05753A27
:1092A9000180F2053A80EE7E0312850B7E0B128552
:1092B9001012921712DD1210000810011510022069
:1092C90080EFE53BB40205753B158002153BD23CA6
:1092D90080DFE53BB41505753B0280F2053B80EE66
:1092E9007E0B12850B7F5A78C41291F31291FB12EF
:0792F900936412836F78C437
:109300001293BC78C61291F31291DE129396751CDB
:109310000012836F78C61293BC7F6578C81291F3F0
:109320001291FB12936412836F78C81293BC78CAAF
:109330001291F31291DE129396751C0012836F78CE
:10934000CA1293BC303C14E53B24F4500B78C9E6B8
:109350002410F618E63427F61293C212AE9B127E42
:10936000F102DD12C2247E15E51C128460F51CD2C8
:10937000247E1BE51B128460F51B1023E77E21E58C
:109380001A128460F51A1023E67E27E5191284600C
:10939000F5191023E822C2247E2DE51B128460F506
:1093A0001BD2247E33E51A128460F51A1023E77E5F
:1093B00039E519128460F5191023E622ECF608EB62
:1093C000F622129C4678C8E6FE0886073395E0FD33
:1093D000FC12B2097FE87E037D007C0012B4ED121E
:1093E000B20978CAE6FE0886073395E0FDFC12B4A0
:1093F000C612B2097F807E697D677CFF12B4C6EC1D
:1094000012B24012B2097F3F7E807D0D7C1D12B1E9
:109410001512B2097F3D7E407D007C0012B20978B2
:10942000BC12B2C612B11512B2097F3E7E807D0019
:109430007C0012AF0712B20978BC12B2C612B11585
:0994400012B2097F3F7E807D001D
:109449007C0012AF0312B20978B412B2C612B11578
:1094590012B18D783C12B2D27F407E807D007C00B3
:1094690012B209783C12B2C612B11512B36C12B21B
:10947900097F3F7EA87D007C0012B20978B812B23C
:10948900C612B11512B11512B2097F407E007D00D6
:109499007C0012B209783C12B2C612B11512B36C33
:1094A90012B2097F3F7EC07D007C0012B11512AF58
:1094B9000712B20978B812B2C612B11512B20978F8
:1094C9003C12B2C612AF07785412B2D212B3567810
:1094D9005812B2D212B20912B11512B20978C012D9
:1094E900B2C612B115784412B2D2785412B2C61269
:1094F900B36C783C12B2D212B20912B11512B20988
:1095090078BC12B2C612B115783C12B2D27F3E7E37
:10951900C07D007C0012B209783C12B2C612B115A6
:1095290012B2097F3F7E007D007C0012AF0712B2A4
:1095390009783C12B2C612B11512B2097F3F7E807A
:109549007D007C0012AF0712B20978B412B2C612BC
:10955900B115787012B2D278C4E6FE088607339541
:10956900E0FDFC12B2097FE87E037D007C0012B4A5
:10957900ED12B20978C6E6FE0886073395E0FDFCD0
:1095890012B4C612B2097FE07E5E7DF87CFF12B488
:10959900C6EC12B24012B2097F3F7E7F7DE57CC9DD
:0595A90012B209787008
:1095AE0012B2C612B11512B18D785012B2D27F3FDF
:1095BE007EF07D007C0012B209783C12B2C612B168
:1095CE001512B2097F3F7EC07D007C0012AF0712DC
:1095DE00B209783C12B2C612B11512B2097F3F7EA3
:1095EE00807D007C0012AF07783C12B2D278BC129C
:1095FE00B2C612B2097F3F7E807D007C0012AF039F
:10960E0012B209783C12B2C612B20978B412B2C6BE
:10961E0012B11512B115784012B2D2785412B2C6E8
:10962E0012B3A4783C12B2D212B20912B1157874E8
:10963E0012B2D27F417E107D007C0012B20978C03A
:10964E0012B2C612B11512B2097F407E807D007C27
:10965E000012B209784412B2C612B11512B2097FC5
:10966E00417E207D007C0012AF0312B209784412B5
:10967E00B2C612B11512B2097F407E407D007C0049
:10968E0012B209787412B2C612B11512B2097F4025
:10969E007EA07D007C0012AF0712AF0712AF03123F
:1096AE00B209785012B2C612B11512B20978501220
:1096BE00B2C612B11512B2097F3D7E2A7DAA7CABCD
:1096CE0012B11512B2097F3F7E007D007C0012AFF1
:1096DE000312B209783C12B2C612B209787012B2F5
:1096EE00C612B11512B209784012B2C612B18D125D
:1096FE00B209785012B2C612B11512B209785012D0
:10970E00B2C612B11512B11512B209785412B2C600
:0C971E0012AF0312B2097F4A7E517DD2C7
:10972A007CCB12B11512B27B78AC12B2D27F407EDA
:10973A00007D007C0012B209787412B2C612B1150B
:10974A0012B2097F3F7E807D007C0012AF0712B201
:10975A0009784412B2C612AF0712B209785012B28F
:10976A00C612B11512B209785012B2C612B1151248
:10977A00B209785012B2C612B11512B2097F3E7EF2
:10978A002A7DAA7CAB12B11512B209785012B2C660
:10979A0012AF0312B209785812B2C612B18D12B2C0
:1097AA00097F4A7E517DD27CCB12B11512B27B124F
:1097BA00B209AF3AEF3395E0FEFDFC12B2097F40E1
:1097CA007E7E7D057C0012B4ED12B2097F607E7543
:1097DA007D587CFF12B4C612B4C678B012B2D278E1
:1097EA00AC751B641298118F1C78B0751B671298A0
:1097FA0011E51C75F00AA42FFF249C50027F007803
:10980A00D7E654802FF62275390012B2C612B20971
:10981A007F0A7E007D007C0012B599A81BE513F62D
:10982A0008E512F608E511F6335004EFF404FF22B6
:10983A00C23D78647BAC12922BD23D78677BB01222
:10984A00922B129C467F007EE47D577C0012B2095F
:10985A0078AC12B2C612B4C612B2097F007E537D2A
:0E986A00077C0012B59912B22885133B7F804F
:109878007ECB7DA47C0012B20978B012B2C612B4B5
:10988800C612B2097F407E7E7D057C0012B5991212
:10989800B228E513F56F04F53A85126E85116D85CA
:1098A800106C7F407E7E7D057C0012B209786C12B8
:1098B800B2C612B4ED12B2097F607E0C7DA27C00A4
:1098C80012B20978B012B2C612B4C612B4D9786C02
:1098D80012B2D278AC12B2C6EC12B24012B2097F00
:1098E800347E9C7D2B7C5F12B115785412B2D21253
:1098F800B356785012B2D2786C12B2C6EC12B2409B
:1099080012B2097F347E9C7D2B7C5F12B11512B296
:1099180009785012B2C612B115784012B2D27F40FF
:109928007E007D007C0012B209785412B2C612B1D2
:109938001512B36C12B2097F3D7EC07D007C001207
:10994800B20978BC12B2C612B11512B2097F3E7EB6
:10995800C07D007C0012AF0712B20978BC12B2C6F3
:1099680012B11512B11512B2097F3D7E407D007CFF
:109978000012B20978BC12B2C612B11512B2097F30
:109988003E7E807D007C0012AF0712B20978BC12BF
:10999800B2C612B11512B2097F3F7E807D007C00ED
:1099A80012AF0312B209785412B2C612B11512AF2F
:1099B8000312B2097F407E807D007C0012B20978D4
:1099C8005412B2C612B11512B36C12B2097F3D7EA1
:1099D800707D007C0012B20978BC12B2C612B115B3
:1099E80012B20978BC12B2C612B11512B11512AF73
:1099F8000712B20978B412B2C612B115785812B269
:109A0800D2785412B2C612B36C783C12B2D27854DF
:109A180012B2C612B3A4785412B2D2783C12B2C6AB
:109A280012B20912B11512B20978BC12B2C612B13B
:109A380015783C12B2D27F3E7EC07D007C0012B207
:109A480009783C12B2C612B11512B2097F3F7E00E6
:109A58007D007C0012AF0712B209783C12B2C61220
:109A6800B11512B2097F3F7E807D007C0012AF07DE
:109A780012B20978B412B2C612B115787012B2D205
:109A8800785012B2C612B20912B11512B20978C0D2
:109A980012B2C612B115784412B2D2785412B2C6B4
:109AA80012B20912B115787412B2D2784012B2C645
:109AB80012B20912B115783C12B2D27F407E807D75
:109AC800007C0012B209784412B2C612B11512B263
:109AD800097F417E107D007C0012AF0712B2097821
:109AE8004412B2C612B11512B209787412B2C61273
:109AF800B2097F407EA07D007C0012AF0312AF0741
:109B080012B209783C12B2C612B11512B2097F3DE1
:109B18007E2A7DAA7CAB12B11512B2097F3F7E0066
:109B28007D007C0012AF0712B209785412B2C61237
:109B3800B209787012B2C612B11512B209783C1285
:109B4800B2C612B11512B11512B209785812B2C6BE
:109B580012AF0712B2097F3F7E7F7DE57CC912B143
:019B680015E7
:109B690012B2097F4B7E187D967C8012AF0712B224
:109B79007B12B2097FE87E037D007C0012B5991241
:109B8900B22878C8A61208A61308A60608A6077858
:109B99007412B2C612B2097F3F7E807D007C00122A
:109BA900AF0312B209784412B2C612AF0712B20952
:109BB9007F3E7E2A7DAA7CAB12B11512B20978408C
:109BC90012B2C612B11512B209783C12B2C612B15C
:109BD9001512B209784012B2C612AF0712B2097F44
:109BE9003F7E7F7DE57CC912B209787012B2C61238
:109BF900B11512B11512B2097F487EF47D247C009B
:109C090012AF0712B27B12B2097FE87E037D007C96
:109C19000012B59912B22878C4A61208A61308A68C
:109C29000608A607223F3F4344454647484A4B4C4E
:109C39004D4E5051525354555657583F3FE4F539FC
:109C4900F5A7909C5A791078B4E493F6A308D9F94A
:109C59002232A5C24A4A19DC3A885CDB3BFFD6DCD2
:019C69003BBF
:10AE9700D2D58002C2D575A70490040078107F0B25
:10AEA70012AEC378267F0512AEC3783C7F2212AE5E
:10AEB700C3786A7F0F12AEC375A7002230D506E6A6
:10AEC700F008DFFB22E0F608DFFB22D2D58002C2C2
:10AED700D575A7049006FA78737F0612AEC375A7D7
:10AEE7000022DA0CD902800BD906303701B350059E
:10AEF70002B076923702B062D9F680F9D236800274
:10AF0700C23612B0A7303606C86002B237C89236CA
:10AF1700DAD0D9E4B8000A12B0EEA236923702B0FE
:10AF27004B60FBB51300400F12B0EEA23692F7A2AA
:10AF3700379236A2F79237C398F40424E740DF2408
:10AF470019AD29AC28AB277A00C394084008CDCCAB
:10AF5700CBCAE4CD80F424086010F9C3ED13FDECEF
:10AF670013FCEB13FBEA13FAD9F1A236303701B31E
:10AF770040308A17E5102BF518E5113CF519E51255
:10AF87003DF51A501A13F51AE51913F519E51813B3
:10AF9700F518E51713F5170513E5137002051402E5
:03AFA700B001E412
:10AFAA00C39AF517E5109BF518E5119CF519E512FA
:10AFBA009DF51A500DB237C378177F04E496F60848
:10AFCA00DFFA7A047019E513C39408F513500215D1
:10AFDA0014E4C517C518C519F51ADAE802B0A22093
:10AFEA00E7BAE5137002151415137817C37F04E640
:10AFFA0033F608DFFA80E8E51A20E7137817C37FEB
:10B00A0004E633F608DFFAE513700215141513E5A2
:10B01A00173378187F03E63400F6500E08DFF77509
:10B02A001A800513E51370020514E51420E754701D
:10B03A0027E513604E046020851A128519118518B8
:10B04A00105326F0AC10AD11A237E51313FFE51229
:10B05A0092E7FEA81302B228E4F512F511F510F5ED
:10B06A00147513FF5326F043260580D8E5FFF51221
:10B07A00F511F510751400F513D2375326F043264F
:10B08A000980C15326F0432603E4F512F511F510A1
:10B09A00F514F513C23780AC5326F080EC79017AA7
:10B0AA00018512F0E513A2F7339237751400F513F0
:10B0BA006002D2F785F012A813B8FF0809E512C298
:01B0CA00E79E
:10B0CB006001098C278D288EF0A2F7EF3304700AEC
:10B0DB000AC2F705F00AD5F0011A146002D2F785FF
:10B0EB00F02922C88813C512C529C512C511C52858
:10B0FB00C511C510C527C51022DA03B8000302B06D
:10B10B0076D9028002D9F702B06212B0A7303701AC
:10B11B00B392377004D9E78005DADEB8000302B0CA
:10B12B00A2D9E2C3947E500215142513F5135002D5
:10B13B0005147815760008B81BFA78277915E608F8
:10B14B00FAE8FC78108AF0E608A427F709E5F0374F
:10B15B00F7500989F00907E760FBA9F0B813E61966
:10B16B0019ECF8B82AD802B00102B08DB8FFFA0278
:10B17B00B076D9FB02B062DAF6B800F002B0A212D8
:10B18B00B2DE12B0A7303701B392377007D9E3B8EC
:10B19B0000E280DBDAE1B8000280E1D9D5C8C398C0
:10B1AB0050021514247F50020514F513781A7600FB
:10B1BB007A1A7B80C3E5109527E5119528E5129542
:10B1CB00294016C3E5109527F510E5119528F511C3
:09B1DB00E5129529F512E64BF688
:10B1E400DA0302B001EB03FB30E703187600C3E592
:10B1F4001033F510E51133F511E51233F51240CA99
:10B2040030E7DD80B6E53905396010D0F0D0E0C014
:10B2140010C011C012C013C0E0C0F08F138E128D85
:10B22400118C1022E539146010D0F0D0E0D013D086
:10B2340012D011D010C0E0C0F01539227920800C52
:10B244007910800479087D007E007F003392D55008
:10B254000312B2B8EC33400FEF33FFEE33FEED339D
:10B26400FDEC33FCD9EE22EECCF5F0747E29A2D5A8
:10B2740013FF92F7AEF022EF8EF0A2F7D2F73392DB
:10B28400D5C3947F5006E4FFFEFDFC2294204004C5
:10B2940074FF80F304CCFEE4FFFAE5F0CC6012C343
:10B2A400CC13CCCD13CDCE13CECF13CF0450EEDAC6
:10B2B400EC30D5D7C3E49FFFE49EFEE49DFDE49CFF
:03B2C400FC22E683
:10B2C700FC08E6FD08E6FE08E6FF22ECF608EDF6C8
:10B2D70008EEF608EFF622CFC513CFCEC512CECDB6
:10B2E700C511CDCCC510CC22E4F513F512F511F537
:10B2F7001022E493FCA3E493FDA3E493FEA3E49359
:10B30700FFA322C0E012B20912B11512B33D12B267
:10B31700F9D0E0C0E012B20912B33412B11512B27B
:10B327000912B2F912AF07D0E0D5E0E722AC48AD79
:10B3370049AE4AAF4B228C488D498E4A8F4B2274B7
:10B34700FF7809FFFEFDFCE52654F048F52622129A
:10B35700B3FD04A2E1927F1420E01590B47E74043B
:10B3670012B30A802912B3FD30E102B27F20E0EB6D
:10B377008C4C8D4D8E4E8F4F90B492740412B30A3D
:10B3870012B209AC4CAD4DAE4EAF4F12B115307F76
:10B3970004EF6480FFEE33EF337001FF2212B3FD39
:10B3A700C0E08C4C8D4D8E4E8F4F90B4B674031207
:10B3B700B30A12B209AC4CAD4DAE4EAF4F12B11538
:01B3C700EC99
:10B3C800C54CFCEDC54DFDEEC54EFEEFC54FFF90DB
:10B3D800B4A6740312B30AD08212B209AC4CAD4DB4
:10B3E800AE4EAF4FE58230E00712B18DB27F809D3F
:10B3F80012B18A8098EE33EF3324605007D0E0D042
:10B40800E002B346EFA2E7547F927FFF12B2097CB5
:10B41800837DF97E227F3E12B115EE33EF3324810E
:10B42800501012B20912B27B12B240EFB2E7FF120B
:10B43800AF07EE33EF33602A2403F8C313FFEE920D
:10B44800E7FEE82481E4501A12B20912B27BEF0435
:10B45800C2E0FCF58212B248EFB2E7FF12AF07E58F
:10B468008203FAEE33EF33600B148FF0A2F713FF69
:10B47800EE92E7FEEA2283FA703AE4E9AABCF8E021
:10B48800813EE6E99DBF0000803F1A3C2839666985
:10B4980099BBE335A33DE75D25BFDB0FC93FCCDB97
:10B4A8008D41EE3649C43F91C9453DF8B0C500000D
:10B4B800803F34F517C373FA2F45DDFD0AC6EF2523
:10B4C80013FFEE3512FEED3511FDEC3510FC02B21E
:10B4D80028C3EF9513FFEE9512FEED9511FDEC953F
:10B4E80010FC02B228EFF88513F0A4FFE513C5F0AD
:0AB4F800CEF9A42EFEE435F0CDFAE3
:10B5020088F0E512A42EFEED35F0FDE433CC851370
:10B51200F0A42CFCE5128AF0A42CFCE51189F0A41D
:10B522002CFCE51088F0A42CFC89F0E512A42DFD7A
:10B53200EC35F0FCE51188F0A42DFDEC35F0FC8A29
:10B54200F0E513A42DFDEC35F0FC02B228E4CCF8B2
:10B55200E4CDF9E4CEFAE4CFFB75F020C3E5133372
:10B56200F513E51233F512E51133F511E51033F554
:10B5720010EF33FFEE33FEED33FDEC33FCEF9BEEC9
:10B582009AED99EC98400CFCEF9BFFEE9AFEED9938
:10B59200FD0513D5F0C622C2D5EC30E705B2D512AF
:10B5A200B2B8E51030E70DB2D512B5BC12B54F12E4
:10B5B200B2B8800312B54F30D515C3E49513F51315
:10B5C200E49512F512E49511F511E49510F51022A7
:10A67C00E57124885002D2191256DC8E4712D1E7AC
:10A68C00129189125A98305E0F125A36128878122B
:10A69C00596712BFED12425412393A1247FB103669
:10A6AC0029201F1C301219E412A80212A81712A993
:10A6BC001712A93930510302A9C312AC94205109C5
:10A6CC00C251E4F552F545F5442275A70075830790
:10A6DC00E559C454F0F582E0F538A3E0F518A3A3CE
:10A6EC00A3E0F51E74FF12A8021256DC8E1C8F1B01
:10A6FC007510DF751100E51164B4700612A7CD75E5
:10A70C00111012A79A4028AE1CAF1B1257642032AE
:10A71C001EAC03AB027A0C125371ED701275A700CC
:10A72C00758304851182ECF00583E510F00511D5D5
:10A73C0010C412A7CD75C70375C6E075A7049005A4
:10A74C00007F0412A788DFFB75A700122B83125A17
:10A75C0036E4F5A7F8F559758307E8C4F582E0658A
:10A76C00387011A3E06518700BA3A3A3E0651E70ED
:10A77C000388592208C3E5589850DC22E0F5BCE068
:10A78C00F5BDE0F5BEE0F5BF124EE605C622E510BC
:10A79C0075F004A4F5C685F0C775B901E5BC334066
:0BA7AC001F05C605C675B90185BE6417
:10A7B70085BF6505C675B90185BC6685BD6785BE5C
:10A7C7006885BF69C322E51124FE502E75A7007F57
:10A7D70010AE111E7583048E82E0FD1582E0CDB5A3
:10A7E70005005012F00582CDF00583E0FD1582E0EB
:10A7F700CDF00582CDF0DEDCDFD72275A7549004BB
:10A807000005A79005007FB4F0F0DFFC75A70022D4
:10A8170012BE41C2517B077AFFE4FFF5A7900400FF
:10A8270012A8FDED244C4035EC603075A7008D82F1
:10A8370005A712A8C37583058D82E02410401CF07C
:10A8470005A7E02CF0500505A7E004F0BA000CBB03
:10A857000009D251EF24DC50027F23DFC3EA6005F1
:10A8670012A8768006EB600312A8AE75A700223007
:10A87700E0047553082230E1047553182230E204CE
:10A887007553282230E3047553382230E404755396
:10A89700482230E5047553582230E6047553682280
:10A8A70030E7037553782230E0047553882230E18E
:10A8B700047553982230E2037553AA22ED54F0C46D
:10A8C700232390A8CD735302FE225302FD22530285
:06A8D700FB225302F722F0
:10A8DD005302EF225302DF225302BF2253027F2283
:10A8ED005303FE225303FD225303FB225303FB228A
:10A8FD0012BD7912BC07E4F5F7C2B2C2B2ADF7F5DD
:10A90D00F7C2B2C2B2ACF7D2B22290050078B4E071
:10A91D006015FD54F0C4CD7C00540FFE1583E0FF8F
:10A92D0012546FEFF005830582D8E4227583047805
:10A93D00FF088882E060FAF5D38812E512244C50A6
:10A94D00012285D3D288D4881279FF0512E51260D1
:10A95D00F00908E875F0B484A8F08882E060ECF5A1
:10A96D00D3B9000280D5B9230050D0C395D292D16E
:10A97D005002F40409FEE4FFFCAD0112547C740195
:10A98D00FA25D475F0B484A8F0AC06AB0712536366
:10A99D00EB30E7010CE5D22C30D1029C9C8882F083
:10A9AD000AEAB501DCE512244C50012285D3D2858B
:10A9BD0012D4A812809390040012AA828C068B05E3
:10A9CD0012AA82E4FFF512F5118C148B13C3ED9BC3
:0EA9DD00F9EE9CFA4012E51199E5129A500A23
:10A9EB008C148B138A1289118F528F82E0F9C3ED6D
:10A9FB0099FDEE9400FEE582245A5002244C75F02A
:10AA0B00B48485F082E0FA2DFDEE3400FEEB9AFB68
:10AA1B00EC9400FCE92BFBEC3400FC0FBFB4B0E56D
:10AA2B005224D3400224B4F552C3E51333FBE5148F
:10AA3B0033FCE511FE2BFBE512FF3CFC1254D1E974
:10AA4B00F890AA9493F511FDEBF513FFECF514FEBA
:10AA5B007C0012546F8F44E890AB9493FAAB13AC19
:10AA6B001412539AAF03AE04AD117C0012546FEF66
:10AA7B007002F552F545227C007B007F5AE02BFBE0
:10AA8B00EC3400FC0582DFF522B4B4B4B4B4B4B436
:10AA9B00B4B4B4B4B4B4B4B4B4B4B4B3B3B3B3B370
:10AAAB00B3B3B3B3B3B3B3B3B2B2B2B2B2B2B2B273
:10AABB00B2B1B1B1B1B1B1B1B0B0B0B0B0B0B0AF83
:10AACB00AFAFAFAFAEAEAEAEAEAEADADADADADAC9E
:10AADB00ACACACACABABABABAAAAAAAAA9A9A9A9C3
:10AAEB00A9A8A8A8A8A7A7A7A7A6A6A6A5A5A5A5F0
:10AAFB00A4A4A4A4A3A3A3A2A2A2A2A1A1A1A0A027
:10AB0B00A0A09F9F9F9E9E9E9D9D9D9D9C9C9C9B60
:10AB1B009B9B9A9A9A99999999989898979797969F
:10AB2B0096969595959494949393939292929191E2
:10AB3B0091919090908F8F8F8E8E8E8D8D8D8C8C22
:10AB4B008C8B8B8B8A8A8A89898988888887878767
:10AB5B0086868685858584848483838382828281AD
:10AB6B0081818080807F7F7F7E7E7E7E7D7D7D7CF0
:10AB7B007C7C7B7B7B7A7A7A797979787878777732
:10AB8B007776767675757574740002030506080979
:10AB9B000B0C0E101113141617191A1C1D1F212242
:10ABAB00242527282A2B2D2E303133343637393AAA
:10ABBB003C3D3F404243454648494B4C4E4F50521B
:10ABCB0053555658595A5C5D5F606163646667689C
:10ABDB006A6B6C6E6F707273747677787A7B7C7E2F
:10ABEB007F80818384858688898A8B8D8E8F9091D7
:10ABFB00929495969798999B9C9D9E9FA0A1A2A499
:10AC0B00A5A6A7A8A9AAABACADAEAFB0B1B2B3B471
:10AC1B00B5B6B7B8B9BABBBCBDBEBFC0C0C1C2C365
:10AC2B00C4C5C6C7C7C8C9CACBCCCCCDCECFD0D074
:10AC3B00D1D2D3D4D4D5D6D7D7D8D9DADADBDCDC9A
:10AC4B00DDDEDEDFE0E0E1E2E2E3E4E4E5E5E6E7DA
:10AC5B00E7E8E8E9EAEAEBEBECECEDEEEEEFEFF030
:10AC6B00F0F1F1F2F2F3F3F4F4F4F5F5F6F6F7F79D
:10AC7B00F8F8F8F9F9FAFAFAFBFBFBFCFCFDFDFD21
:10AC8B00FEFEFEFEFFFFFFFFFFC251E4F544F8148A
:10AC9B00FB900400A9007C0FC2D112ADAFE82405D4
:10ACAB00F8B8B4F08B13E5122403FA244C5001FAD4
:10ACBB00BBFF012275112C8A1912ADE68F16203DB0
:10ACCB0012AA1975112312ADE68F15751600303DBA
:10ACDB00E2801175112312AD8E751500303D05E81C
:01ACEB002F39
:10ACEC0013F51575111212AD8E751400303D05E873
:10ACFC002F13F514EA2404F552244C5002F552E4B7
:10AD0C00F51AF51BF51CE516600AFB7A00AF137EED
:10AD1C00FF12AD54E515600AFB7A4FAF137EFF129C
:10AD2C00AD54E516600DFB7A00E5146006FF7ECF8E
:10AD3C0012AD54AE1CAF1B7C00AD1A12546F8F4574
:10AD4C00EF2513F544D25122EFF5F0A4FCADF0EB56
:10AD5C00F5F0A49CFCE5F09DFDEB8AF0A4FAABF0B9
:10AD6C00EF8EF0A49AF8E5F09BF9E833F8E933F9A3
:10AD7C007B00125515051AE51B2BF51BE4351CF54C
:10AD8C001C22EA2511F9244C5001F9C2D112ADADA7
:10AD9C00303D428F00C3EA9511F9500324B4F9D227
:10ADAC00D17C09E4FDFEFF8982E060062FFFE43EC2
:10ADBC00FE0D09B9B4027900DCEDED20D118F51EB9
:10ADCC0024FE923D500F12547CEFB50300500685C3
:10ADDC001E1FFB881222F51D80E612AD8E203D430E
:10ADEC00740212AE8512AD8E203D38740412AE8DF5
:10ADFC0012AD8E203D2D740612AE8512AD8E203D07
:10AE0C0022740812AE8D12AD8E203D17740A12AE4C
:10AE1C008512AD8E203D0C740C12AE8D12AD8E20B1
:10AE2C003D0122C3E89F605088148F158A16400894
:10AE3C001ABAFF0A7AB380060ABAB4027A0012ADC3
:10AE4C008E303D34C3E89FF9602EC3E5149515FB95
:10AE5C006930E7D4E930E703F404F9EB30E702F4A6
:10AE6C0004C3995002AA16E5142515C82F28FFE42F
:10AE7C00FC33FE7D0412546F222AFA244C5001FA42
:0BAE8C0022C3CA9AFA500324B4FA2231
:10BBCE00758000C2B212DE08D2B275F830227580CE
:10BBDE0000C2B2F5F7C2B2C2B2D2B222758000C2B2
:10BBEE00B2F5F7C2B2C2B2856CF7C2B2C2B2856B01
:10BBFE00F7C2B2C2B2856AF722758000C2B275F77B
:10BC0E0003C2B2C2B2856FF7C2B2C2B2856EF7C2BC
:10BC1E00B2C2B2856DF72212BC5E740612BBDC7422
:10BC2E000212BBEA8FF7C2B2C2B2D2B222909F5DAD
:10BC3E007F631276F012DD12D214120E9412766E0B
:10BC4E00124EE612BC5E740612BBDC74C712BBDC6D
:10BC5E0012BC6440FB22758000C2B275F705C2B2F9
:10BC6E00C2B2C2B2C2B275F705C2B2C2B2C2B2C2DB
:10BC7E00B2E5F7D2B2A2E022120E9485BF6C85BE59
:10BC8E006B756A00E56B7015E56A701112BC5E7417
:10BC9E000612BBDC74D812BBEAD2B2D21F22E54B1D
:10BCAE000475F03C8485F04B12BF69852E72E55FFA
:10BCBE00030354C0F8E55E543F28F57C305501224D
:10BCCE0012BD0312BC6440F7E54C60F312BC5E1269
:10BCDE00BD1A12BCE880F112BC5EC21F740612BB04
:10BCEE00DC740212BBEA787086F708B880FAD2B21A
:10BCFE0012BD37808F787075A704758304E54CC428
:0CBD0E00F5827F10E6F0DFFC054C801988
:10BD1A00787075A704758304154CE54C30E701E487
:10BD2A00C4F5827F10E0F6DFFC75A70022741025A7
:10BD3A006A54F0F56AE4356BF56BE4356C540FF52B
:10BD4A006C22E54B75F010A4256A54F0F56AE5F00B
:10BD5A0080E4E56A24F054F0F56AE56B34FFF56B8C
:10BD6A00E56C34FF80D7E56A24FF80ECC380EBE5FD
:10BD7A006D24F054F0F56DE56E34FFF56EE56F3421
:10BD8A00FF540FF56F2212BDE812BE10C22DC25425
:10BD9A00C255E57F7002D255147002D254E54A307A
:10BDAA00E00122B4061C20540D12BD5C12BEB8126A
:10BDBA00BF4812BF802212852F7E0412DE00754A08
:10BDCA00012220550D12BD3712BF2712BF6912BEBC
:10BDDA00912212852F7E0412DE00754A0522740311
:10BDEA0012BBEA7870E4F5F7C2B2C2B2A6F708B895
:10BDFA0080F3D2B222740312BBEAE4F5F7C2B2C2EC
:10BE0A00B2E5F7D2B222E575F8541F30E40244E0F5
:10BE1A00F57585722EA2779226E57C543F30E502AD
:10BE2A0044C0F55EE57C54C02323F55FE57FC2E795
:10BE3A0079BCF709A77E22856C6F856B6E856A6D62
:01BE4A0022D5
:10BE4B00856F6C856E6B856D6A22E4FEFF740775DA
:10BE5B00A704F5838E8274FFF0DFFD75A7002274B3
:10BE6B00067E007FB012BE5AE4F55AF55B2275A729
:10BE7B0004758306E55A600A75F00A84E5F07002D2
:10BE8B00740AC4F58222307720E55A240240020559
:10BE9B005A12BE79E55AF0E573F0E574F0E575F0EA
:10BEAB00E576F0E577F0E578F075A700223077F9C5
:10BEBB0012BE797F1074FFF0DFFDE55A24F55003B5
:10BECB0012BEE3155AE55AB4FF02055AC3E55A955B
:10BEDB005B50D6755B0080D112BE417F0A056D05A4
:10BEEB006D12BC07E4F5F7C2B2C2B2E5F7D2B230BD
:10BEFB00E704DF02800512BD7980E2056D12BC07F5
:10BF0B0012BE79E55A24F6F07F06E4F5F7C2B2C209
:10BF1B00B2E5F7F0DFF4D2B275A70022053FE53F9B
:10BF2B00B43C17753F00053EE53EB43C0D753E0035
:10BF3B00053DE53DB41803753D00024ABB153FE5D1
:10BF4B003FB4FF17753F3B153EE53EB4FF0D753E05
:10BF5B003B153DE53DB4FF03753D17024ABB05425A
:10BF6B00E542B43C0F7542000541E541B43C057513
:0CBF7B0041000540221542E542B4FF0FD2
:10BF870075423B1541E541B4FF0575413B1540221C
:10BF9700AC40AB41A842EC75F03CA42BFBE435F078
:10BFA700FC7A3C125363EB28FBE43CFC22AC3DAB30
:10BFB7003EA83F80E178AE8604AB3EE53FC313F869
:10BFC700800C7800120E5DE5BE75F005A4FBE5BF99
:10BFD70075F03CA42BFBE435F0FC7A1E125363EB9F
:10BFE70028FBE43CFC2212BFC9AE04AD0312BFBC60
:10BFF7008C148B13120E67E5BFFF24F650027F01E6
:10C00700E5BE75F096A4AAF0F9C3ED9513FBEE957E
:10C0170014FC924E4B701120110E30480B75364BA5
:10C027003003037536FFD22E304E02DF1F7A02121D
:10C03700536375A7009004EEECF0A3EBF0C3E5BFE4
:10C047009F04BF0102D2E79005CBF022ED29FDEE58
:04C057003AFE80B578
:10DDED0012DDF612DDF612DDF67E0480067E02806F
:10DDFD00027E017F0080087F6480027F017E00EF3C
:10DE0D004E6012E4FD0D1D0DEDC394AD40F7EF1FF7
:10DE1D0070ED1E80EA22753500C200C201C20222D9
:10DED400F5D8D2DCE5F520E7FBE5DA540FFEAFD93F
:04DEE40075D80022CB
:10DADB007F767E06909C7E127702740412DED47CD5
:10DAEB00007D5212546FEFF875F00A84C0F07F7608
:10DAFB007E2312D4C17E29742E12D4D47E2ED0E074
:10DB0B0012D4C17E35745612D4D47F6B7E1190DB48
:10DB1B004412D500E824E04001220423F824E75006
:10DB2B0002781812DB34D8FB227F6CE82411FE79C3
:10DB3B000512DE2D0E0FD9F922071DFFFFFFE08026
:10DB4B00000020C0000038E0000008F0000038F8AA
:07DB5B00000020FFFFFFE0C6
:10DB620012DB8A30E6022409540F75F00AA4F51577
:10DB720012DB8A30E6022409540F25152212DB8AB1
:10DB8200540F2275F000800875F044800375F00789
:10DB9200E4206D09D5E0FAD5F0F7D24C229247C2C3
:10DBA200ACE54F623885504FA26E926D859950C296
:10DBB2006FD2ACC24CA2472212DBC4C4FA12DBC43D
:10DBC2002A2212DB8A20E603540F22540724092258
:10DBD200E612DBD918E608FAC412DBDFEA540F4476
:10DBE20030F924C6E950112407800D75F00A84C06B
:10DBF200F012DBF8D0E0443030530975F00085E0D4
:10DC0200E0D5F0FA3099FDC299F599623822E538EB
:10DC120080F2E53812DBD9800812DBFAE53812DB34
:10DC2200FA740D12DBFA740A80CE744012DBFA74B5
:10DC32004080C5742C80C1742E80BD75380080B8B8
:10DEFA0085A0835383FE438380858384F0758400E1
:01DF0A0022F4
:10D9890074A212DEFA74A112DEFA74A612DEFA7417
:10D99900A412DEFA74C012DEFA742512DEFA12DA63
:10D9A9001975C70375C6FC75B90112B5D274081289
:10D9B900DED4EE75F020A4FEEF54F80303032E2401
:10D9C90092C313FE24EA50027E16EE90DA029325E2
:10D9D900BCFE24E6501F24E8401B748112DEFAEED7
:10D9E90012DEFA12DA26744012DEFA742F12DEFA07
:10D9F90074AF02DEFA7E2680E1F7F7F8F8F9FAFB50
:10DA0900FCFDFEFF00000000010102020203030306
:10DA1900A8BCA9BDAABEABBFACC7ADC62288BC898C
:0ADA2900BD8ABE8BBF8CC78DC622DC
:10DD1200C006C007C5F075A7019000007EB7E58C6C
:10DD2200240340FA12DD341EBEAFF3C5F0D007D093
:10DD3200062275A700EE12DEFA741012DEFA7404DF
:10DD420012DEFA85A08343838185838475A7517F80
:10DD520020E0F0E0F0E0F0E0F0DFF6E4F5A7F58493
:01DD6200229E
:10DEE80075A711900000E4C583F0C58330E2F8F50A
:02DEF800A7225F
:10DE2D00EF20E723EE20E71F20E61C05A7C45403CF
:10DE3D00F583EE5408C42FF582EE5407240983F5BB
:10DE4D00F0E045F0F005A722804020100804020103
:10DE5D00EF20E723EE20E71F20E61C05A7C454039F
:10DE6D00F583EE5408C42FF582EE5407240983F58B
:10DE7D00F0E055F0F005A7227FBFDFEFF7FBFDFEC9
:10D48100FDA42582F582E5F03583F583ED229060D8
:10D49100AC7A0475F00512D4817D05805E7A058031
:10D4A100027A04547FC0E0C083C082C3942050013B
:10D4B100E490605C12D494802E9061BA7A05800564
:10D4C1009062777A0675F00712D4817D07802C7AF5
:10D4D1000580027A06C0E0C083C082C39420500157
:10D4E100E490620712D4C6D082D083D0E022905F4C
:10D4F100D075F00A12D4817D0A7A07C2D18002D296
:10D50100D1C0A7C082C083C007C006C0E030D10926
:10D5110075A704E493FDE493FAEEFB75A704EBFE13
:10D52100EAFC7901D9067908E493F5D4E5D423F529
:10D53100D420E01612DE5D0EDCEA0FDDE1D0E0D092
:10D5410006D007D083D082D0A72212DE2D80E890AA
:10D551005F1075F00E12D4817D0E7A0812D4FC9002
:10D561005FB875F00212D481E493FDE4A393FACE7F
:10D571002408CE7C0812D57D7C06AD02ED23FD206A
:0ED58100E00712DE5D0FDCF42212DE2D80F7D3
:10D36C00F5D2C2D58036F5D2D2D58030F5D224F69E
:10D37C0050090E0E24A650030E0E0EE5D2F5D275F2
:10D38C00F0648485F0D3C2D57009D2D5742012D440
:10D39C00D4800312D4C1CE2406CEE5D375F00A8412
:10D3AC0085F0D3700A30D507742012D4D4800312C0
:10D3BC00D4C1CE2406CEE5D312D4C1E5D222F5D207
:10D3CC0075F0648485F0D3C2D58022F5D2C2D580A5
:10D3DC0025F5D2D2D5801FF5D275F0648485F0D3B3
:10D3EC00C2D57009D2D5742012D4D4800312D4BA09
:10D3FC00CE2405CEE5D375F00A8485F0D3700A30BF
:10D40C00D507742012D4D4800312D4BACE2405CEFE
:10D41C00E5D312D4BAE5D222F5D2C2D58035F5D2F5
:10D42C00D2D5802F30E70DF404C0E0742D12D4A2B5
:10D43C000E0ED0E0F5D275F0648485F0D3C2D570B1
:10D44C0009D2D5742012D4A2800312D48FCE240416
:10D45C00CEE5D375F00A8485F0D3700A30D5077405
:10D46C002012D4A2800312D48FCE2404CEE5D31282
:05D47C00D48FE5D2226F
:1076E700909F5D1276F002DD127E00800E7405FE1B
:1076F700F51EE4FFF51DF51F203C3375A700E49345
:10770700700122A3B40204051D8003B4010A051FFA
:10771700EF2409FFAE1E80E612D4D47D06B44002E2
:107727007D03B421027D02EE2DFE80D27E0075A777
:1077370000E493700122A3B40204051D8003B40181
:107747000F051FEF2407FFAE1E80E612D49E8008A8
:10775700B45B0050F612D4A20EB4210280D30EB44B
:10776700400280CDB42C0280C80E0EB45F0280C1E7
:10777700B45B0040BC0E0E80B8E60812D4D4EE24E9
:1077870006FED513F422909CAC307409909CB0305F
:107797007303909CB502770275F019D5E0FDD5F01B
:1077A700FA12484F12DC2C744F12DC3D744B12DC7A
:1077B7001BC322C2501277FE12484FD2AC12DB8590
:1077C700304C1212DB85304C0C12DB85304C06D264
:1077D70050C2ACD322B440E512DB8AB4400312DBBB
:1077E7008AB44FED12DB8AB44BE712DB8A12DB8ACD
:1077F70012DB8AC2ACC32230530975F008D5E0FD0D
:10780700D5F0FA227F0575F019D5E0FDD5F0FA120B
:10781700484F12DC2C745712DC3D745012DBFA749B
:097827008112DBFAE56312DBFAC1
:10783000E56212DBFA78D0E612DBFA08B8D7F8E690
:10784000F8795F30E702792FE912DBFA12DBFA12DE
:10785000DBFA12DBFA745812DBFA744312DBFAE437
:1078600012DBFAE8C2E775F00A84C425F012DBFAED
:107870007864E612DBFA08B869F8E612DC1B1277C6
:10788000BA400122DF02800A20508B75F000808010
:10789000D250C2ACD3221277FEC25012484FD2ACA3
:1078A0002002EF12DB85204CE7B440F412DB8AB4EF
:1078B000400312DB8AB457DAF53812DB8AB450D2AF
:1078C00012DB8A12DB8AF56312DB8AF56278D0124A
:1078D000DB8AF924A0500353015FE924E0400279D8
:1078E0005FA60108B8D8E8780612DB8AD8FB12DB5D
:1078F0008AFC53040FC4540F75F00AA42CFC249C7A
:1079000050027C0078D78601E4B92F02D2E72CF62A
:10791000786412DB8AF608B86AF812DB8AE5386008
:107920000302789212DB8A12DB8AC2ACC32290A3D4
:10793000468003909FA27F2012773312DD1202DD72
:10794000FE753400C26B1279FD12DDFE127DADE5CD
:1079500016600312795902025912800F121E461244
:10796000DD1210002010010280F8127E1850131250
:107970001E5112792E10000D10010280F8121DF315
:0579800080D7127B9D81
:1079850022C26BD22775480A122B77753400127EF6
:10799500E5C26A1233CF106A0512024A80ED12025F
:1079A5004A127D3F127E97127EF178D0E6642660FA
:1079B5004412800F121E4612DD121000381001020B
:1079C50080F8127E18501BE965156018121E5112B9
:1079D500792E12DDF610001D10010280F8121DF33C
:1079E50080BCD26B127EC3751607855917122BF012
:1079F5007535008096020259127DAD127A1F127EEE
:107A0500F17F19127A3990A3707E121277357E2391
:107A1500E51602D44090A4BA80EF7862E4127A3079
:107A250078D0745F127A3018E4F6227F08F608DF02
:107A3500FC227F7B7E007810742012D4A2CE240411
:107A4500FED8F5227F197E081277357E28909F840F
:107A5500305303909F89027735C26B127A1F127AD1
:107A650069020259C251127EF190A368127A491235
:107A75001E19127DAD7F20127A0812DD12E51670EF
:107A85000512DDF3803675A6FF3051031277A81273
:107A9500484FD2AC200025306DFA127899400C126F
:107AA5007E184011127B9DD25180BB105003127974
:107AB50033C25180D1D25112792E80CAC2AC22D2A2
:107AC5002775480A122B77753400C26B127EE5C202
:107AD5006A1233CF106A0512024A80EB12024A126B
:0D7AE5007D3F127E97127EF1127AF550DA85
:107AF200020259909F9D127A49121E2B12DD12C367
:107B020010001310010510020E80F412780B4001D0
:107B12002212793380DDD3C2AC22D227C26B7548E0
:107B22000A122B77753400127EE5C26A1233CF1027
:107B32006A0512024A80EDD26B127D3F127E9712C5
:107B42007D6775B901E5BCB2E7F5BC124EE6751664
:107B520007855917122BF080CB127DADE516601FF9
:107B620078D0E53D127B8EE53E127B8EE53F127B9F
:107B72008E765A08765F12C805127EC3027D7E7F1A
:107B82003E7E11909F7412770202DD1275F00A8414
:107B92004430F608E5F04430F60822D26B127EC378
:107BA200127D7EE51775F01084240AF54824E8500A
:107BB2000375480A122B838558592275320012BE6A
:107BC2005575A704900700751500127D6775B901F8
:107BD200E5BC20E705E515F0801004600D648260C5
:107BE2000975BCFF75B90575B9020515E51524209F
:107BF20050D8E58224FE4003027C96A882187F00BA
:107C020075A7007583078882E0FE75F004A4127DD3
:107C120012A9BCAABDABBEACBF1582E0FD75F004D3
:107C2200A4127D12C3E995BC404C7052EA95BD4046
:0D7C320045704BEB95BE403E7044EC95BF95
:107C3F004037703DEE75F004A404127D12A9BCAA62
:107C4F00BDABBEACBFED75F004A404127D12C3E949
:107C5F0095BC4015701BEA95BD400E7014EB95BE98
:107C6F004007700DEC95BF5008EEF00582EDF01552
:107C7F0082E5826009C3EF95825003027C0A0FC32D
:107C8F00E89F4003027C0275A70490070075C703A5
:107C9F0075C6A8E0F5BCE0F5BDE0F5BEE0F5BF7533
:107CAF00B90575B90205C6E58224204006E5C6244C
:107CBF002050E00875C70375C68075B901E5BC1281
:107CCF007CFCF5BCE5BD127CFCF5BDE5BE127CFC71
:107CDF00F5BEE5BF127CFCF5BF75B90205C6E5C65A
:107CEF00245850D6E5320470FB75A70022B4FF016B
:107CFF0022F975A704900700E582686005E06970B6
:107D0F00F7E922F5C685F0C775B901E5BC645F7068
:107D1F000375BC27E5BD645F700375BD27E5BE64C1
:107D2F005F700375BE27E5BF645F700375BF2722C1
:107D3F0075C703E54875F004A42480F5C6E55975A9
:107D4F00F00484A8F00825C6F5C675B901A9BCAA28
:077D5F00BDABBEACBF8615F1
:107D660022E515242050037515DFE51575F004A4EA
:107D760054FCF5C685F0C722E51724204028E517F0
:107D860075F00484A8F00824A8F5C675C70375B96C
:107D960001A9BCAABDABBEACBFA61589BC8ABD8B6A
:107DA600BE8CBF124EE622E4F516F51579FF127D5C
:107DB6006775B901E5BCB4FF040516A9150515E5F7
:107DC60015242050E9891579FF75C70375C6A8756E
:107DD600B90109E5BC04601B09E5BD04601509E5A8
:107DE600BE04600F09E5BF04600905C6E5C6242088
:107DF60050DD09891722751600751501127D677504
:107E0600B901E5BC20E70205160515E51524205045
:107E1600EB227900E975F004A454FCF5C685F0C799
:107E260075B901E5BC20E73078D066702B08E5BD52
:107E360066702508E5BE66701F08E5BF6670190501
:107E4600C675B90108E5BC66700E08E5BD66700822
:107E560008E5BE667002D32209E9242050B6C32283
:107E6600127E86127E6EA8017F08E0F608DFFB22EE
:0B7E7600127E86127E7EA8017F08E6C7
:107E8100F008DFFB2278D0796275A704758307EBD0
:107E9100C454F0F58222127D6778D0127EB1E5BC20
:107EA100F9C23C20E702D23C127EB17862127EB167
:107EB10075B901A6BC08A6BD08A6BE08A6BF0805DF
:107EC100C622127D6778D0127ED3127ED3786212D9
:107ED1007ED386BC0886BD0886BE0886BF08124EC2
:107EE100E605C622125A3612DEE812866E02DD124D
:107EF10012DEE87F007E0990A3551277027F0A7E89
:107F010012E5150412D3787F1412C9EF121DF37F05
:107F1100277E0875130778D0127780E6793E30E71F
:107F210002792F7E34E912D4D47F3D7E0190A4D60C
:107F310012773520311B3030031291A9C23B1281D7
:107F4100A1127F57D23B1281A1127F691281E88071
:107F51007C12C05B80E6C23B7F44745320170274DD
:107F61004E7E0012D4D48017D23B7F4F7457201716
:107F71000274457E0012D4D47E06E51E12D4C17E61
:107F81000CE51D12D4C17E12E51C12D4C17E1774FA
:107F91008112D4D47E1CE51B12D4C17E22E51A12B3
:107FA100D4C17E28742E302602742712D4D47E2D9B
:107FB100E51912D4C17E33E51812D4C17E393026B9
:0F7FC10007742C12D4D07E3BE53702D4C1742D47
:107FD000201702742B7F707E1512D4D4127FEC7E92
:107FE0003A12D3217E0190A5010277027E1BE51C87
:107FF00012D4C17E21E51B12D4C17E27E51A12D40A
:10800000C17E2DE51912D4C17E33E51802D4C11208
:10801000808D1280B812838F127EF11283E72017B1
:108020001E10021B1248F012C805128075121DFEA8
:108030007F347E2F12778D127F2A12DD1280E2129A
:108040001DF3203026203128C23B1281A11280CDA1
:1080500078661282A1D23B1281A11280E278691265
:1080600082A11281E812815C02834412927280F232
:1080700012C07080EDE57D75F01084AAF075F00AED
:10808000A42A547FFA78D7E654802AF6227F277EE6
:108090000879D08700C001D224B9D002C22412844A
:1080A0006ED001A70010230909EE2406FEB9D7E31C
:1080B0002219EE24FAFE80DB7E3479D7E7A2E7921C
:1080C0001712841B79D7E7A21792E7F722C224C2BE
:1080D0003B751E007F447E0012842B801E1023ED12
:1080E000802AD23BC2247F4F7E00128433D2247E6A
:1080F00006E51E128460F51E1023E7D2247E0CE5EF
:108100001D128460F51D303BD41023E1D2247E1271
:10811000E51C128460F51C1023E17E1CE51B128413
:0381200060F51BEC
:108123001023E67E22E51A128460F51A1023E87EF6
:108133002DE519128460F5191023E87E33E5181232
:108143008460F5181023E87E393026027E3BE5373C
:10815300128460F5371023E3227F707E1512842387
:10816300C2247E1BE51C128460F51CD2247E21E50B
:108173001B128460F51B1023E77E27E51A12846027
:10818300F51A1023E67E2DE519128460F5191023E4
:10819300E87E33E518128460F5181023E82278D7B7
:1081A300E6C2E775F00A847866F537303B057869EF
:1081B30085F03712821130262BE53775F003A404BE
:1081C3000475F00584FBE51975F00AA4251875F00C
:1081D30006A42BFBE435F0FC125585F537125585C3
:1081E300F5188B1922E563FC339217AB6250031227
:1081F30055F6305C0A7AD21253717840125513AE99
:1082030004AF037C277D1012547C8F1C8037E6FD5E
:1082130033921718860418860350031255FE7A0901
:10822300792778C01255108B1EADD3ACD2AB06792B
:10823300EA786012550E8B1DAF06AED27C177D70A7
:1082430012547C8F1CAF05AE047C037DE812547C72
:0F8253008F1BAF05AE047C007D6412547C8F1A24
:10826200ED75F00A84F51985F01822EC3392175057
:10827200031255F6751D30301786751D2D808178D5
:10828200427B607CEA800678407B207C4E12C13BB8
:108292007927781012550E8B1CAF06AED280AB3008
:1082A200262AE51975F00AA4251875F00AA42537BF
:1082B200FBE435F0FC7A051253638C068B077C00D5
:1082C2007D0312546F8E048F031281DBE51E75F05D
:1082D2000AA4251D75F00AA4251C75F006A4251B09
:1082E200FBE435F0FC7A0A125363EB251AFBE43CFB
:1082F200FC7A0A125371EB2519FBE43CFCE43DFDC8
:108302007A0A125383EB2518FBE43CFCE43DFD3072
:1083120017031255FEA60518A60418A60378D7E679
:10832200A2E7923DC2E775F00A84FCABF0303B0E47
:10833200AB37EC75F00AA42BA23D92E7F622AC37DC
:1083420080F012835F305C0A7A4012537178D21245
:1083520055133017031255F68C638B622212836F0A
:108362007A0A125363EB2518FBE43CFC22E51C75E8
:08837200F00AA4251B75F00AB6
:10837A00A4251AFBE435F0FC7A0A125363EB25199B
:10838A00FBE43CFC221283C112DDFAC202C22312B0
:10839A0083C110000810010510021B80F51031ED91
:1083AA0010300D102604D22680E3D230C23180DD8F
:1083BA00D231C23080D7227F3590A4BF1277339052
:1083CA00A4DD20300F90A4F920310990A4CE2026F4
:1083DA000390A4C61F7E1712770202DD127F357E34
:1083EA0001909F501277357F347E3A128510744E71
:1083FA0012D4D412DD1212DDFAC2027F347E3AD2CE
:10840A001775115975124E802675112E751227800F
:10841A001E75113E75122F801675112B75122D803F
:10842A000E75114E75125380067511457512571245
:10843A008510E511301702E51212D4D412DD12109C
:10844A00000810010510020B80F5D23C1017E3D288
:10845A001780DF02850B4430F812846AE8540F2231
:10846A00C2218002D221A22492229223128510E8EC
:10847A0030E709D23C7430302102745FF812D4D448
:10848A0012DD1210003410010510025D80F5D23C95
:10849A00102266102367B43909745F2021DF743013
:1084AA0080DBB45F04742D80D4B42D04744180CD74
:1084BA00B45A04743080C60480C3D23C30240610F7
:0F84CA002237102338B44104742D80B1B42D042F
:1084D900745F80AAB45F04743980A3B43009745AF4
:1084E90020219B74398097148094B48908D223E899
:1084F90012D4D4800DF8C223800874898001E8025F
:1085090084879085258003908521C007EF2408FF83
:1085190012D500D00702DD120205F8F802050000A5
:10DCB20075A70090DCE475F02D84C2D5C2D160173F
:10DCC200D2D1146007D2D514600DC2D1E5F093FC15
:10DCD200742D95F093FB22E5F093FB742D95F09350
:10DCE200FC220009121B242C353E474F58606870F5
:10DCF2007880888F969DA4ABB2B8BEC4CACFD4D95F
:10DD0200DEE2E6EAEDF0F3F6F8FAFCFDFEFFFFFFD5
:10DDAC00D23D8002C23DED8BF0A430E70205F0C3FA
:10DDBC00E895F020D50425F025F0FEED8CF0A4308C
:10DDCC00E70205F0C3E995F030D10425F025F0FF0A
:10DDDC00203D0B2487500122EF24CC40012202DE8F
:01DDEC002D09
:10D75000203A7A7E1C7F5312DE2D7F5912DE2D1E59
:10D760007F5712DE2D7F5512DE2D7E2312DE2D7F98
:10D770005712DE2D1E7F5912DE2D7F5312DE2D1F14
:10D780007E2012DE2D7F5A12DE2D7E1E12DE2D7FB0
:10D790005212DE2D120E67E5BD20E0143006117F17
:10D7A000357E1C90D80CE571700390D81602D50018
:10D7B000E5716018E57012DCB2781F79567D0912A8
:10D7C000DDB0303A0312D7DF0DBD16F3227E1C7F89
:10D7D0005390D7F512D500200CD612CA4B80C0C08A
:10D7E000060E30D5021E1E12DE2DD0061F30D102CD
:10D7F0000F0F02DE2D070700386C446C380005055A
:10D800002070D8702005057088A888700807103827
:10D810007CFE383838000807102844C6282838000D
:10C82A0090A50B7F717E23127735120E67E5BC7EC9
:10C83A003112D48F30121AC23C120E67E5BCFB7556
:10C84A00F00AA4F904FAC23D12BE4112CAC8303D28
:10C85A000122DAF712C9CF7C00EBF4042E4019AD9D
:10C86A000312546FEFA2D1203C077E237F6502D0CA
:10C87A00EEAE16AF1702C970AD0112546FEF12D1A6
:10C88A00DC203C077E237F6502D112AE16AF170269
:10C89A00C9947F567E0512C9FB7F3D12CA0E7F6F6F
:10C8AA0012CA0E12CA4B7E0A7F4112CA7E7E227FAC
:10C8BA005912CA7E2012012212BE41857A1D855E56
:10C8CA001C857B1B855F1A7AC0C23D12CAC4203DF3
:10C8DA005212C9CF7C007D1412546F74562F20D186
:10C8EA00029F9FFF24CB40028037EF2488500280AA
:10C8FA0030EA1475F00384FE12DE2DC3E51B957B26
:10C90A00FEE51A955F92D55004EEF404FEEEC313C9
:10C91A00FE24E0400C741F2E30D5029E9EFE12DECD
:10C92A002DDAA8227F5212C9407F5A12C9407517C0
:10C93A0053751600802B7E0012DE5D0EBE12F922A0
:10C94A007F157E28742012D4D47F1C7E2812DE5DC7
:04C95A000EBE40F9D4
:10C95E00223012E712C94A75171575162DD23C02F0
:10C96E00C843C23D6002D23D92D175F080305C0466
:10C97E00F5F08001A4A2E792D5E5F075F03284F8C7
:10C98E00E5F075F00584C0E0E5F0A2D533C0E0E82F
:10C99E00601E12D4C1EE2406FED0E0F8D0E012D410
:10C9AE00C1EE2406FE742C12D4D40E0EE802D4C1AD
:10C9BE007420303D07742B20D102742D12D4D480F4
:10C9CE00D4C3ED957AFFEC955EFE92D150031255CD
:10C9DE00E6227F1512C9E77F327E3E12DE2DDEFB88
:10C9EE00227E0912DE2D0EBE36F9227E0112DE2DBA
:10C9FE000E0EBE3FF8227E3312DE2D0EBE40F92201
:10CA0E007E047D1112DE2D0E0E0EDDF81F1F7E35FB
:10CA1E0090A514305C057E3190A51802773574050B
:10CA2E00305C097E32740112D48F74067E3612D4B5
:10CA3E008F7E3A740012D48F7E3D02D48F7F417E5A
:10CA4E001F7D0F12DE2D0F0F0FDDF8227F687D0385
:10CA5E0080047F677D0512DE2D0FDDFA227F667D55
:10CA6E000780F37E1F7F5012DE2D1F1FBF3EF82260
:07CA7E007D0A12DE2D0E0EF1
:10CA85000F0FDDF722203D07123C767003D23D22C1
:10CA9500056D12BC07E4F5F7C2B2C2B2ABF7F5F704
:10CAA500C2B2C2B2E5F7FA30E411EB251DF51DE47B
:10CAB500351CF51C0519EA30E3010ED2B280157854
:10CAC5000380027801203D07123C767003D23D2297
:10CAD500D8F3056DE56D2409F56D12BC07E4F5F78E
:10CAE500C2B2C2B2ADF7F5F7C2B2C2B285F71BF555
:10CAF500F7C2B2C2B2E5F7FCD2B2543F30E5024408
:0FCB0500C0CC54C02323F51AE56D24F6F56D223C
:10D677007E017F0990D6F512D5002051097E037FE0
:10D6870000743F02D4D4E4FEFFC3E54512CF46FD44
:10D69700940AED403D9464ED4002746312D3727EA8
:10D6A700017F09E552240575F02D84AAF075F00570
:10D6B700A4CA75F00B842A90D6E09312DCB2BCB8EA
:10D6C700027BB87D04EE2DF8EF2DF90D12DDACDDF0
:10D6D700FB227E0312D4C180C6000C1622222D39EC
:10D6E700444F4F5A66707C7C87939EA9A90009090D
:10D6F7000800410000000000888000000000410091
:10D707000800120E7BE5BCB4F8339004C3E0602C2C
:10D71700FA24F340277F137E0012DE2D0F0F12DE4F
:10D727002D0E12DE5D1F1F12DE5D0EDAEC7F147EFA
:10D737000012DE2D0E12DE5D0EBE12F5229005CC14
:09D74700E0C3941240F60480C70F
:10CF4600305D0A75F08AA42480E5F034002220744E
:10CF5600157F017E1190CFCE12D5007F0A7E0AE59D
:10CF66002E540702D3897F087E1190CFDE12D5009A
:10CF760020730C7F0A7E1712DE5D0E0E12DE5D7FB9
:10CF8600007E0BE57112CF4612D3787F0C7E11E539
:10CF960071602F0EE57064B4602864B475F0328455
:10CFA600C0F012D4BACE2405CED0E075F00584C008
:10CFB600F012D4BACE2405CED0E023302D010402DF
:10CFC600D4BA90886A027702070FFFFFC473BDAF19
:10CFD600A463B5FBCDE7FFFF030F0100FFFE03804F
:10CFE600306701227F357E00748812D4D4E5516003
:10CFF6001712CF4675F06484F87E06E5F012D3D793
:10D00600E860E07E0002D4C17E003074D63073162C
:10D0160079BCE7FC09E7FB12530B781D201704E6E1
:10D0260070011802D2A2909CB0027702202C012235
:10D0360090D03C02D500050EFFF0E01CF004F81C71
:10D04600FFF0301201227F637E00909CC712D5004C
:10D056007F1512C9E77F1F12C9E77F2912C9E77F2B
:10D06600177E06E53F30E00B90A528305C0390A5BF
:10D076003C80132074077E01909CE7800990A51DD3
:10D08600305D0390A532127702307306E54E6002DA
:10D09600154E205718E54EB40113120E8AC3E55CEF
:0DD0A6009560F5BCE55D9561F5BD124EE6A7
:10D0B3007F217E01E53F30E021305705909E0A80B5
:10D0C30016E54E7005909E16800D909CF212770225
:0BD0D3007E30E54E02D3DD1277022212
:10D2440012530B7F207E05751900781DC2D5E63078
:10D25400D51712D4BAEE2405FE18B818F17E1F743F
:10D2640063305C02748202D4D47005B8191880E269
:10D27400D2D5CE24FACE7484301702742D12D4D4AD
:10D28400EE2406FE80C8742012D4D080C8781C8096
:10D294000D7F007E23AC5EAB7A12530B781DC2D592
:10D2A400E630D50C12D4C1EE2406FE18B818F122CB
:10D2B4007005B8191680EDD2D53017E4CE24FACE15
:10D2C400742D12D4D4EE2406FE80D5742012D4D446
:10D2D40080D512530B781DC2D5E630D51612D48FE3
:10D2E400EE2404FE18B818F10E745E305C02742744
:10D2F40002D49E7005B8191680E3D2D53017DACE61
:10D3040024FCCE742D12D4A2EE2404FE80CB74200F
:10D3140012D4A280CBC23D12D32C0F0F0E0E746315
:10D32400305C02748202D4D412530B781DC2D5E649
:10D3340030D50C12D4EFEE2408FE18B818F1227080
:10D3440005B8191680EDD2D5301716740BCE24F813
:10D35400CE12D4EFEE2408FE80D5740C12D4EF80E4
:08D36400D5303DCB740A80E5D1
:10D820007F797E24E55F30E70122AC5F1CAB7B1281
:10D830005339E51B700E742012D4D4EE2405FE1269
:10D84000D86E800C12D86EE51B12D4BAEE2405FEF9
:10D85000E51A12D4BAEE2405FE742C12D4D40E0E9E
:10D86000E51912D4BAEE2405FE745E02D4D4742DE8
:10D87000201702742B12D4D4EE2406FE22E55F306A
:10D88000E70122AC5F1CAB7B125339E51B700E74B1
:10D890002012D4A2EE2404FE12D8C7800C12D8C7DE
:10D8A000E51B12D48FEE2404FEE51A12D48FEE2469
:10D8B00004FE742C12D4A20E0EE51912D48FEE249D
:10D8C00004FE742A02D4A2742D201702742B12D4E1
:06D8D000A2EE2404FE227A
:10D0DE007F097E2530040512D1D88028A275E57906
:10D0EE00C23D6002D23D92D175F080305C04F5F005
:10D0FE008001A4A2E792D5E5F075F03284F8E5F050
:10D10E0075F00584C0E0E5F0A2D533C0E0E8602AF2
:10D11E0012D4EFEE2408FED0E0F8D0E012D4EFEEF9
:10D12E002408FE0F0FE52B5403701F746012D4D425
:10D13E001F1FEE2404FEE802D4EF740C303D06747B
:10D14E000A20D1010412D4EF80C9205904742E8014
:10D15E00DC205804747F80D5748080D13004051291
:10D16E00D1D88028A275E579C23D6002D23D92D118
:10D17E0075F080305C04F5F08001A4A2E792D5E54D
:10D18E00F075F03284F8E5F075F00584C0E0E5F056
:10D19E00A2D533C0E07F3E7E1CE8602012D550D071
:10D1AE00E0F8D0E07F3E7E2812D5507F447E327468
:10D1BE002E12D4D47F3E7E37E802D550303DE07437
:10D1CE000A20D1010412D55080D59005CAE075F021
:10D1DE000A84F8E4C5F0C2D522301105E54AB4023E
:10D1EE0050C39006E9E0957AFB9006E8E0955EFC68
:06D1FE0050031255F6EC8F
:10D20400C31360047B63800FEB13FB249C40F52461
:10D214004F4004C20480079005CAEBF0D204900684
:10D22400E6E09006E8F09006E7E09006E9F0E55EB7
:10D234009006E6F0E57A9006E7F02212D22280DE2C
:10CB1400E54424F64001227800E552206607C395D7
:10CB240070500224B40475F00384F9E928FE24C487
:10CB34005001FE12CB5612CB621E12DE2DC3E998B1
:10CB4400FE5003243CFE12CB561E12DE2D08B81FE5
:10CB5400DA22EE2420FE24C250032402FE22E8241A
:10CB6400F1E8C2D55006D2D5E8F4241F23FF90CBB8
:10CB7400E493CF0493FAE545F5F0A4ACF0FB12532B
:10CB84009AE544F5F0A49BFBE5F09CFCEB2420FB28
:10CB9400EC3400FC12CBC5FAE5458FF0A430E70273
:10CBA40005F0E5F020D502F4042A75F005201903F8
:10CBB40075F00384FF24DF50027F20C374329FFF8B
:10CBC40022EC24F0500BEB2460EC340090CC349332
:10CBD40022EB33FBEC33FCEB33EC3390CC049322A9
:10CBE400FF00FF03FA0BF318EA2ADE40CF58BE73A6
:10CBF400AB8D96A880C068D64FE835F51BFD00FFC5
:10CC040000080B0E101214151718191B1C1D1E1FDB
:10CC140020212223242526262728292A2A2B2C2DA5
:10CC24002D2E2F2F303131323333343435363637DD
:10CC3400373839393A3A3B3B3C3C3D3D3E3E3F3F39
:10CC44004042444648494B4D4E505253555658590C
:10CC54005B5C5D5F60616364656668696A6B6D6E89
:10CC64006F7071727374767778797A7B7C7D7E7F4E
:10CC7400808182838485868788898A8B8B8C8D8E3C
:10CC84008F9091929394949596979899999A9B9C46
:10CC94009D9E9E9FA0A1A2A2A3A4A5A6A6A7A8A963
:10CCA400A9AAABACACADAEAFAFB0B1B1B2B3B4B492
:10CCB400B5B6B6B7B8B9B9BABBBBBCBDBDBEBFBFCC
:10CCC400C0C1C1C2C3C3C4C5C5C6C7C7C8C8C9CA11
:10CCD400CACBCCCCCDCECECFCFD0D1D1D2D2D3D45F
:10CCE400D4D5D5D6D7D7D8D8D9DADADBDBDCDDDDB5
:10CCF400DEDEDFDFE0E1E1E2E2E3E3E4E5E5E6E610
:10CD0400E7E7E8E8E9EAEAEBEBECECEDEDEEEEEF71
:10CD1400EFF0F1F1F2F2F3F3F4F4F5F5F6F6F7F7D8
:10CD2400F8F8F9F9FAFAFBFBFCFCFDFDFEFEFFFF47
:10CD3400E54524FD400122E552206607C395705065
:10CD44000224B40475F00384241FFE24C250032477
:01CD540002DC
:10CD5500FE12CD8FEEFD241EFE24C250032402FEDA
:10CD650012CD8FE544240275F00520190375F003F3
:10CD750084F4042432FF24EE500F12CD84AE051E38
:10CD85001E7C0512DE2D0EDCFA227F1512DE2D0F1C
:05CD95000FBF2DF82284
:10D58F007E00206615E5700475F0B484E5F075F043
:10D59F000384FE6004C3743C9EFE745312D5BA74A8
:10D5AF005712D5BA744E12D5BA74457F2F12D4A222
:10D5BF00BE00077E3C12D4A27E00EE240875F03C1C
:10D5CF0084AEF00F0F0F12DE2D0E12DE2D0F12DEB6
:10D5DF002D1E12DE2DEE240775F03C84AEF02230A6
:10D5EF00745C301259E54AB4040122B4060122E5F5
:10D5FF007112CBAE8F057C037E1E30662AE5700458
:10D60F0075F00384241EFE24C6501C24FB500424F2
:10D61F00038013C00612D636D0E024C67C01600604
:10D62F000C1460020C14FE12D6420EEE24C14002FE
:10D63F00DCF5228D0712DE2D0FEF24CE50F722E5F9
:10D64F0053206607C39570500224B40475F0038409
:10D65F00241FFE24C250032402FE12D66D0E7F2318
:08D66F0012DE2D0FBF2DF92280
:10DD6300AF177E00E53C12D36C7E0C742E12D4D414
:10DD73007E12E53B12D36C7E1E742E12D4D47E2405
:10DD8300E53A02D36C7E0E78ADE612D3D77E1874D3
:10DD93002C12D4D47E1B18E612D3D77E25742C12F2
:09DDA300D4D47E2818E602D3D77F
:10CD9A007F797E00E54012D3D77E0A743B12D4D045
:10CDAA007E0CE54102D3D77F797E16743B12D4D02C
:10CDBA007E18E53F12D3D77F797E0078AEE612D38C
:10CDCA00D77E0A743B12D4D07E0CE53E02D3D7300C
:10CDDA005EE52043E27F6D7E0078AEE612D3D77E11
:10CDEA000A743B12D4D07E0CE53E12D3D77F757EEF
:10CDFA000075F00A84E5F012D4EF0F0F7E08743A3A
:10CE0A0012D4D01F1F7E0DE53F75F00A84C0F012C0
:10CE1A00D4EFEE2408FED0E002D4EF851C1E851B59
:10CE2A001FAB1BAC1C305D0A7A1B1253717832128D
:10CE3A005513C3EB33FBEC33FC923D125342303DA6
:10CE4A00087409F51DF51CF51B7F75E51D60157E37
:10CE5A002412D4EF7E2CE51C12D4EF7E34E51B128B
:10CE6A00D4EF803D7E22E51C601912D4EF7E2AE5BC
:10CE7A001B12D4EF7F787E31742E12D4D07F75E5E1
:10CE8A001A8019E51B12D4EF7F787E29742E12D4EA
:10CE9A00D07F757E2DE51A12D4EFE5197E3512D4AE
:10CEAA00EF7F777E3C125CCC851E1C851F1B227F80
:10CEBA00397E1F12DE2D0FBF40F9781F79567A008E
:10CECA007D1A12DCB212DDB0EA2406FABAAEF378A1
:01CEDA001B3C
:10CEDB00C3E5119570500224B4FA604214603E14FD
:10CEEB00603A2450603A146036EA24A540278A1E23
:10CEFB00751D007D1912CF0B0D30740312CF0B0D66
:10CF0B00781F7956AA1DEA12DCB212DDB00AD3EAF9
:10CF1B00951E40F2228A1D751EB380D7080808089B
:10CF2B007F367E1C90D80CE571700390D81612D505
:0BCF3B00007F3CAE0090852102D50075
:10DA3300787512DA837453201702744E207406E546
:10DA43002E54074430AF1712DAAD7E3BE57DC45444
:10DA53000F12D4C12074077E07742012D4D47878AF
:10DA630012DA83E5172409FF74572017027445203F
:10DA73007402742012DAAD7E3BE57D540F02D4C1EB
:10DA8300E6FD3392171886041886033017031255E0
:10DA9300FE7917787012550E8B13AF06AED27C0049
:10DAA3007D6412547C8F148D15227E0012D4D47E93
:10DAB30007E51312D3897E19748112D4D47E20E52D
:10DAC3001412D36C7E2B742E2073030E742C12D479
:08DAD300D47E2FE51502D36C8F
:10DC4200E54A602E7A2420E00E7A26141460087ABF
:10DC520028141460027A297F667E01EA12D4D42045
:10DC62005505205406800B745B8002745C7E0012A2
:10DC7200D4D420110778A9B60007802130261EC20D
:10DC820026909D857F681276F07F66A85AE54AB491
:10DC9200060108E875F06484E5F012CE1320080F3F
:10DCA200E537640260097F367E2E744112D4A222C7
:10D8D60020144F740512DED4EF33EE33F9EF030351
:10D8E600541FF5F090D929E993A4C5F013C5F01398
:10D8F600C5F013C5F013C5F0135403FCE5F013FB94
:10D90600E9242093C9244093C39BC4540FFBE99C8C
:10D91600C4FC540FF9EC54F02B2446F57BE934F69D
:10D92600F55F22FFFFFFFFFFE6C5AD9C8F857D7784
:10D93600726E6C6A696A6A6C6F747A828D9DB4D9EC
:10D94600FFFFFFFAE9DCD3CEC9C6C3C0BEBBB9B779
:10D95600B5B4B2B0AFADABAAA8A6A4A2A09E9C993E
:10D9660096918C00381CE735D137246F00C5B3C1BA
:10D97600E61F66B60E68C21867AADBF4EDB94675EF
:03D9860010A200EC
:10DEB400D2A27408D2A1D2A300C2A3C2A1D2A30049
:10DEC400C2A3D5E0EF7405D2A300C2A3D5E0F82223
:10DE8D00C2A3D2A2D2A1D2A300C2A375F00833922D
:10DE9D00A1D2A300C2A3D5F0F5C2A175F003D2A300
:07DEAD0000C2A3D5F0F8222A
:10C4440012DE8DD2A300C2A3C2A175F008E4D2A368
:10C4540000C2A3A2A233D5F0F5FE75F008E4D2A37E
:10C4640000C2A3A2A233D5F0F5FFD2A300C2A32237
:10C47400E478806608B88BFB70012274D512C4443A
:10C484007881C3EE13FEEF13F692D118EE2460F612
:10C4940074D612C4447888EF33CE33CE33CE33CE41
:10C4A40033A2D192E25407FCEEFB7A08125363ECF8
:10C4B400244FF608EBF674D912C444EF543F788243
:10C4C400F67886EF33CE33CE33CE33CE335403F601
:10C4D40008EEF618161608E6C4FF54F0F618E6C47B
:10C4E400CF540F2FF674DA12C444EF232354FC788C
:10C4F40083F67884EEF608EF54C0F67880E4660894
:10C50400B88AFBF62212C44C7889C3EF96FF18EE62
:08C5140096FEA2E792165010FA
:10C51C001255E6740FF8F91253B0EF2CFFEE3DFEF6
:10C52C00788BEEF608EFF622E6182016072CF7E6C5
:10C53C003D19F722C39CF7E69D80F66A405E805653
:10C54C00E050F04B0044803DC0384031D02BA0254A
:10C55C00601F2018D014000F000AA00144015801DC
:10C56C00680178018801A001B401D001EC0210022D
:10C57C0038026802A002DA030C034D78BE802085D5
:10C58C008E8A9D8F4D95BA9A97A0BEA631AC53B2A8
:10C59C002AB801BD6AC1EDC4D1C78812C44C788DCC
:10C5AC00EEF608EFF67887798C1253B07883799091
:10C5BC0012C5347885798C1253B07881799212C572
:10C5CC0034788DE624E4FE08E63392D13392D554C8
:10C5DC00FCFFEEA2D133A2D533FE780F7992125321
:10C5EC00B078947990C3EC97F61819ED97F6799486
:10C5FC0090C5477F1F7D11EF93C3971F19EF93973A
:10C60C001F091DED600240EF0F90C567798DEF9308
:10C61C00F7090FEF93F7788E79941253B090C58782
:10C62C00EF93C39BFB1FEF939C2420FC7897E62B86
:10C63C00F618E63CF618E436F6740612DED4D23759
:09C64C00EE24F74006240250021E
:10C65500C237EEFCEFFD740712DED4C3ED9FFFEC8D
:10C665009EFE78B7E6FD337C0050011CEF2DFFEEF2
:10C675003CFE789CEF26F618EE36F62220141220A2
:10C68500370F789DE6B4050912C73912C76E12C770
:10C69500B72220145E7897799A12C7E812556EC3AF
:10C6A500EE9420FE924550031255E67C007D05125E
:10C6B500547C3045031255E6E531B40C3612DA19CF
:10C6C500120E80E5BC2FF560E5BD3EF56120E71152
:10C6D50024F8500DFAC3E5609AF560E5619400F51C
:10C6E50061120E8AE5BC2560F57AE5BD3561F55E1A
:10C6F50012DA267897799AC3E697FB1819E697FC1C
:10C705007A0212536330370B7A02125363ECFEEB55
:10C71500FF800312C73912C76E20140312C7B778FA
:10C72500957998E6F776000809E6F776000809E6B0
:10C73500F7760022799CE77700FB19E77700FC780C
:0CC745009DE6B40506EB33FBEC33FCEC86
:10C75100A2E792D550031255F67A32125371ECFBCF
:10C76100EDFC30D5031255F6ECFEEBFF22EE24086A
:10C77100FE74042037167406307511789DE6B405F1
:10C7810004740C8007F42406C323540FFD7C0012AB
:10C79100534F789FE6FC08E6FBC374109DFA1253D1
:10C7A10071EFF8EEF912556EE878A02FF6FF18EE4A
:10C7B10039F62480FE22927540031255E678BBE6D5
:10C7C100F5F02438400375F0E1EF33EE3378A8F645
:10C7D100A485F07930E7020579C276307508E579EC
:10C7E10024F15002D27622E627FB1819E637FC180D
:10C7F10019E637FD2212BDE87F087871793A12C82F
:10C8010011024ABB855E63857A62787379647F061B
:10C81100E6F70809DFFA227864797380F178737991
:09C82100AF80EB78AF797380E57C
:1052E900E4FEFFFC7D0A791DE7540F2FFFE43EFE23
:1052F900B9190280061912534F80ED301703125560
:10530900E622305C2BEC33921750031255F6EC244D
:10531900D950047C277B007AD2125371EB33CC33FA
:10532900CD33CC33ED33FBEC33FC3017031255F698
:10533900EC33921750031255F67919125585F7096E
:10534900B91DF8A70322EFF88DF0A4FFEDC5F0CE43
:10535900A42EFEEC88F0A42EFE22EB8AF0A4FBE535
:10536900F0CC8AF0A42CFC22EB8AF0A4FBE5F0CC6B
:105379008AF0A42CFCE435F0FD22EB8AF0A4FBE5CD
:10538900F0CC8AF0A42CFCE435F0CD8AF0A42DFDF4
:1053990022EB8AF0A430E70205F0E5F0CC8AF0A40C
:1053A9002CFBE435F0FC2286F0E7FDA4FAABF019FA
:0653B900E786F0A42BFBC7
:1053BF00E435F0FC18E68DF0A42BFBEC35F0FCE4A3
:1053CF0033FDE687F0A42CFCED35F0FD22EB89F0E0
:1053DF00A4CBAEF08AF0A42EFEE5F03400FDEC89EC
:1053EF00F0A42EFEE5F03DFDE433CC8AF0A42DFDB4
:1053FF00E5F03CCEFC22EB89F0A4CBAFF08AF0A411
:10540F002FFFE5F03400FEEC89F0A42FFFE5F03E0E
:10541F00FEE433CC8AF0A42EFEE5F03CFCED89F0DF
:10542F00A42EFEE5F03CFCE433CD8AF0A42CFCE581
:10543F00F03D8E058C068F04FF22C2D5EC30E705B8
:10544F00B2D51255EEEE30E70DB2D51255E6125425
:10545F007C1255EE800312547C30D5031255E62290
:10546F00C3EC13C0E0ED132FFFD0E03EFEBC000BEA
:10547F00BE0029EF8DF084FFADF022E4CCF975F07A
:04548F0008EF2FFFF4
:10549300EE33FEEC33FCEE9DEC994005FCEE9DFEF5
:1054A3000FD5F0E9E4CEFD22EDF9F5F0EE8420D23C
:1054B3001CFEADF075F008EF2FFFED33FD400799AB
:1054C3005006D5F0F222C399FD0FD5F0EA22EC3352
:1054D300EE3400FEEF3400FF7D007A007900780996
:1054E300C3ED9AFDEE9BFEEF9CFFB392D54009ED11
:1054F3002AFDEE3BFEEF3CFFA2D5E933F9ED33FD88
:10550300EE33FEEF33FFD8D92279007A00C380153A
:1055130079007A00C3EA13FFE913FEE8132BFBEECD
:105523003CFCEF3DFDE4F5D2F5D333FE7F19C3EE2A
:1055330098FEE5D299F5D2E5D39AF5D3B392D54047
:105543000DEE28FEE5D239F5D2E5D33AF5D3A2D54F
:02555300EB3338
:10555500FBEC33FCED33FDDF0122EE33FEE5D23308
:10556500F5D2E5D333F5D380C3EDC454F0FEECC4D6
:10557500FF540F2EFEEF54F0FFEBC4540F2FFF2204
:10558500EC75F00A84FCEB54F025F0C475F00A8440
:10559500C4CBC454F025F0C475F00A842BFBE5F0A8
:1055A50022AC10AB11125585A904AD03FA7C197B09
:1055B50099125363AE04AF03EA75F006A4F8AC1272
:1055C500AB131255852875F00A8485F014F8EF2B76
:1055D500FFEE3CFEEF28FFE43EFEE43DFDE439FC32
:1055E50022C3E49FFFE49EFE22E4C39DFDE49CFCF0
:1055F50022C3E49BFBE49CFC22C3E49BFBE49CFCF0
:10560500E49DFD2275D4107B807A0079807800EACC
:0A561500F5F0A4FCADF0EBF5F0A4F5
:10561F00FEAFF0EB8AF0A4C333C5F033C5F092D5DB
:10562F002DFDC5F03EFEE430D501043FFFB5150D4D
:10563F00EEB51409EDB51305ECB51201224006EADB
:10564F0098FAEB99FBD5D40ABB0001220ABA0001E4
:10565F000B22C3E913F9E813F8EA28FAEB39FB80B8
:10566F00A478087B807D807C00EDF5F0A4FAE5F04E
:10567F008EF0B5F007EA8FF0B5F001224003ED9BF5
:10568F00FDD827BDFF0122EDF5F0A4F9A8F0ED0438
:10569F00F5F0A4C399FAE5F09813CA1329F9E83A7B
:1056AF00F8C3E99FE89E50010D22C3EB13FBED2BCE
:1056BF00FD80B6C374689511FB74019510FC8004CE
:1056CF00AC10AB117A0B79B81253DC80177473F8E6
:1056DF00F9E627FB0809E637FC0809E637FD30E74E
:0556EF00031255FEEB63
:1056F40033FBEC33FCED3323FD242083F8ED241C31
:1057040083FFED241883FAED241483F9EF99F9E863
:105714009AFA1253DCEF9DFFE89EFE22FFFFFFB6CC
:10572400FED7FD63FB5DF8C4F59BF1E3ED9EE8CF86
:10573400E379DD9ED743D06BC919C153B91CB07945
:10574400A7709E06943F8A237FB674FF6A045ECBDB
:10575400535B47BB3BF1300423FB17DE0BB2FF80E6
:10576400C21DC232532CF8C3E5679576FBE56895F4
:1057740077FCE5699578FD30E705D2611255FE2482
:10578400F05003125838AA06A907125405EC2480D5
:10579400E43DFBF9F51AE43EFCFAF519E43F600236
:1057A400D2321253DC8B128C138D148E15C3E56424
:1057B4009573FBE5659574FCE5669575FD30E70525
:1057C400D2621255FEEBF9F51FECFAF51DED6002FD
:1057D400D232303201221253DCEB2512F512EC35B1
:1057E40013F513ED3514F514EE3515F51540E102F6
:1057F400560912576420323BEB242E40D3EA24018D
:10580400CB3400FC7A07793D1253DCC010C0118EF2
:10581400108D118C128B13E4FCFD7E077FD012B522
:0E5824004F851203851302D011D010BB000572
:10583200BA0002D21D22B261C374809BFB74F59C34
:10584200FC74209DFD22204D69204866303F637F15
:10585200697E0112C9FB7E1F12CA6B75A7009004F4
:10586200EDE0A2E792171392E7FC1582E013FB30FA
:1058720017031255F6BC003AEB603720E73420E6F6
:105882003110E513201707C3741F9BFE80027E1F91
:1058920012CA600EDBFA22FB2017097E00C37420B5
:1058A2009BFB8008EB241FFE74209BFB12CA5A0E3E
:1058B200DBFA2275A700758307E559C4440FF58208
:1058C200E0A2E792522212C81E1258B5C2E775F042
:1058D2000A84FEAFF075A7045382F1786412593E30
:1058E200AE07786712593E75A700E57DC4540FFED6
:1058F200E57D540FFF7873125932AE07787612594C
:105902003274AF1256DE1257F68B148A1312092024
:10591200ACCCAB017A0A125363E5139B9004ECF012
:10592200FBA3E5149CF0FCA2E7923DD23F02C824FF
:10593200860308860408860518188006E0FBE0FC4A
:0A594200E0FD7A0A12538320E70CFF
:10594C00EB2EF608E43CF608E43DF622C3EB9EF69B
:10595C0008EC9400F608ED9400F622204D0920483E
:10596C0006C23F302A0522C23380F6E54824F640B1
:10597C00F5E5580460F075A700758307E559C42454
:10598C0008F582E0FEA3E0FF1209207437125A2AB0
:10599C00500B30381BC23878C586468013743212CF
:1059AC005A2A400C203809D23878C5A646754600CC
:1059BC00740D125A2A404A1258C8303D3820112210
:1059CC00204D1F20481C204019BCFF16EB243250E0
:1059DC0011D240120E62E5BF75F019A4F536D22E25
:1059EC00D22F205238E55965586032204D2F20486F
:1059FC002CD2338028201109204D062048037536FF
:105A0C0000303319204D1220480F1291460559C30E
:105A1C00E55895595003855859C233C2402229FB89
:105A2C00E435CCFCC3EB9FEC9E22E558B4FF01227D
:105A3C0085581175A704758307E54824F650028034
:105A4C005C201259202905202A02805112C81EE41C
:105A5C00F516F517751000125AC2E510700312C82E
:0B5A6C0018125ADB302910E51B25172B
:105A7700F517F51BE51C3516F516F51C125AE81235
:105A8700C8180510C3E511951050D175A70002C8B5
:105A970024E55AF51124F6500375110A75A7047504
:105AA7008306751000125AC2125ADB125AE8051003
:105AB700C3E511951050EE75A70022E510C4F582D5
:105AC700E0E0F564E0F565E0F566E0F567E0F568C8
:105AD700E0F5692275A701125ED4123ED775A704B7
:105AE70022E9F0E51CF0E51BF022E510C454F0F5BF
:105AF70082E0F512E5822406F582E0F511E0F51C57
:105B0700E0F51B22E512B426157F757E34740D125D
:105B1700D4EF20442575110012CEB9025C397F6D90
:105B27007E3BE012D4D4E5137E3512D4D4E5127E41
:105B37002F12D4D420440312CEB912CE25025C39D9
:105B4700202852E558B4FF012275A704758307E59D
:105B570059F51030330965586005204802051012C1
:105B67005AF1E0F513305E07204304E5376095E00E
:105B77007F797E3D12D4A2E5137E3912D4A2E512B5
:105B87007E3512D4A230480B7F7F7E3512DE2D0E74
:105B9700BE40F980392012012275A7047583068556
:105BA7005B10125AF1305E0A204307E53770030293
:025BB7005D5B34
:105BB900E512700B7E3A7F79745D12D4D4800D752D
:105BC900F06484E5F07E397F7A12D424E537B40293
:105BD90005128FDE8045B403028040E51C7006E59E
:105BE9001B24FB5036E511F964B4602F20062CE51F
:105BF90037600D200C0AC3E99570F9500324B4F9F4
:105C0900E912DCB2781D79547D1D90D7FEE53F205D
:105C1900E00390D80512DDB012D500751779751615
:105C29001930280375161DE51264266003125C7C81
:105C390075A7009006E3E511F0A3120E7BE5BC758C
:105C4900F01970040475F014A4951BFBE5F0951C7C
:105C5900FC922450031255F6ECF0A3EBF0C24FC2AC
:105C690063EC700EEB24E64002D24FEB24C84002ED
:105C7900D26322E51C24ED402BAE1CAF1B125E9EA5
:105C89007C007D3212547CC005EFAF17AE1612D3DB
:105C9900DDCE2405CE742C12D4D40E0ED0E02312FE
:105CA900D3D7801B125E95125CD6CE2405CE742CF8
:105CB90012D4D4CE2402CEE875F0058412D4BACE1B
:105CC9002404CE7422305D02748302D4D0EE243DC4
:0D5CD90050047EC37F4B7C017DF412547C8F
:105CE600C004C005EF6007AF17AE1612D3DDD007AC
:105CF600D0067C007D3212547CA805EFAF17AE1695
:105D0600CE240ACE02D4BA125E95EE2450305D033C
:105D1600EE24A150047EC37F4B7C017DF412547C9B
:105D2600C004C005EF6007AF177E2F12D42AD00734
:105D3600D0067C007D3212547CC005EFAF177E374B
:105D460012D48F7E3B742C12D4A27E3DD0E075F027
:105D5600058402D48F7F6D7E2F746312D4D4E5122E
:105D660075F06484E5F07E3512D36C12CEB902CE9E
:105D76002530480320740122E4FCF5A79006E3E0F1
:105D8600F9A3E0FE24FE40EFA3E0FF7D78E537604F
:105D960008304FE3200C2A800B120E67E5BD20E089
:105DA60010304F0DD206E57124FE5015125E8B8021
:105DB600107D3CE546600A7D141460057D0A14706A
:105DC600B6891112534F7D6F12546FBE00A9EF248E
:105DD600E240A4AD07E51112DCB2202404B2D5B22C
:105DE600D1781F795612DDB0A806A907E511242D32
:105DF60075F0B484E5F012DCB27407304F02740E0D
:105E0600FDFA12DDB0B2D5B2D112DDB0B2D5B2D143
:075E1600DDF0AD0212DDB06A
:105E1D00850616850717B2D5B2D112DDB085061EDF
:105E2D0085071F7A03304F027A06E511241675F0A7
:105E3D00B484E5F012DCB2A816A917AD0212DDB0DC
:105E4D00DDFBE51124EA400224B412DCB2A81EA940
:105E5D001FAD0212DDB0DDFBE5377021304F1E9016
:105E6D00A5E0305D0390A5DC7F3C7E3312773512C3
:105E7D000E67E5BD20E00612CA7112D79F22C3E955
:105E8D009570500224B4F922E51B2402FFE4351C61
:105E9D00FE305D1ABEC305BF4D028012AC06AB07C6
:105EAD007A1B1253717832125513AE04AF03227858
:105EBD007379641256E01257F6751CC3751B4B208F
:105ECD0032048B1C8A1B22125EBC30320122AC19AB
:105EDD00AE1AA91DAF1FB90005BC00028010C3E9A1
:105EED0013F9EF13FFC3EC13FCEE13FE80E8BF298B
:105EFD00005006BE2900500122C3EF13FFC3EE135D
:105F0D00FE80EB3E7FE3E3E3E3E3E3E3E3E3E37F01
:105F1D003E0C1C3C7C7C1C1C1C1C1C1C1C7F7F3EDA
:105F2D007FE3E3E3070E1C3870E0E3FFFF3E7FE302
:105F3D00E3030F0E0F03E3E3E37F3E070F1F3F77EE
:105F4D00E7E7FFFF0707070707FFFFE0E0E0FEFFBA
:105F5D00030303E3E37F3E1E3F73E0E0E0FEFFE358
:105F6D00E3E3E37F3EFFFFE3E30303070E1C383853
:105F7D003838383E7FE3E3E37F3E7FE3E3E3E37FBF
:105F8D003E3E7FE3E3E3E37F3F030303E77E3C0015
:105F9D000000181818FFFF18181800000000000066
:105FAD00000000FFFF0000000000003FF00000387F
:105FBD001C38F00180C1F020F0FC0038F03FE0000B
:105FCD000000007CC6C6C6C6C6C6C6C67C183878D4
:105FDD001818181818187E7CC6C60C183060C0C664
:105FED00FE7CC6C6061C0606C6C67C0C1C3C6CCCCC
:105FFD00FE0C0C0C0CFEC0C0C0FC0606C6C67C3CDC
:10600D0066C0C0C0FCC6C6C67CFEC6C6060C18302F
:10601D003030307CC6C6C67CC6C6C6C67C7CC6C6FD
:10602D00C67E060606CC78000018187E7E1818006D
:10603D0000000000007E7E00000000000000000057
:10604D000000000000C6E2E2D2D2CACAC6C6C20033
:10605D000000000000000000008080A0C0A0003003
:10606D004020C08080C0A0A0000060A0600000A003
:10607D0040A05098D090882050A850888850A850A3
:10608D002060806000000040E040000000000080C3
:10609D000000E000000000000040002040800040B3
:1060AD00A0A0A04040C04040E0C02020C0E0E020C3
:1060BD004020E02060A0E020E0C02020C06080E013
:1060CD00A0E0E020404040E0A0E0A0E0E0A0E02023
:1060DD00C0004000400000800080002060E0602093
:1060ED0000E000E00080C0E0C080E0E0E0E0E00023
:1060FD000000000040A0E0A0A0C0A0C0A0C040A033
:10610D0080A040C0A0A0A0C0E080C080E0E080C022
:10611D0080806080A0A060A0A0E0A0A0E0404040F2
:10612D00E0202020A040A0A0C0A0A080808080E022
:10613D00A0E0A0A0A0A0E0E0E0A040A0A0A040C0F2
:10614D00A0C0808040A0A0C060C0A0C0A0A0608002
:10615D004020C0E040404040A0A0A0A060A0A0A072
:10616D00A040A0A0A0E0A0A0A040A0A0A0A0404062
:10617D0040E0204080E02020A870202070A8202042
:0D618D0008F030D0100000F0A8A8000000BD
:10619A00E0000000902048708898984000E0E0E015
:1061AA0000A0E0E0E04060301030604040E0404055
:1061BA0060909090909060206020202020706090E5
:1061CA0010204080F06090102010906010305090A5
:1061DA00F01010F080E010109060609080E09090D5
:1061EA0060F0102020404040609090609090606085
:1061FA00909070109060C0E0F0F8F0E0C0000000ED
:10620A000000000000000000000000506050007014
:10621A007050000078807008F000F8888888F800CC
:10622A00C0C8102040981800C0B098B0C0006020C4
:10623A0040000000000090D8FCD8900000246CFCBC
:10624A006C24000020A870A82000002020F820203C
:10625A000000000000000080000000F000000000C4
:10626A0000000000606000081020408000708888EC
:10627A00888888702060202020207070880810206C
:10628A0040F8F810201008887010305090F810105C
:10629A00F880F008088870304080F0888870F80824
:1062AA00102040404070888870888870708888788C
:1062BA0008106000606000606000000080000080DC
:1062CA0000002040F84020000000F800F80000001C
:1062DA002010F8102000708808102000200000000C
:1062EA000000000070888888F88888F08888F0881C
:1062FA0088F070888080808870E09088888890E034
:10630A00F88080F08080F8F88080F0808080708843
:10631A0080B8888878888888F888888870202020BB
:10632A00202070381010101090608890A0C0A090A3
:10633A0088808080808080F888D8A8A88888888803
:10634A0088C8A898888870888888888870F088881B
:10635A00F080808070888888A89068F08888F0A08B
:10636A00908870888070088870F82020202020206B
:10637A00888888888888708888888888502088884B
:10638A0088A8A8A85088885020508888888888506B
:10639A00202020F80810204080F800CCAC9CACCC1F
:1063AA000000CCD4E4D4CC0004781828C800FC40FF
:1063BA00A04018202018000000000000F80000008B
:1063CA0000A040A05000788888986870884030887B
:1063DA0070200000F0A8A8A8A878484848487888FB
:1063EA0070888080887020A88898A8C8888880507B
:1063FA0048FC485080304C5C6060603C00E0F0082B
:10640A000808F88044485C484480F880808080808E
:10641A008078484848484888B8A8A8E8A8A8B8880A
:10642A0088888888F808500070888888708080F08A
:10643A0088888888F8888888888888F090909090DA
:10644A0090F0A8A8A8A8A8A8F8888888F808080832
:10645A0050008888888878A8A8A8A8A8F808000002
:10646A000000000000000000000000008888888802
:10647A00E8A8E8A8A8A870A8A8A80000000000003A
:10648A000000000000000000000000000000000002
:10649A000000000000000000006000606000600072
:1064AA0060006060205020000000005090B890D03A
:1064BA0090886050500070705000882020887000CA
:1064CA000080C0A090F8003048B4B448300030488A
:1064DA00B4B44830FC0098D02058C800F8E8D880F6
:0A64EA00D8E8F8404050F850404058
:0300000002005E9D
:03000B0002B5DF5C
:0C000E00206E06859950D26E32D26F32FF
:0E00230010990AC298206DE385994FD26D3274
:10003800E4F537F534F52F12DE23C229C22AC26847
:09004800C227C214C215022D9C4E
:03005B00022B2A4B
:10B5D2008530F0C5F065308530F060F722C0D0C00C
:10B5E200E0C0F0C0A775A700C083C08275D00875FF
:10B5F2008A00300503758A7A758CEA0532E5327065
:10B602000215320530E530640A6026201520E53146
:10B61200B40C0BE530B4010612BA5A12D8D6E53191
:10B62200B4180BE530B4060612BA5A12D8D602B7CD
:10B63200F9C2AFD2C075C07AD2AFF5300531E5316B
:10B6420064197040F531201529C225C22C7D0A7477
:10B652000412DED4EF33EE339005CCF0EE24F54045
:10B66200112402400B24014005DDE4022B2AD225DD
:10B67200D22CE5A6600215A678B5E660011678B66A
:10B68200E6600116302E0BE5367007C22FC22E126D
:10B69200B987E5367004C24B8002153678A9E66098
:10B6A200011678D8E66001160535E53570021535C4
:10B6B200E590307B0B30E008D278C27BC200801A62
:10B6C200307C0B30E108D279C27CC201800C307D23
:10B6D2000930E206D27AC27DC202E59044F8F470E3
:10B6E20003753500304A09E53324FA5003753305F2
:10B6F200E5336005153302B79EE590F454077003F5
:0DB7020002B79EA2E09200A2E19201A2E235
:10B70F00920230100320143D75330820001B2010C7
:10B71F000C2011098013E59030E10E8006E53724E7
:10B72F00FC40F3E543541FF53320100375A6FF20AB
:10B73F002E5D301004E536705620100C201109E5EF
:10B74F003524F55003753304D21BD2A5D2A612B9F6
:10B75F008775B44075B24078D8E67002053420275B
:10B76F002E20682B202928202A25A2107211501F65
:10B77F00E52054076019E53424375004C24A800F7E
:10B78F002401400B200026200119D27D7534C820DA
:10B79F001558E531702412DEB474E812DE8D802A5C
:10B7AF0002B8CCE53724FC40E6D27C80DF3011DFD5
:10B7BF00E53724FC40D9D27B80D275F00384E5F0C5
:10B7CF0070DE12C50974E812DE8DE531B40605127C
:10B7DF00C6818016B40C0512C697800EB4120512DE
:10B7EF00C6818006B4180312C697E59030E1053084
:10B7FF00E202800620100820110520103C807D20D9
:10B80F0027F82068F52029F2202AEFE5342430406C
:10B81F00E9240750E5600B205E088590F020F202C6
:10B82F00740190B84193D2A5201002C2A512B9722B
:10B83F00806FC8A08269554646202F12E536603CBE
:10B84F0024AA500AE53675F01984E5F06040D2A6B7
:10B85F00201002C2A6D2A5202F0C7418304B0274F0
:0EB86F006412B972803BE53675F00C30480368
:10B87D0075F00684A2E0744640E9743780E5E52B47
:10B88D005403600C20100E301106E54A6402600569
:10B89D0012B98D800312B8E4101B08A25892A5A20C
:10B8AD005992A675A700D082D083D0A7D0F0D0E052
:10B8BD00D0D0201009C5A67003022B2AC5A632C20E
:10B8CD0018B40202D21812C5A730180874E412DE9B
:10B8DD008D02B7D902B7D478A7E5B4600924E0404A
:10B8ED0005760002B98DE534702920412220751F9F
:10B8FD00300D1CE57924CE40167AFFE5B110E70135
:10B90D000A2325B3F5B3EA35B4F5B4C313F5B2E69E
:10B91D0060021622C2412075028075E579FF6058DC
:10B92D0020120424FD5051206502C21CD265FF2453
:10B93D00B050027F4FEF90BA0A9375C70375C6FCDE
:10B94D0075B90185BFF0A4E5F0F624F44002760C3C
:10B95D00301C2DE5BEC39FF5F0A4E5F024E04003B7
:10B96D0075F020E5F0C21C79AA770375B300F5B424
:10B97D00C31375B100F5B222C26578A77680D241A6
:10B98D0079AA7703D21CE4F5B3F5B4F5B1F5B2227B
:10B99D00C26579A1E57924CE500DE720E7E276283E
:05B9AD00301CDD7432C6
:10B9B20080BE7680E720E7D3E5799740CE79AAE783
:10B9C200FAE5792323B4C500400274C42437300E4B
:10B9D20031F42437300D15F7BA0302FA0AC39AF587
:10B9E200B175B300EAF5B4C313F5B222101C07D245
:10B9F2001C76C802B974763274FF200E02749B0260
:10BA0200B974C313247E80CCFFF3E8DDD3C9C0B878
:10BA1200B0A9A29A948F8A85817D7975716E6B68BF
:10BA220065625F5C595653504E4C4A484644424008
:10BA32003E3C3A383634333231302F2E2D2C2B2ADD
:10BA420029282726252524242323222221212020B8
:10BA52001F1F1E1E1D1D1C1CD2B5C28EAE8DAA8DAF
:10BA6200AF8BAB8BE4F58DF58BD28E30140122783F
:10BA7200B6BE0007EF24E24002800806E624EC503E
:10BA8200027614206705E624F64005E4FEFAFFFB81
:10BA92007C007D0A12534F7C007D5E12546F8F51E1
:10BAA200EE60037551FFEAFC7A33125363EBF5F053
:10BAB200A4E5F0CB8CF0A425E0C5F035E0CB92D51F
:10BAC20025F050060BBB0002D2D530E7060BBB00B7
:10BAD20002D2D5ECF5F0A42BFBE5F03400FC30D516
:10BAE200010C78A6E6C39BFF18E608F6EB18F618D9
:0EBAF200E69CFE18E608F6EC18F63014012269
:10BB00007A0050040A1255E67C007D6E12546F8F45
:10BB1000F078A2E6A4FBACF0125585EBBA0002F473
:10BB200004FAE4F8FFEA30E70118E57960062075C9
:10BB3000031FF4042AF579EF38D27520E708600373
:10BB40007579FF02C7DAC2750470F5E579F404600F
:10BB5000EFF57980EE120E5D78BBA6BC120E7BE588
:10BB6000BE78A2F624F65007E4F5BEF6124EE612B1
:10BB70000D46E5BEF54824F65008E4F5BEF548123A
:10BB80004EE6E5BFF54324F3503924F34035120E59
:10BB90007178A1A6BCE5BF789DF61424FB5008740B
:10BBA00003F6F5BF124EE678B7A6BE120E67E5BDE6
:10BBB000A2E39266A2E49267035403C253B4010263
:0EBBC000D25322740DF5BFF543124EE680C03D
:10005E0078FFE4F6D8FDF4F5A6D2B4D2C075C07A16
:10006E0075D75075AE1375AF017581D87590F8754B
:10007E00EFBC75FDFFD2A412DDFAC2A47450122B90
:10008E0042758951D28C75A882D2BC12BBCE12DEBB
:10009E00B412C47F12BB5512D989122A087F407E32
:1000AE0001909C73127702124D4A12DDFA12DADBBE
:1000BE0012DD1212DE237C1412DE04300003022B3A
:1000CE002ADCF512489F753A001248EDE53A701693
:1000DE0012DEE87F437E0690A3C512770212DD1270
:1000EE003000FD022B2A75A6FF12489F12BB551237
:1000FE002A0812DD1212DDF612DE2378B5761E12F4
:10010E00D98912C474C215C214122A08909CBA7FDF
:10011E00781276F0205E0A7F767E12909CC712D5FA
:10012E00007F4012DD887F497E0978AEE612D36CDF
:10013E007E15743A12D4D47E1AE53E12D36C7E2606
:10014E00743A12D4D47E2BE53F20E00805A6E5A62E
:10015E00700215A6E53F12D36C7F5312C9EF7F577D
:10016E007E0B12D29912D3217F60207303020208F4
:10017E007E0BAC5DAB5C12D29D12D3217E31127719
:10018E008D7F697E1212D8243025087E1290DB44B2
:10019E0012D500E5A60303543FFDFE0D7F7312DE5C
:1001AE002D0F12DE2D1EDDF478B5E57124F640021A
:0801BE00761E307419E660564C
:1001C6007F727E16744012D4A27E17E612D42A7E5F
:1001D6001F745312D4A212DD12100037100137100B
:1001E600023712483FD2AC75369612DB8AB4E00568
:1001F600124935800AE53670F112488D12DDF30298
:10020600010D2074097E2BE52E540712D4C17E17EA
:1002160002018C022B2A022D628072E53524C85019
:1002260049E59020E244D0E0D0E012027102735614
:10023600E53524D25034E59020E22FD0E0D0E0120C
:10024600DEE88038E53524D25020E59020E21BD048
:10025600E0D0E012DEE8306B0B7F091276E7124F32
:100266001E127BBD1202710206BE2212DEE890A4A7
:100276007C7F001276F012DD1202DDF312DEE890CA
:10028600A47C7F001276F012DD1212DDF6C215C2D2
:1002960014C227C26812DE23753701909DA2121C74
:1002A600FF9002AB730200F70217C2020B56021F41
:1002B60012021F0E0206BE0206FB0273560202C699
:1002C60012DE2375370790A125121CFF9002D67304
:1002D60002029302096B0209A50209D90202FA0277
:1002E60005AD0202C60202C60203180202FF024B55
:1002F600B30203261248F0805A7F517E00747212B0
:10030600D4D0121E5C40B9124E3512D98912BB5593
:1003160080AE7F49A25E120D31925E120D5080A012
:100326007F64120E9E121E5C401DE5352480F47516
:0C033600F0198460157F727E1F12D4C184
:1003420012DD121001E810000280E30202C612BCA4
:100352003B0202C6124EE612DE2375370290A2F469
:10036200121CFF900369730202C6020EA8020F0D4F
:10037200020F61020FB6020FFA02100902035902BC
:10038200051302038980D0D21412DEE87F147E05A1
:1003920090A33B127702121E1912DD1212486875E1
:1003A200A6FFD2AC1000DE12DB8A204CF2B405EFBD
:1003B200E4F511F514F5151204411204D51248683A
:1003C20075A6FFD2AC1000BD12DB8A204CF2B41528
:1003D200051204C880E7B406E712047FE51424FC82
:1003E20050D5E4F56FF56EF56D12048B1204D5123B
:1003F200486875A6FFD2AC10004212DB8A204CF28C
:10040200B415051204C880E7B406E71204B5E56F17
:1004120024F050D5124868743B12DC067A47909C4F
:100422006A1224C9742A12DBFA909C731224C974CA
:100432002A12DBFADAF912DC2312DE04020359ACC7
:1004420014AB157A0412536375A704900400E4F008
:10045200ECF0EBF08514C78515C67F08120467DF40
:10046200FB75A7002275B901E5BCF0E5BDF0E5BE5C
:10047200F0E5BFF005C6E5C6700205C722E5152402
:1004820008F515E43514F5142275A704900400E567
:100492006F4410F0E56EF0E56DF0740312BC077F57
:0404A20020E4F5F766
:1004A600C2B2C2B2E5F7F0DFF4D2B275A700227489
:1004B60020256D54E0F56DE4356EF56EE4356FF587
:1004C6006F2205117F287E00E51112D3E380069086
:1004D6000402E070177F287E15900400E012D3E333
:1004E6007E2A900401E012D3E312DD1212486874EA
:1004F6003A12DC3D75A7009004007F23E0A312DBCF
:10050600D9DFF912DC143099FD2202035912DEE814
:100516007F0F90A66F1276F0121E1912DD12C2140A
:10052600C21512DDF37510651000DFE53170F9E5CF
:10053600106465700D855E14857A15E4F512F51361
:10054600800C78A8E51326F513E43512F5127F1E04
:100556007E19E51012D389C3E57A9515F517E55E80
:100566009514F5167F287E0BAC16AB1712D29D128A
:10057600D32112DD1212DE04D510ADAB17E516FC41
:1005860030E7031255F67A0A79001253DCA912A84D
:1005960013125515EBF510243840037510C8120ECA
:1005A6005D8510BC02035612DEE8909CFD7F017E3D
:1005B60009127702909D057F0A7E091277027F1342
:1005C60012C9E7751700120E6CE5BC12068DE5BD63
:1005D60012068DE5BE12068DE5BF12068D909D555D
:1005E6007F5F7E06127702121E9E12DD12751700BD
:0605F60012066D10000862
:1005FC0010011510024880F20517E51724F7500377
:10060C0075170075100080E2E51764087015120E5E
:10061C006C75BC0175BD2375BE4575BF67124EE682
:10062C000205ADE51012069F12DD1212064D0510E3
:10063C00531007E51724FE400353100380AC02024D
:10064C00C6A9BCAABDABBEACBFE5171304F8E64007
:10065C00085407C42510C4800454702510F6027D7C
:10066C00A17800E875F009A42417FF7E3B7D20E8F3
:10067C00651770027D89ED12D4D408B809E502DD46
:10068C0012F8C4120693E812069F7E030517E517AD
:10069C0002D4C1540775F009A4909D0D2582F582F2
:1006AC0050020583E51775F009A42417FF7E0C0290
:1006BC007702C26812DE23753705909EDD121CFF8F
:1006CC009006D073020293027941027986027B1C58
:1006DC000206BE0206F4027A5E027AC402178B028C
:1006EC0006BE021771020C627F2E12168680C31290
:1006FC00DE23753706909FB3121CFF90070B730215
:10070C0002930217C802182A0218A30219700219C0
:10071C00A2021A19020750020749021A62021B07A9
:10072C0002072F7F64120E67E5BDA2E7120D31128E
:10073C000E67E5BD92E7F5BD124EE680B27F491219
:10074C00168680AB12090C122B6912DEE8121DF30F
:10075C00E55804607790A07D1207F912871E12DD10
:10076C001210000810011310021C80F50559C3E586
:10077C0058955950D575590080D01559E55930E721
:10078C00C985585980C4E559B40F02802FB51F0292
:10079C00802A75F007A42408F51775162774B82558
:1007AC0059F987001207E712DD12100028100128F2
:1007BC0010020280F574B82559F9A700E53524FA22
:1007CC00508878C7A64812090312DEE812DD12120F
:1007DC00DDF60206FB1880CC0880C9E875F005A48C
:1007EC0085F01CF51BC000125C7CD000221287AF78
:1007FC00B4FF0122751000751FFF1287C6E5106447
:10080C000F6017120830401274B82510F8E675F016
:10081C0005A485F01CF51B125D0D0510C3E558955C
:10082C001050D7221211AEF8602E6404602AE8141E
:10083C00B51025F51F120E7BE5BC70060475F0147F
:10084C00800375F019A485F01CF51B125D0D7E223A
:10085C0090A610127735D322C322E558B4FF01229B
:10086C00751000E510640F602EE51075F007A424D8
:10087C0009FF74B82510F8E61208ED75F00A84C06B
:10088C00F07E2012D42A7E28742C12D4A2D0E07EC2
:01089C002A31
:10089D0012D48F1208AD0510C3E558951050C32220
:1008AD001211AEF8603964046035E8146510702FCC
:1008BD00120E7BE5BC1208EDF8C313923D7E1C129F
:1008CD00D4407E28742C12D4A2E4303D067405B8B1
:1008DD000001147E2A12D48F7E18742312D4A22202
:1008ED00305D1275F036A42432FBE435F0FC125560
:1008FD0085125585EB221209151276D5DFFB2212D2
:10090D000915127EB1DFFB2275C70375C6F078B8E5
:10091D007F042275C70375C6F375B901E5BFB548E8
:10092D0031E55924F1402BE55975F00484A9F024E3
:10093D00F0F5C675B901C5F0A9BC600CA9BD146070
:10094D0007A9BE146002A9BFE975F005A4F985F0E9
:10095D00CC22120E7BA9BD75CC0022124EE612DE02
:10096D002375370390A18F121CFF90097B73020230
:10097D00C6020C7B02131F020C90020C9B0216E6A2
:10098D000213A6020D5C0213DA02142002173802BC
:10099D00138E021465124EE612DE2375370490A2F3
:1009AD004F121CFF9009B5730202C6020CAA020C6D
:1009BD00B50209A5020CCB020CD60210230209A523
:1009CD00020CE5020CC0020CFF124EE612DE23757E
:1009DD00370B90A29F121CFF9009E9730202C60209
:0B09ED0010D10210D1020A6F020AAD07
:1009F800020A10020A330217CE02117602123E02D0
:100A080011E70212CF020D19120E67E5BF1470C16B
:100A18007F2E120E9E1F120E67E5BDA2E6120D3143
:100A2800120E67E5BD92E6F5BD80A37F37120E9ED4
:100A3800120E62A8BFE8120A6712DD121000081031
:100A4800010D10021280EE18B802EA780A80E60852
:100A5800B80BE2780380DE120E6288BF0209D67FE7
:100A6800367E2CE802D3727F1C120E9E120E67A8E7
:100A7800BE120AA112DD1210000810010D10021496
:100A880080EF18B800EB780B80E708E824F450E111
:100A9800780180DD88BE0209D67F1B7E35E875F0B7
:100AA80005A402D36C7F25120E9E120E67A8BF12F2
:100AB8000ADF12DD1210000810010D10021480EF79
:100AC80018B800EB780980E708E824F650E17801C7
:100AD80080DD88BF0209D67F247E3BE802D4C1129C
:100AE8000E5DE5BF75F03CA4ACF0FDE5BE75F00504
:100AF800A42DFDE5F03CFC120E67E5BF14603675C9
:100B0800F005A485BEF0A42DFFE5F03CFE7C007D39
:100B18003C12547CC005EF75F01884E5F07F2D7EFB
:100B28002412D36C7E30743A12D4D47E35D0E012BD
:070B3800D36C02DD127F2DDA
:100B3F007E0590A632127702120E67E5BDA2E67F00
:100B4F002D12161502DD12D25712DEE8121DF31206
:100B5F000B640202937F177E02909DFE1277027F35
:100B6F004C7E02909E16127702AC5DAB5C7F577E77
:100B7F000412D319120E8A85BC6285BD63E5612408
:100B8F00F84044909E227F371276F0AE61AF607CC2
:100B9F00017D5E12547CC3741F9FFAAC63AB62EC91
:100BAF0033921750031255F6125363AB047C003087
:100BBF0017031255F674F52BFB74033CFC125339D3
:100BCF007F377E1512D291909E2F7F697E0F1277FD
:100BDF0002E560240FFBE43561FCA25C923BD25C22
:100BEF007E1E12D29DA23B925C7E30742012D4D412
:100BFF007E36742012D4D4E5602562FBE56135633F
:100C0F00FC7F227E0412D319E56245637016742EA1
:100C1F007E3A12D4D412DD1210000D1001151002FD
:100C2F0026020B8C742080E81562E562B4FF0C1568
:100C3F006380080562E56270020563E53524F550AF
:100C4F0003753301020B8C120E8A8562BC8563BD5E
:100C5F00024EE67F637E00747212D4D0121E5C4087
:100C6F00087F631276E7124EED0206BE120E71E593
:100C7F00BCA2E77F0A120D34E5BC92E7F5BC02096E
:030C8F00687F1C5F
:100C9200A20D120D31920D80097F25A20E120D3187
:100CA200920E120D5002096B7F0AA20F120D3192A1
:100CB2000F802A7F13A208120D319208801F7F52E3
:100CC200A20C120D31920C80147F25A20B120D3151
:100CD200920B80097F2DA209120D319209120D503B
:100CE2000209A57F49120E67E5BDA2E3120D31127A
:100CF2000E67E5BD92E39266F5BD0209A27F5B1223
:100D02000E67E5BDA2E5120D31120E67E5BD92E553
:100D12009243F5BD0209A27F6D120E67E5BDA2E006
:100D2200120D31120E67E5BD92E0F5BD0209D61231
:100D32000D468F1F9217120E9EAF1F1F7E3912840F
:100D42000BA21722120E7685BC2B85BD2122120E14
:100D520076852BBC8521BD024EE6203714120E711A
:100D620085BE12120D89120E718512BE124EE680D8
:100D7200057F3F120D7B02096B7E0390A219127749
:100D82000212DD1202DDF375A6FF12DEE812B5D201
:100D9200740712DED48FF0740612DED4EF2512C36C
:100DA20095F0A2E7923D4010FD24CD50027D32AC79
:100DB20005C3743F9DFD800FF404FD24C850027DDD
:100DC20037AC0574402DFD7F4012C9E77E1212DE5A
:0F0DD2002D0EBE1EF91F303D020F0FEF6D70ED9D
:100DE100E536700A753606EC2513F5148C13120ED0
:100DF1000712DD1210000710010830020722151238
:100E01008002051280827F377E28742E12D4D47F0F
:100E1100347E21740A303D010412D4EFE514FC2420
:100E21009C50027C637F347E2DEC12CE137F437E77
:100E31001E12D2997E00E51212D4307F057E0290F7
:100E4100A2241277027F6D7E0190A22F1277357F47
:100E5100747E0490A23F127735021DF375C6F480AB
:100E61003575C6F5803075C6F6802B75C6F78026B8
:100E710075C6F8802175C6F9801C75C6FA8017758C
:100E8100C6FB801275C6FC800D75C6FE800875C64E
:100E9100FF800375C6FD75C70375B9012274721F02
:100EA10012D4D00F02DD127F0A120E9E7E2A124842
:100EB100F0120E7BA8BF120EDC10001210010510FB
:100EC100021580F508E824E750EC781880E818E866
:100ED10030E7E3780080DF88BF805F7F097E05907F
:100EE100A4F3B80C0390A4ED1277027E27E53D2808
:100EF100240C75F01884E5F012D36C7E33743B1228
:100F0100D4D47E35E53E12D36C02DD127F13120E6E
:100F11009E120D46120F3E10000810010510021717
:100F210080F2105C07205D0BD25C80E8105DE5D299
:0D0F31005D80E1D25C80DD852BBC020356A3
:100F3E00205C10205D1890A5467F127E231277024A
:100F4E0002DD1290A55A205DF090A54D80EB90A584
:100F5E005380E67F1C120E9E120E76A8BF120F98BB
:100F6E0010000810011110021A80F2E824F250034A
:100F7E001880EA780D80E6E824E740030880DE78E2
:100F8E001980DAE8F5BFF54380A37F1B7E26E412B5
:100F9E00D4C1E82323B464087E26740112D4C1E4BC
:100FAE007E2E12D36C02DD127F25120E9E120E853E
:100FBE00A8BCE8120FF112DD1210000810010D107E
:100FCE00021F80EEE824E050E9188006E824CF40A6
:100FDE00E108120E8588BC124EE6D21512D9898010
:100FEE00D180157F247E3724E202D3DD7F2EA20A24
:100FFE00120D31920A120D500203597F37120E67ED
:10100E00E5BDA2E4120D31120E67E5BD92E49267C2
:10101E00F5BD0203567F367E00747212D4D00F7E59
:10102E0016743F12D4A2120E71A8BD12109C12DDBE
:10103E001210000810010510021080EFE8248750EE
:10104E0004240A800224E8F880E17F377E1674209B
:10105E0012D4A27E2C743F12D4A212109C12DD1256
:10106E0010000810011410022080EF18B80904783F
:10107E007880E7B878E478E780E008B87904780AF1
:10108E0080D8B8E8D5787980D188BD0209A2E82445
:10109E0087923DE8500224917F367E30C313923BF7
:1010AE0012D3DD7E3CE4303B02740512D4BA7E1AB4
:1010BE0090A43A303D0390A43E1277027F3C7E3AD4
:1010CE0002DE2D7F127E00747212D4D00F7E207439
:1010DE003F12D4A2120E5D85BE1085BF111211589B
:1010EE0010000810011110021B80F21511E511B449
:1010FE00FFEB75111780E60511E51124E850DE753A
:10110E00110080D91211587F137E20742012D4A2A0
:10111E007E31743F12D4A212DD121000081001119C
:10112E0010021B80DF1510E510B4FFD875100B8070
:10113E00D30510E51024F450CB75100080C6120EA6
:10114E005D8511BF8510BE0209D67F127E24E51182
:10115E0012D36C7E30743A12D4D47E35E51075F00D
:10116E0005A412D36C02DD127F49120E9E1211AE2F
:10117E00F81211B410000810010D10021280F218AE
:10118E00B8FF02780480EA08B80502780080E212FF
:10119E000E5D88BD124EE6B800030209D902123E5A
:1011AE00120E5DE5BD227F487E0590A45412770293
:1011BE00E8601CB4040A7E0590A449127702800CE4
:1011CE0090A4601277027E38E812D4C102DD12902C
:1011DE00A45B7E2912770280F31211AE601D6404A7
:0211EE00601986
:1011F0007F5B120E9E120D46121219120E7610000F
:101200000B10010810020C80EF0209D9105FE9D21F
:101210005F80E5852BBC0209D61211AE601F640405
:10122000601B7F5A7E0590A4541277027E2390A4FF
:1012300064305F0390A46B12770212DD1222121148
:10124000AE70030209D97F527E11120E9E120E7BE0
:10125000A8BC12127E120E7B1000081001081002AA
:101260000880EF1880EC0880E9120E7B88BC124ED3
:10127000E6120E85E875F005A4F5BD0209D6121137
:10128000AE604BE875F03270040475F028A4ADF040
:10129000FC305D11ACF0FB7A8A125371EB30E7053C
:1012A0000CBC00010DAE05AF047C007D6412547CC3
:1012B000C005EF7F517E1A12D3897E2C742C12D474
:1012C000D4D0E07E2F12D36C1241B712DD12227FF0
:1012D00064120E9E120E7BA8BD121300100008109F
:1012E000010F10021680F218E824CD50EC783280FD
:1012F000E808E824CD50E2780080DE88BD0209D6F7
:101300007F63E823C2E012CF4675F06484C0F07EAC
:101310002612D4C17E2C742C12D4D4D0E080A47FA9
:1013200013120E9E120E71E5BCA2E7923DC2E7F8C1
:10133000E812135E12DD1210000810010D100212E7
:0313400080EE1824
:10134300B800EA783280E608B833E2780180DEE854
:10135300A23D92E7F5BC79A1F78079547F305C0117
:10136300237F127E2375F00A84C0F012D3DD7E2D15
:10137300742C12D4D4D0E07E2F12D4BA0F7E3590C1
:10138300A560305C0390A5BC0277357F64120E9E86
:10139300120E7BE5BE7F637E2C128460F5BE79A2BC
:1013A300F780317F37120E9E120E76A8BC530003CE
:1013B3007F367E32E812D4C112DD1210000810010C
:1013C3000710020780E718180880E2E5BC54FC48C0
:1013D300F5BCF52B0209687F49120E9E120E85A8F3
:1013E300BE12141112DD1210000810011110021A9E
:1013F30080EFE8240AF8242450E778DB80E3E8242C
:10140300F6F8247F40DB788180D788BE80C6E8F475
:1014130024DC75F00A847F487E3B02D4C17F5212DC
:101423000E9E120E85A8BF12145812DD121000086A
:1014330010011110021A80EFE82408F8245750E72E
:1014430078A880E3E824F8F824A040DB786080D70C
:1014530088BF0213D7E8F424A923C47F517E3B023B
:10146300D4C1122C74754A00D210C211D214D27591
:1014730075791475340012DEE87F007E0290A1FABC
:101483001277029041E07F087E2612D500E52B54A7
:10149300030F7E3912D4C1121E0E12D16A128ED1DD
:1014A30012DD1210000810011A10022480C52075E5
:1014B30004057980BE1579E579B4FF05C2757579A0
:1014C3000180B02075EB1579E57970A7D27580A3FB
:1014D300C210C21402096B120E76E5BE7F097E3A72
:1014E30002D4C1120E7BA8BF120EDC120D46120FDE
:1014F3003EA8BF120F98120E85E5BC120FF17F2D87
:10150300A20A1216157F36A267121615120E5DE592
:10151300BC7F487E3202D3E3120D467F1BA20D121D
:1015230016157F24A20E121615120E71E5BC1213A6
:101533005E7F09E5BCA2E7121615A8BF121724E5C2
:101543002B54037F367E3212D4C1120E7BE5BE7F4D
:10155300637E2C12D4C1120E85A8BE121411A8BF2B
:10156300121458120E67A8BC021769120D467F09A0
:10157300A20F1216157F12A208121615120E67E596
:10158300BDA2E37F48121615E5BDA2E57F5A1216E8
:10159300157F51A20C1216157F24A20B1216157F6C
:1015A3002DA209121615120E71A8BD02109C120E5F
:1015B3005D85BE1085BF11121158120E67A8BE12A9
:1015C3000AA1A8BF120ADF120AE7120E76E5BE7F50
:1015D3003F7E3A12D4C1120E62A8BF120A67120EDE
:1015E3005DA8BD1211B4120E7BA8BC12127E120E9E
:0415F3007612121941
:1015F700120E7BA8BD121300120E67E5BDA2E07F95
:101607006C800B7F098040120D467F48A25E744EA6
:10161700400274597E3A02D4D4127DAD7F73127A98
:101627000B127DFC7F6C127A1A7F2D801A120E67BF
:10163700E5BDA2E77F63121615120E76E5BE7F0998
:101647007E3A12D4C17F4812166EB40104BF090155
:10165700E4F51075F005A47E1E909F842582F5821F
:1016670050020583027702120E67E5BD035403C2D9
:1016770034C25330E103D2342230E002D253221273
:101687000E9E1F12164E12DD12E5101000121001E9
:101697000610020280ED22045403B4030AE4800713
:1016A700145403B403011423C5BD54F925BDF5BD76
:1016B700124EE680CE1275D1EBF516F5147F6C123B
:1016C7007A1A1275B57F647E23E51612D440C3E5F6
:1016D700169514F5167F73127A0B7F2D02164E7F1F
:1016E7002E120E9E120E71A8BFE824FA400330375F
:1016F70002780312172412DD1210000810010D10D2
:10170700021280E518B800E1780580DD08B806D92F
:10171700780180D5799DE8F7F5BF0209687F2D7EAE
:101727002C7420B80502742E12D4D47E32E802D469
:0C173700C17F5B120E9E120E67A8BCE87A
:1017430012176912DD1210000810010D1002128029
:10175300EE18B800EA780380E608B804E27801805E
:10176300DE88BC0209687F5A7E2CE802D4C1D268A5
:1017730075480A1248F0D214122B77127EE5123301
:10178300CFC26B12024A80F3D214751501127D6722
:1017930075B901E5BC20E71C127E9775A6FF127E82
:1017A300F1121E1912DD1212780B10000F500512E0
:1017B300793380E70515E515242050D10206BE12C2
:1017C30017D40202931217D40206FB1217D402098C
:1017D300D91217E0120E768548BE024EE6122B6927
:1017E300122B83125A3612DEE890A029D2491287AF
:1017F3004B128704121DC912DD12100014100105CB
:1018030010021B80F50548E548640A7002F548801C
:10181300CF1548E54864FF700375480980C28548C1
:1018230049122B83E558221248F0122B6985484947
:10183300C250E558B40F02D250125A36803AD2271A
:1018430075480A122B77125A3612DEE812866E900A
:10185300A40C20290390A417121E8BC26A1233CF43
:10186300106A0280E1C227127D3F854948121C3667
:10187300122B83D229125A3612DEE8909F41128727
:101883004920500E121E7512DD121000101001AE09
:1018930080F8121E1912DD1210000280FB0206FBF3
:1018A300122B69E55830E7137F1B90A3F67E0512D0
:1018B300770212DD1212DDF60206FB122B83125A97
:0A18C3003685594912DEE8121E03B3
:1018CD0090A41712874912870E12DD12100008100E
:1018DD00010A10020C80F512193B80DB12194880A9
:1018ED00D612DEE8121E0390A03712874912870E1A
:1018FD0012871212DD1210000810010A10020C805E
:10190D00F512195480DB12196280D6121BFC122BB2
:10191D0083125A3612DEE890A35E128749121E41D9
:10192D0012DD1210000510028880F80206FB055921
:10193D00C3E55895595003755900221559E5596459
:10194D00FF7003855859220549D3E5491495584030
:10195D0003754900221549E54964FF70058558490D
:10196D00054922122B69E55830E7057F240218AD91
:10197D00122B83125A3612DEE890A04012874912BC
:10198D001E8012DD1210000A10010280F8121CA533
:10199D0080DE0206FB122B69E55830E7057F2D022C
:1019AD0018ADC26B7559FF125A3612DEE8121DF3CF
:1019BD00E55930E703121E0E90A051128749128788
:1019CD001E12DD12E55820E7061000081001111057
:1019DD00021B80F00559C3955950CF7559FF80CA28
:1019ED001559E55964FE70C285585980BDE55920D9
:1019FD00E711D26B75A700758307C4F582E0B2E7D6
:101A0D00F080A7306B03121C530206FB122B69E505
:101A1D005830E7057F360218AD122B83125A361255
:101A2D00DEE890A05C128749121E5C4009121C9AD8
:091A3D00121CCF121A460206FB2E
:101A4600120E7BE5BD75F00584F5BCF5BDF5BEF55A
:101A5600BF120915124EE605C6DFF922122B69E5FB
:101A66005820E7087F5190A0660218B012DEE89071
:101A7600A421128749121E1912DD1212484FD2AC48
:101A860010001FE55830E7F8306DF5121B9C7E20DC
:101A96007F00501390A47212773512DD1212DDF614
:101AA60080CAC2AC0206FB1B8B13909F5D12773572
:101AB60012DD12C26B7B007514B8121C8F127E6683
:101AC600127E185025A814E824384004A6010514EF
:101AD6000BC3E5139B50E678B8121CD1306B03128A
:101AE6007BBD122B83125A368082127DADE51660BD
:101AF600E6D26B127EC3C003127D7ED003A9158089
:101B0600C4122B69E55830E7057F5A0218AD122B2F
:101B160083125A3612DEE890A071128749121E36D9
:101B260012DD1210003510010280F8754605121BF1
:101B36006450157F007E357407954612D44012DD39
:101B46001212DDF6D546E7D390A42C500390A4726A
:101B560012874912DD1212DDF680B30206FB124827
:101B66004F12DC2C745212DC3D745412DBFAE55829
:101B76000475590012DC1B1277BA4016127D3F120B
:101B86007E9712780B400B0559C3E558955950ECD2
:101B9600C322C2ACD32212484FD2AC12DB85204CF2
:0D1BA600F1B440F712DB8AB4400312DB8A71
:101BB300B452E2F53812DB8AB454DA12DB8AFA60E3
:101BC300D424EF40D012DB8AE53870C912DB8A12C5
:101BD300DB8A12779F7B007E031278965010205089
:101BE300B412DB8A204C03B440F7DEED80A7127EEB
:101BF300760B12779FDAE0C322121CE0E55924C862
:101C0300F88602E54924C8F9986013146010500F50
:101C130018E608F618E86970F7A702121CCF22E548
:101C230059640F60F91908E618F608E86970F7A710
:101C33000280E8121CE078C8C250E6B4FF028007B5
:101C430008B8D8F6D25022B8D702D250A615807C55
:101C530078B8121CE2E4F9F5A7758307E9C4F582A5
:101C6300E030E70AE924B8F82438400276FF09C3D4
:101C7300E5589950E7121C9A78B879C8E6B4FF0280
:101C83008002F70908E8243850F2804079B877FFDA
:101C930009E9243850F82279C877FF09E924285044
:101CA300F822121CE0C23D78D7B6FF04A900D23D4A
:101CB30018B8C7F5203D0279D81978C8B6FF0122B4
:051CC300C3E899500781
:101CC800C6C7C6081980F478C8121CF1127ED31250
:101CD8007ED3127ED3027ED378C8121CF1127EB155
:101CE800127EB1127EB1027EB175C703E54875F068
:101CF80004A42480F5C62212DEE8C23C1276F4E57C
:101D080037605314604D14604514603D14603514F9
:101D1800602D14602514600E14600B14600D14609F
:101D28001414600C803012160E802B1216BC8026FC
:101D38001215B1802112160A801C1216348017124F
:101D48001620801212156E800D12151B80081214B1
:101D5800E680031214DA12DD1212DDFA121DF312F4
:101D6800B993A81F08E814C23BB51D02D23B75F011
:101D780007203C0375F009A4FF7E00303C0C74205A
:101D8800303B02743E12D4A2800A740B303B0274BA
:101D98000A12D4BAD8CF12DD12E51D1000081001BE
:101DA8001010021880B9651F7003751DFF051D808E
:101DB800AE7005851F1D80A7151D80A375F003A4AF
:101DC800227F7B7E0090A376127735E54824F64083
:101DD800087E0A90A3D712773522127A377E0574C7
:101DE8005B12D49E7E1D745C02D49E121DE27E346A
:101DF80090A387027735127A378003121DE27E316D
:0E1E080090A38B027735121DE27E3190A47DEF
:101E1600027735127A377E008005127A377E2D904A
:101E2600A47D027735121E367E31909F9802773553
:101E3600121E197E1A909F9D027735121E1980C0B8
:101E4600121E197E18909F4B027735121E197E1AA4
:101E560090A482027735121E197E1A90A4871277F3
:101E66003512DD12D3100006C310010280F62212CD
:101E76001E197E1A90A032027735121E197E18900E
:101E8600A04B0277357F007E2012773502DD1212D5
:101E96007A3790A48C027733127A3790A49D027712
:101EA6003312BE55120E94E5BDF55EF56CE5BCF534
:101EB6005FF56B756A007561FF75A70490070012E0
:101EC600BDFFB4FC23E582C313F561E56CF0E56B59
:101ED600F0E582600F12BD76E56C655E70E1E56B3C
:101EE600655F70DB75A700223024EA0460E7240FE3
:101EF60040D380E1E560758307C333F582E0A3F53F
:101F06006CE0F56B756A0022D2248002C224D214DA
:101F1600C21F121EA7756000E561B4FF1612DEE847
:101F2600909E327F0A7E0512773512DD1212DDF39E
:101F3600020293C210C21112DEE8121DF3301F0A0C
:101F46007F07909E4112773380647F007E01C3E550
:101F56006012D4407E0E742812D49E8560487407A1
:101F6600F51FFF7E00743E12D4A2E548121EFC1235
:021F7600C7F6AC
:101F78001224D80548C3E5619548FD401CE51F2497
:101F880007F51F24C850E17F387E01ED0412D440C4
:101F98007E0E742912D49E800DE51F2407FF7E0152
:101FA80090A47C127735201F0312251B12DD121016
:101FB800001910012C10020280F5120236301F3D64
:101FC800020282101F02D21F021F39E56160F4E588
:101FD8006065617005201FF080E9201FE6056080BC
:101FE800E7E56160DEE56065617005201FD5800961
:101FF800201FD5E560700280CA156080CB121EA72D
:10200800121EFA12C7F612260F756A1012BDE812D0
:1020180026C6909E48D23C1276F4121D6490202960
:1020280073021F3902330F022049022035121E5C49
:1020380040CB121EFA12BDFFC2E2FF12BC25021FDE
:102048001212DEE87F6490A6551276F07F7990A68A
:10205800621276F012DD1275160010000A100109DE
:1020680010020280F505160516C253121EFA12C791
:10207800F675370A909E63121CFF90208673022023
:10208800050220AD02227C0222810220710220B4C6
:102098000220B90220710220F70220FB0220FF0271
:1020A800210602210A7F0A12168680BD124868801E
:1020B8000312485D780A1221D9740912DBF812223A
:1020C8001812DC1412225312BDE812BE1012BD37CA
:1020D80012BF27122362D5150C75150A1222661233
:0C20E800248912DC14100204E57F70DB78
:1020F400022005780A800678048002780112486874
:102104008009780A8002780112485D1221D9740985
:1021140012DBED122218E54812DBD9E5165403440C
:102124003012DBFA742A12DBFA12DBFA12DC141214
:10213400225312BDE812BE1012BD3712BF2712235C
:1021440062D51548854815122266E51C12DBD9E5CF
:102154001B12DBD9E51B2548F51BE4351CF51CE4F3
:10216400A27792E7A27492E0A27392E112DBD9AD56
:1021740075AC74AB73E57DC412219AAD78AC77ABC2
:1021840076E57D12219A1224A712DC14100204E5CC
:102194007F709F022005540F2375F00584F8C3EB6C
:1021A40033FBEC33FCED33FDC3EB33FBEC33FCEDE1
:1021B40033FD20E713EB28FBE43CFCE43D12DBD9C0
:1021C400EC12DBD9EB02DBD9C3EB98FBEC9400FCFB
:1021D400ED940080E88848121E20E4F54AF549751C
:1021E4006A2075150112BDE812BD37D5150E854854
:1021F40015E5492401F549E4354AF54AE57F70E5DA
:10220400744012DC3D747812DBFA746312DBFA74E6
:0F2214002102DBED122464E56012DBD9121EFA01
:1022230012C7F6E53A12DBEDE53B12DBEDE53C12B6
:10223300DBEDE53D12DBEDE53E12DBEDE53F12DBC9
:10224300ED740112DBD9E54A12DBD9E54902DBD98A
:10225300121EFA756A20E4F51CF51BF514F51375C7
:10226300150122753800E51412DBD9E51312DBD909
:102273000513E513700205142212486880031248FF
:1022830052121E201223BC12DDFE756A2075150141
:1022930075A6FF754A0112BD9012BD3712BF2712F2
:1022A3002362D5150975151E12238612DE08122422
:1022B30089E57912DBD9E412DBD9E57112234712E0
:1022C300DBD9E57012DBD9E57B24ACFFE55F34098C
:1022D30012DBDFEF12DBD9E51520E033857D56E411
:1022E30012DBD9E52EC412DBDF12DC2312DE081069
:1022F300021A30559B744012DBFA744512DBFA74F0
:102303004F12DBFA744612DBFA12DC23022005E5D6
:1023130056122321C4FAE57D1223212A80C2FBC46D
:1023230012232E2323CB12232E2B22540FFC24F60D
:1023330050027C0090233DEC932200000101010236
:1023430002030303FA2440400A24804003EA3322B1
:10235300D2E72274FF2220E703C3132224C022E51D
:102363003F701F7F7B7E0078AEE612D42AEE2404F2
:01237300FE6B
:10237400743A12D4A2EE2404FEE53E12D42412DDF3
:102384001222C015C016D21212A6ADC212D016D097
:102394001578AEE612DBEDE53E12DBEDE53F12DB30
:1023A400EDE54512DBD9E55212DBD9740A12DBD90B
:1023B40074C012DBD902DC23744012DBFA745412A9
:1023C400DC3D744E12DBFA743012DBFAE51654036A
:1023D400443012DBFA122464742112DBEDE53D1261
:1023E400DBEDE56012DBD9121EFA12C7F678ABE614
:1023F4000812DBEDE60812DBEDE60812DBEDE6126F
:10240400DBEDE53E12DBED1229EFE51212DBEDE523
:102414001112DBED740112DBD990A4AE1224C9753C
:102424006A1012BDE8057F057F787F12DBD2787BC6
:1024340012DBD2787D12DBD2787712DBD2E4FEFF96
:10244400780712DBD212DBD2E57412DBD9E5751200
:10245400DBD9E412DBD9E412DBD912DBD202DC23B0
:1024640075C70375C6FF75B901C217751D0085BC14
:102474001C85BD1B85BE1A85BF191252E9EE12DBFD
:10248400D9EF02DBD9E57512DBD9E57412DBD9E5A6
:102494007312DBD9E57812DBD9E57712DBD9E5765F
:1024A40012DBD9E51664016011E55E12DBD9E57A29
:1024B40012DBD9E516640260012278BCE612DBD98E
:0A24C40008E602DBD975A700E493D7
:1024CE00700122A312DBFA1A80F4AF1F7E0478ADDE
:1024DE00E612D4247E0C742C12D4A27E0E18E612B0
:1024EE00D4247E1A78AEE612D4247E22743B12D403
:1024FE00A27E24E53E12D4247E2FE54012D42A7EFD
:10250E0037743B12D4A20E0EE54102D4247532006C
:10251E00121EFA12C7F6857946787A796412C80FB8
:10252E0074641256DE8E4712260F756A20D23D1243
:10253E00BDE812BE10122646303D09307406C23D6B
:10254E008E1E8F1FE57F602BE54C24FFF54CE54D6D
:10255E0034FFF54D454C600512BD4C80D2751D3CC7
:10256E0012BDE812BE1012BD37122646E57F60037B
:10257E00D51DED1226A79026BF12D500203D0DAE1B
:10258E001EAF1F1226A79026B812D500E546FD7085
:10259E000B90A5E4305D1190A5E0800C04701090B6
:1025AE00A5E0305D0390A5DC7F381241B2804BE48C
:1025BE00FFFC7E05305D047E027FB312546FAC06C5
:1025CE00AB071253397F38C23DE51C6007D23D7E02
:1025DE002C12D48FE51B203D026007D23D7E3012B7
:1025EE00D48FE51A203D026007D23D7E3412D48F7F
:1025FE00E5197E3812D48F1241B7E53224C850FA4D
:10260E0022E54075F03CA42541FFF54CE435F0FE83
:10261E00F54D7C007D1012547C0F8F4BAF4CAE4DA0
:10262E007C007D3C12534F7C00AD4B12547CEE4F20
:10263E0070010F8F4C8E4D2278647973C2D11226A1
:10264E005DFF78677976D2D112265DFE02DE2DC34C
:10265E00E796FB0809E796FC0809E796FDA2E792C4
:10266E001750031255FE75135A30D10E751320B242
:10267E0017AA47125383AB04AC05E546600B046002
:10268E000BAA4612539AEB03FBEB03FBEB543FFBF7
:10269E00E5132B2017029B9B22EE141430E701E466
:1026AE00FEEF141430E701E4FF2205057088A888B8
:1026BE007005052020F8202075320012DEE87E1EFF
:1026CE007F1C12DE2DDFFB12DE2D7E1E7F1C12DE26
:1026DE002DDEFB7E1D7F1D12DE2DDEFB7F007E219B
:1026EE0078ADE612D4247E29742E12D4A27E2D1833
:1026FE00E612D4247E35742E12D4A27E3918E61238
:10270E00D4247F077E21745412D4A27E25744F12D6
:10271E00D4A27E2D78AEE612D4247E35743A12D42D
:10272E00A27E39E53E12D42478AE1229EF7F0E7EBA
:08273E0021744C12D4A27E2587
:10274600744112D4A27E2DE51212D4247E35743A39
:1027560012D4A27E39E51112D4247F157E25744445
:1027660012D4A27E2DE54012D42A7E35743A12D4B4
:10277600A27E39E54112D4247F217E0190A5AF12B5
:1027860077357E0EAC77AB7612D2D67E2B85795F07
:1027960085787B12D87D7F287E0190A5B312773588
:1027A600751D2B751E10E5741229A37E25742F1234
:1027B600D4A2751D2D751E2BE5751229A37F367EB5
:1027C6000290A59F127735E5721228501228E8125A
:1027D6001EFA756A209004E6E56CF09004E7E56B56
:1027E600F0AE4DAF4C7C007D4012547CBF00010F13
:1027F6000FAC07AD07E4FED23D12BDE812BE1012C3
:102806002891E57F602CE54C24FFF54CE54D34FF1F
:10281600F54D454C600512BD4C80DE751D3C0E1213
:10282600BDE812BE10122896E57F600612BD37D5A8
:102836001DED1228667F7812C9F97F767E00743006
:1028460012D4A2E53224C850FA227E2112CF4612B3
:10285600D4407E2F90A5B7305D0390A5BC02773596
:102866009004E6E0FD9004E7E0FCC3E56A9420FBF3
:10287600E56B9CFCE56C9DFD50032410FD12556E26
:0D2886009004E8EEF09004E9EFF022DD038D
:10289300AD040E7F78E55E20E72AE57A8549F0A44A
:1028A300A9F0E57A854AF0A429F9E435F0FAE55E62
:1028B3008549F0A429E435F02AFAE55E854AF0A4B7
:1028C3002ACF9FFF12DE2D103D18C3EF9B50131B21
:1028D300EF6B600E8F018B0712DE2D1FEF6970F80F
:1028E300AF01AB072290A564305C0390A57D754AC8
:1028F30040754900AF76E577FE20E76B7005EF245E
:10290300105064EF24A8EE34FD401190A569305CAB
:102913000390A581754A1975499A8075EF2450EE85
:1029230034FB401190A56E305C0390A586754A0C6C
:102933007549CD805CEF24A0EE34F6401190A5716B
:10294300305C0390A58B754A067549668043EF2476
:10295300F0EE34F1401390A574305C0390A59075AC
:102963004A04754944802A8028EF2490EE34E840D5
:102973001190A577305C0390A595754A0275498F30
:10298300800F90A57A305C0390A59A754A0175492A
:102993009A7F401277337F4612C9F97F5F02C9F9E4
:1029A300AE1E75F064305C0375F03284C0F0F870CD
:1029B30004EE2404FEE51D12D4A2EE2404FEE86016
:0129C300070C
:1029C40012D48FEE2404FED0E075F00A305C037557
:1029D400F00584A8F012D48FEE2404FE742C12D4D3
:1029E400A20E0EE8305C012302D48FE53E2541F5AA
:1029F4001124C45003F511D3E63540F51224E850F0
:102A040002F5122212B98DC21012DEE87F057E098A
:102A1400909C6A1277027F137E08902A3C12D5009C
:102A24007F2B7E01902AA412D50020370A7F277EAF
:102A340027902B1612D50022113007FE1FE001E16A
:102A440001F80F00061B00F80C00180E007C1000A3
:102A54007006003C2000E006003E4001E004001E39
:102A64008003C004001F0003C004000F000780009F
:102A7400000F800780000017800F00000027C00FA0
:102A840000000043C00F00100083E00F002003018A
:102A9400F00700C00F01F80383007F87FE01FC00EC
:102AA4000E3E1800000300000000180000030000A0
:102AB40000003800000000000000300000000000AA
:102AC4000000FC761F0E1C6030ECFCBC3F172DF0A0
:102AD400F978613866264F619A706070C60E1EE3FD
:102AE40030E06060C60C1CC360C0E0618C0C18C789
:102AF400C0C0C0E18C1C39C611C0C4C19C993196B8
:102B04003180C8C1FF1E31E7E180F0C0EE1C31C343
:102B1400818006163091882892884924904927900C
:102B24009248A0E3C8BCC2AFD2C075C0107581D8AA
:102B340074FE122B42E4F5F9F5FBC2B480F7D2A679
:102B4400C2A512B97212DDFA02B99375C703E5483A
:102B540075F004A42480F5C6C23C75B901E5BC0433
:102B64007002D23C22120E76E5BEF54824F65003DC
:102B7400754800753400753704C228D229D22A75E5
:102B8400C703E54824E75003754800E54875F00499
:102B9400A42480F5C6751607751700C23C122BC411
:102BA400122BC4122BC4122BC485175815587559EF
:102BB40000E548B40A09E5586005F46002055922A5
:102BC400203C1D75B90105C6AABCABBDACBEADBFEA
:102BD400EA122BE5EB122BE5EC122BE5ED122BE5BB
:102BE40022203C07F515B4FF03D23C22C0C7C0C65F
:062BF400127D6775A704C5
:102BFA00851683E517C4F8F58275B90105C6E5BCE3
:102C0A00F0C582F82406F92403C582E5BDF0E5BEC5
:102C1A00F0E5BFF075B90105C6E5BCF0E5BDF0E524
:102C2A00BFF08516838982E4F075B90105C685BCB3
:102C3A001385BD14E4F0F08882E5BEF0E5BFF075B7
:102C4A00B901E5BCF0E5BDF0E5BEF0E5BFF075837E
:102C5A0006E51723541E24B0F582E513F0E514F0B7
:102C6A0075A700D0C6D0C705172212BB5578BEA6D5
:102C7A004808E4F6F55908761808F6D23608760AAE
:102C8A0008F6060876BEC254C25512BE6A122B77DF
:102C9A00C229C22AC207C227C268120E67E5BDA2AC
:102CAA00E59243C24AE4F52EF534F536F52F78B6A7
:102CBA00F678B5F678A9F6789EF678B8A65E08A6EC
:102CCA007A12D23FC26BC233C238C240C223C22276
:102CDA00122CF475460278C5A646C23AD221C21908
:102CEA00C226E4F542F541F54022E45407205E0984
:102CFA00B4040040027403801B120E6CC313A9BCF7
:102D0A00600C14A9BD600714A9BE6002A9BFE940FE
:102D1A0001C45407F53722122B69125A3612090CCC
:102D2A0012DEE8121E41E55804700A7F327E0590D1
:102D3A00A3F612770290A64C12874B1208667F728E
:102D4A0090A6411276F012DD1210000510020480DE
:102D5A00F8D322C3220200F7120E67E5BD20E70569
:102D6A00122D2140F0754E50122C7412852C754488
:102D7A00031248ED12AED2D54403022B2A201EF1CB
:102D8A00789F7680754A0012BC86D210C211C2138F
:102D9A00C21212483F75A60C12D98912C474E5A64C
:102DAA0024FA400612488D75A60C20250CE590548D
:102DBA00057009E53524E25003022E54E532241841
:102DCA00400D75F00C84E5F070D41233D280CFD266
:102DDA001ED2AC306DC87532F012DB8FB4E0BF1270
:102DEA004935E53124F39205201203123264122E7A
:102DFA001AC014128E17D014200A03122F3D123350
:102E0A00D212A67C1233D212852F1233D2022D9CF3
:102E1A0030122EE54024F0401C7A0AC3E53F954B58
:102E2A006013401E24E2400D305405C254757F01E0
:102E3A0012BCACDAE679BCE7D2E7F57F09877EC235
:102E4A007722F40424E250ED80DE12DEE87F2A7E47
:0C2E5A000E90A4B212770275A6FFC21001
:102E66001012137F367E08909F7B12770212DD12B6
:102E760012DDF30200F7D22112491112BCB67F1EF1
:102E86007E0B90A3CF12770212DD12122EA77F3E81
:102E96007E0790A10312770212DD1212DDED022BDE
:102EA6002AD215D21412BE41120D4675B90575B94E
:102EB6000212BE4BD25512BD707F0012BC2512BE47
:102EC6004BE56A600512BD3780F7857A62120E946B
:102ED60085BEBC85BFBD856BBE856CBF75B90575E6
:102EE600B90285BD6C85BC6B756A2012BE41123075
:102EF600DE12BE4B756A0012BDE8E57064FE7034E2
:102F06007570FC854077854178851F797818797AC0
:102F160012C80F12BCE512DE0812BE4B756A1012FB
:102F2600BDE87F087810797212C81185627C855ECB
:102F36007D12BCE5C2152212486812308A745212FC
:102F4600DBFA744D12DBFA744312DBFA1230991273
:102F5600DC357441207402745612DBFA122FE61225
:102F6600303012DC35E53C12DBEDE53B12DBEDE5FE
:102F76003A12DBED12306612DC35744512DBFA12BA
:102F860030CF12308A744712DBFA744712DBFA74B8
:102F96004112DBFA123099122FE612DC35E4307456
:102FA600010412DBF812DC359004C3E012DBED12EB
:102FB600DC359004E4E075F00A84AFF012DBED1224
:102FC600DC39EF12DBF8AC5EAB7A1230ABAC5DAB42
:102FD6005C1230AB12DC3512DC351230CF02483FC2
:092FE6007875C23D122FF17878D4
:102FEF00D23D12DC35128211303D05E51E12DBF8A1
:102FFF00E51D12DBF8123073E51812DBF8E57D20C2
:10300F003D01C4540F12DBF812DC35303D09744515
:10301F0030170274578007744E301702745302DB57
:10302F00FA207408123066123066802775A7049054
:10303F0004BFE0FCE0FB7A1B125371783212551378
:10304F001253391230709004C1E0FCE0FB12533977
:10305F0012307075A7002212DC35E4F51AF51980CD
:10306F000D12DC35E51C12DBF8E51B12DBF8E51A57
:10307F0012DBF812DC39E51902DBF8742412DBFAE3
:10308F00744712DC3D745002DBFA12DC35E53D1259
:10309F00DBEDE53E12DBEDE53F02DBED12826D125B
:1030AF00DC35E51D12DBFA781CE612DBF818B817D1
:1030BF00F812DC39E412DBF812DC35744D02DBFA5E
:1030CF00C038742A12DBFAD03812DC1402DE08780A
:1030DF00107F0EE4F608DFFCF564F565F567F5681B
:1030EF007515FC751AC0751DC075664075694075FC
:1030FF004A0112BD9030550302319412BD37E5716C
:10310F00B510004002F510E4F511E512207502E547
:10311F0013C395795006207545857913D3E57A95B4
:10312F0014E5156480FFE55E64809F400C857A147A
:0E313F00855E15857B16855F173074B3C2D18F
:10314D007864797312317278677976123172D2D1CF
:10315D0078187973123172781B79761231728091E9
:10316D0085791280B9D3E7960809E7960809E664D0
:10317D0080FFE764809F20D101B3400AE7F618195C
:10318D00E7F61819E7F622E51AB4C00E7873791828
:10319D0012C80F7873796412C80F78187964C2D188
:1031AD0012320574181256DE8E47AE1EAF1F781BF5
:1031BD007967D2D1123205C3E51F9FE51E9E5004DB
:1031CD008E1E8F1F7EFF7FFFAC1EAD1F12547C7AAB
:1031DD0004EF8AF0A4E5F0CE8AF0A42EFEE435F0DB
:1031ED00BEFF011E60051460057EFF8E1F22EE7E60
:1031FD000020E7F77EFE80F3C3E697FB0809E6970C
:10320D00FC0809E697FD1818191930E7031255FE49
:10321D00C3EB33FBEC33FCED33FDEB33EC33FBED68
:10322D0033FC30D105AA4712539A0BBB00010C7524
:05323D001E03751FFFD8
:10324200EC24FC40048C1E8B1FE627FB0809E637A2
:10325200FC0809E637A2E713F618EC13F618EB138D
:10326200F62210131978B5E624FA401AE57124F60D
:103272004008E57924F6400280360606803212DEE6
:1032820004E59030E2DF753612D22EE4F534F55AB9
:1032920012BE9C1232B5C219C257122CF4129146B8
:1032A200129173D212853F4B754C00205E02D228D8
:1032B200022CECD214123304E6F008DFFB857A62AA
:1032C2001232FA7570FE783A797112C80F12BCE5A3
:1032D2001232FA85627A855E7B120E8A85BC7E8501
:1032E200BD7F7570C012BCE5123304E0F608DFFB47
:1032F20075A700D254C2142274FF7870F608B88001
:10330200FB2275A7049004F078707F1022121EFA37
:10331200122C7412DEE812DD12C258C259754A012B
:10332200753901756A2012BD901256DC8E47C210A3
:10333200D211D214D21212BE9C1291461291731261
:10334200D98975A6FF753609753200E59020E20627
:10335200E5352405400CE5905405701FE53524E25F
:103362005019C211C21212DEE812DD12E4F535F56F
:083372002F7E0612DE00C202EC
:10337A00022005C221E54AB40202D22112BD9012EE
:10338A00A67C30260F125A9812852F753606E53616
:10339A0070FCC22612852C1233D2E54A20E021B4F1
:1033AA000209753900E53670F9808CE53960FAFD55
:1033BA0024E24002053912BD902026C9DDF880E9D1
:1033CA0075390080E475370410003A1001161002AE
:1033DA0016E52F5407600312B98720783D20790A31
:1033EA00207A1F220235C802351CE53760091460AD
:1033FA00091460090236740235E7023645C27902B9
:10340A00369102354FE53724FC500FE537640760E3
:10341A000302370C0236D00234E62011FAE5902076
:10342A00E2028056753400201203D2132278A9E6EC
:10343A007017C226767DE5377005106B02D26BD203
:10344A0077753614D22E02BE91E537604314604078
:10345A00B40227200B24E6249B401F2414501C127C
:10346A00914690A3A27F207E0812770212DD127580
:10347A003608D22E78A9E624ECF622241940FB2439
:10348A001450F712914612917390A3AB7F2980D7FB
:10349A002028E7E54824F640E1E5580460DC7F5D32
:1034AA007E10E6249B40D324145015C2330559C319
:1034BA00E55895595005855859D22690A39080A968
:0434CA00241940B6CB
:1034CE00241450B2E55960021559102606E55960CC
:1034DE0002155990A399808D10780122753900E557
:1034EE003424384007754A0175340022700AE54AC3
:1034FE0030E0F2754A0280F0146008754A061291A7
:10350E00738006754A0412914675390180DA3029A6
:10351E0009C229D22A7559008005302A1BD22912D8
:10352E0086FA1286C8E53524AF400475340022753C
:10353E003700C229C22A80F3206841302703D26A9D
:10354E0022D2221238A812DD12107A0122E534247A
:10355E00384007122CF475340022700FAA37122C43
:10356E00F46A70F27401122CF580EB04122CF5241F
:10357E00FC50E3E537B40706D22880DA8036C2283D
:10358E00E53724FC2324BEF879C4E7F9A74809A738
:10359E005979C4E8F78648088607E537B4050575F6
:1035AE004818D236122B838F59E53764067002D233
:1035BE000702356412388402382EE537601B14601A
:1035CE007614600F146009E53724F9400902378636
:1035DE000236740236BF023753D223124096107948
:1035EE000122E534243840077546017534002278EF
:1035FE00D87020304A0BC24AE624F85004B24380F9
:03360E000AD24A93
:103611007614E54624FE40DDE54660D9154680D89E
:10362100B600D5B40500500C04F54624FA50C9750E
:10363100460580C424F95005127B5B80BB100FB88E
:10364100D20F80B4D223E53464C8600312409610CF
:10365100790122E534243750097011105B32D25BB5
:10366100802E100802D2081240968024100C21D21C
:103671000C801DD22312409610790122D24BE534E1
:1036810024374010C258C259201105D22E75360771
:103691007534002224FD401524037006D258C25906
:1036A10080EEC258D2591460E7D25880E3120E71ED
:1036B100E5BCB2E7F5BC79A1F7124EE680D278B845
:1036C100A65E08A67A2011C8753605D22E80C130B3
:1036D100122B128734055BE55B75F00B84E5F0F581
:1036E1005BE55A24F64009E55A955B5003755B008A
:1036F10012873812DD12E5346003D534D2753400F7
:1037010022D229D22A75480A0237F4C2401007F1A1
:103711003029030237F41286F612870A102A1BC2D7
:10372100330559C3E558955920E7025008755900EA
:10373100E548B41816E558B4FF0375590012871E01
:1037410012DD12E5346003D534C122D22A1286FA81
:1037510080EE301223128734155BE55B30E70C7580
:023761005B0A01
:10376300E55A24F64003855A5B12873812DD12E5C9
:10377300346003D534DA75340022D229D22A75484D
:1037830017804CC2401007F22029441286F6128794
:103793000A102A22C2331559E55930E71C855859B6
:1037A300E558B4FF03755900E548B41802800AD2FE
:1037B3002A1286FA800E855859E558B4FF037559C5
:1037C3000012871E12DD12E5346003D534B52220C2
:1037D300106220115F7F180548E54864187008F5EA
:1037E3004830270375480A122B4F303C2DDFE88001
:1037F3002620105A2011577F181548E54830E70551
:10380300754817800A640970063027037548171234
:103813002B4F303C05DFE275480A122B83125A36D0
:10382300E532244C50051286C8800312866E753427
:103833000002DD1212386B7F15E5486B70048A486D
:1038430080020548122B4F303CD0DFED80CC12387C
:103853006B7F15E5486A70048B4880021548122B6C
:103863004F303CB6DFED80B27A007B09E537B40414
:1038730001227A0A7B17B40601227418FAFBF54871
:103883002275A704758307E559C4F582E0E0F57353
:10389300E0F574E0F575E0F576E0F577E0F5787539
:1038A300A700025A36E59020E23EE534243750382B
:0638B3001238EC1238C9C6
:1038B900205E4F7F2C909D1F123933909D28806A7E
:1038C900E534243775F009A42435FF205E0624BEAB
:1038D90050027F3EEF249B50027F627E3274891230
:1038E900D4D42275A7049000317E087F3AE4F0DF32
:1038F900FDE5822446F582E43583F583DEED75A77F
:1039090000227F2C120E6CE5BD12391CE5BE12395E
:103919001CE5BFF8C4123922E8540775F009A490D0
:103929009D0D2582F58250020583EF2409FF027659
:01393900F09D
:108529000285E312DEE8E53724FC40F4B4FE1420AA
:10853900110EE590F45407600122E532247450EFDE
:10854900028E2312DEE812D67712D70912CF5412FF
:10855900D29512D0DE7E197F3612D03212DC421249
:10856900D048C206E53760051460338053C23A1219
:1085790086871241591242EE1245D41264F41265EB
:108589001C123E04E54864186009E54824F65003C6
:108599001246BF128DB912CDD91241F48014D23AC4
:1085A9001286AD1239421241C312C95F128DB91236
:1085B900CD9A125D7712D750125848125B47801234
:1085C90012869312C89C12D82012C92E128DB91284
:1085D900CDB130101112CFE6800C12DEE8E5372458
:1085E900F9401E1286703022091238A8E53470024B
:1085F900C222302309124096E5347002C22302DDFB
:1086090012121DF375170012DA337F1212C9E730FF
:10861900124A75100075A704758306125AF1E51000
:1086290075F009A42415FFF5177E00E512602F7572
:10863900F06484E5F00F12D4241F7E0EE51112CFE9
:108649009C751623125CAD0510C3E55A95104006BA
:10865900E51024F550BF3012031287388088745D05
:1086690012D4D480D5C249302905121DC9800312FC
:108679001DF3909F4112874B202A7602871E3012E4
:1086890023305E2030501D028A2F301217305E06CB
:03869900200B11A2
:10869C0002909012C9E07F1712DD8875172002DA5C
:1086AC003312D5EE12D58F30121120510512D64E41
:1086BC00800612CD3412CB141251AB22E4FEFFE52E
:1086CC004824F6400D90A3D71277357E16E5480264
:1086DC00D48FB40E0690A3DD02773590A3E6127703
:1086EC00357E12E54824F702D42A7D20800C7D3F8C
:1086FC00302A077D633029027D3C7F0080247D2059
:10870C0080127D3E800E7D3CE54975F007A4240661
:10871C00800A7D3FE55975F007A42409FF640270B7
:10872C0001FF7E1CED02D4A27D2080027D3FE55B23
:10873C0075F009A42416FF7E09ED02D4A2C24912D9
:10874C0087AFB4FF01227510001287C67920E03084
:10875C00E702792F3049171211AEFAB40408E5106C
:10876C00700C79658008EA14651070027923E97E33
:10877C001812D4A27E20E51230E708909F7B127766
:10878C00358016E51112883C125D0D201005201164
:10879C000280063012031287EE0510C3E5589510BF
:1087AC0050A7227E207F001277351286C87E007F6C
:1087BC000690886E12D500E5582275A704758307BC
:1087CC00125AF1E51075F007A42409FFF5177E0085
:0B87DC00E51212D4A27805EE2404FE82
:1087E700E012D4A2D8F6221288F612890CFD7C007A
:1087F700AE1CAF1B12546FBE003A8F00C3E57A95CB
:1088070013FFE55E9514FE402B7C007D2812547CF7
:10881700C3EF98401F75F0058404FB24F950027BD1
:10882700067E2CAF170F12DE2D0F12DE2D0F12DE74
:108837002D0EDBEF2264B4602464B475F03284C07B
:10884700F012D48FCE2404CED0E075F00584C0F0AA
:1088570012D48FCE2404CED0E02302D48F90886A1E
:108867000277352D2D2D000140FFFFFFE0FFFFFFB1
:10887700FFC25030123F20283CE558F460372048AB
:1088870003200931D250E559F51030330665586099
:108897000205101288C012891C75A7049006DCE532
:1088A70012F0E511F0E517F0E510F075A704900652
:1088B700E0ECF0EBF075A7002275A70475830712AB
:1088C7005AF17813E0F608B819FA9006D07811E64D
:1088D700F008B819FAE51CF516F0E51BF515F012C6
:1088E70088F69006DAE514F0E513F075A70022750F
:1088F700A704758306E51023541E24B0F582E0F51E
:1089070013E0F51422120E71E5BD2487E5BD923BF5
:0289170050020C
:1089190024912212890C75F005A485F012F511E451
:10892900F519FEF51CF51D12BE41C23DC2567F3C2C
:1089390012CA8A303D05751900807DDFF3E5596556
:1089490058700A301007EE24D35002D2568C1B8D72
:108959001AE519FD24E250DEAE1CAF1D7C0012544D
:108969006FEFF51924F650CEAC1BAD1A12C9CF2002
:10897900D1108E048F05E51975F0A7A4AEF0FF128A
:10898900546FAC12AB117AA012539AEB33FBEC3350
:10899900FC20D11AEF9BEE9C5014C3E51213FCE5A1
:1089A9001113FBC3EF9BEE9C4004AC06AB072048B8
:1089B90007203B048C128B119006E2E519F0128A0C
:1089C90004AC16AB157AC8125371A912A811125525
:1089D90015ED7005EC249E50057C807B0822C3E5CB
:1089E9007A305602E55C9513FFE55E305602E55D87
:1089F9009514FEC3EF9BFBEE9CFC22AE16AF157CD3
:108A090000E519FD24F6501A12546F7C007D0612F8
:108A1900534F7C007D0512546F8F10EEF51724E932
:098A290050037517FF2212C9E089
:108A3200128A4C128A8F12D244128AB52048091225
:108A42008BA3128BD3028C3680747F177E20204832
:108A52000E748A204D101258B5500E742F80077470
:108A62006A305F02746712D4D475A7049006D07876
:108A720011E0F608B819FA7F177E00781275190509
:108A8200E60812D4D4EE2406FED519F42275A70402
:108A92009006D8E0F516E0F515E0F514E0F513E0E0
:108AA200F512E0F511E0F517E0F510E0FCE0FB75DA
:108AB200A700227F187E26AC14AB1302D2D69006F2
:108AC200E4E0F51CA3E0F51B7F2A304E13120E677B
:108AD200E5BF90A442B4010390A63B1276F0804217
:108AE2000F7E00745312D4A29005CBE0F830E70554
:108AF200E53F30E0091F7E00E8540F12D4BA90041B
:108B0200EEE0FEF51EA3E0FFF51F128B4BE51E24DF
:108B1200E9500C7E06742B12D4D47E0C12D4D412DB
:108B22008B7BC20375172A751627125C7C202415CD
:108B3200205F15D2037F2A7E1E908B69304E0390F0
:108B42008B7202D500205FEB227C007D3C12547CAC
:108B5200A805EF7F2A7E0812D3DD7E12743B12D461
:108B6200D07E14E802D3D70707384C9EBAF2643895
:0F8B72000707387CE6C2E67C38AC1CAB1B7A48A0
:108B8100305D027A27125371A91EA81F125515EDE7
:108B91004C60027BFF7F207E28EB12D3E37E3902FB
:108BA10091237F2B90A3EC127733E517F46022AE6B
:108BB10017AF107C007D3C12547CA805EF7F2A7E04
:108BC1000C12D3DD7E16743B12D4D07E18E812D37A
:108BD100D722AE12AF117C007D0A12547CA805EF9A
:108BE1007F207E3012D3DD7E3A742C12D4D47E3CA9
:108BF100E812D4BA0F7E29744502D4A27485800785
:108C0100748720560274867E2912D4D430170774D3
:108C11002D7E3A12D4D4227C007D0A12547CA80500
:108C2100EF7F2A7E3012D3DD7E3A742C12D4D47EAB
:108C31003CE802D4BA128D67E54824F65005128C3F
:108C41001880B9E559046558600D128C18128BFD16
:108C5100E559655860AA22A217923D8E1E8F18858C
:108C610015179006D0E0F51185581015101245B46E
:108C7100C3E51195105002F404F924A65005C374FC
:108C8100B399F9E975F00584F924EE500279119050
:108C91008DA7E993F5F0120920E5CC7004E930E7DE
:108CA10002747F23A4A9F0E51B2517FDE51C3516E9
:108CB100FEC3ED99F515EE9400F51675A7007583C1
:108CC10006E55823541E24B0F582E0A3F513E0F520
:108CD10014128D67203D2C201729120E71E5BD2439
:108CE10087E5BD5002249175F007A4FB9518E5F0C6
:108CF100951E400FEB9FE5F09E4008EF9518EE950D
:108D01001E500EA23D9217AE1EAF18128C18028B88
:108D1100FD306B10128D04E53F20E00774867E2242
:108D210012D4D42275A7009006E0E516F0A3E5154C
:108D3100F0128C18128C0174857E2312D4D48558BC
:108D4100101288C0128A4C128A8F8C168B15128AC7
:108D5100B51289CA1288B212D2449006E2E0F5191E
:108D6100128A04028BA3C3E57A305602E55C95139F
:108D7100FFE55E305602E55D9514FE921750031231
:108D810055E6AC16AB157AC8125371A906A807129D
:108D910055157E037FE7ED700CEB2418EC34FC4095
:108DA10004AE04AF032200172E43576C8092A4B681
:108DB100C5D3DFE6EDF3F8FD305E4F30504C75A7BB
:108DC100009006E0E0A3FCE0FBECA2E79217402054
:108DD10024FE50047F3B8022AE04AF037C007D144F
:108DE10012547C74542F2017029F9FFF7462800CD1
:108DF1001255F6EC24FE50E07F6D743D7E0012D4D6
:108E0100A27E017D197C03128E0C227F3D12DE2D84
:108E1100EF2DFFDCF822E537B40206E534243750A4
:108E2100292212DEE812D67712CF54128FA312C86C
:108E31002A12CDC1128FFB125B477F207E2B12D0ED
:108E41003212D70912DC421238A812D16A128ED11D
:108E510012514502DD1220041EE579FD24A05002C5
:108E61007D5FED24CD401E744520750C2DFFF5125C
:108E7100128EA61FBF44F922C39DFFF512128EA6C2
:108E81000FBF46F92220750EED2413FFF512128E45
:108E9100A60FBF78F922C374779DFFF512128EA633
:108EA1001FBF12F922EF24BA40082433FCC37432E5
:108EB1009C1404FC24D750047C238009EC2375F016
:108EC10005842413FC7E0512DE2D0EECB506F82276
:108ED100E59020E206E53424374003128E577F45A2
:108EE1007E047D1212DE2D0EDDFA7F437E00746456
:108EF10012D4A27F4F7D12128F8C7F3B7D12128F75
:108F01008C7F597D16128F8C7F317D16128F8C7F4D
:0F8F1100637D1A128F8C7F277D1A128F8C7F6DD4
:108F20007D1E128F8C7F1D7D1E128F8C7E057F19FA
:108F300012DE2D0FBF72F97804E57924CD50027846
:108F400009E8305C0123F87F1B128F7B7F6B128F47
:108F50007B18305C01187F25128F7B7F61128F7B1D
:108F600018305C01187F2F128F7B7F57128F7B1870
:108F7000305C01187F39128F7B7F4D7E00E875F0E1
:108F80000A847004E802D48FE802D42AEF651260E4
:108F90000C7E04EE20E00712DE2D0EDDF62212DE3E
:108FA0005D80F790A5017F287E2C1277357E3B12DD
:108FB000D2EDAC5EAB7A7F307E19C23D12D32C90DD
:108FC000A3F07F5D7E2D12773578B9C3E57A9618C8
:108FD000FBE55E96FC7F507E19D23D02D32CE51155
:108FE00064B4700122E51112DCB27831790F7D0B87
:108FF00012DDB01F1E90908B02D500E5716012E566
:109000007012DCB27831790F7D0412DDAC0DBD0A2F
:10901000F97F011290637F1D1290637E2312906D81
:109020007E3F12906D7E247F171290777E397F02EB
:109030001290777E247F071290817E397F1C1290D8
:10904000817E317F0212DE2D7F1C12DE2D7F0F7E8E
:109050002412DE2D7E3E12DE2D7F0C7E2E90D7F563
:1090600002D5007E2A12DE2D0EBE39F9227F0812AB
:10907000DE2D0FBF17F9227D0612DE2D0E0FDDF952
:10908000227D0612DE2D0E1FDDF9220303E0A0E093
:1090900012C9E07F18909D5D1277337F217E0174A5
:1090A0004112D4A27F2A7E01745312D4A29005BE2D
:1090B000E0F51AA3E0F519A3E0F51EA3E0F51D8580
:1090C0001A1C85191B751720129140E519251DF5ED
:1090D0001BF51DE51A351EF51CF51E751729129195
:1090E000409005BA129130AC1AAB19751720129046
:1090F000FE9005BC129130AC1EAB1D751729EC70AB
:1091000006EB24CD4001227A48305D027A271253C3
:1091100071125515ED4C600122AF177E07EB12D38B
:10912000897E1A0F90A5C4305D0390A5C7027735DC
:10913000E0FEA3E0FD12BF97C3EB9DF8EC9EF92281
:10914000751627025CAD12BF9775A7049005B47819
:10915000737F06E6F008DFFBECF0EBF0E0E0E0FC0C
:10916000E0FDE0FEE0FFEF2DFFEE3C9005C0F0EFEC
:0B917000F0801275A7049005BAE0FB28
:10917B00E0CBF0EBF0E0E0E4F0F075A7002275A790
:10918B00049005B478647F06E0F608DFFB75A70052
:0E919B00125EBC9005BEE51CF0A3E51BF022A1
:10393A00D23C799E77008002C23C12BE41E4F51067
:10394A00F511F512F513F514F515F516F517C23D2F
:10395A00123C8A203D1F123C8A203D19E51F30E5A2
:10396A001130E40E1239B1303C08799EE724F55043
:10397A000122D510DBAE14AF157C00AD12125449EA
:10398A008F55AE16AF177C00AD1312546F125670D6
:10399A007E00E55530E7011E2DFFE43E30E7027F49
:1039AA0000740A2FF55622C235E51CAF1DBFFF056C
:1039BA000FD235F404FABF003F532CF8E518AF19BB
:1039CA00BFFF050FD262F404BF002D20E72A205B57
:1039DA000123FF24AA4021E51AAE1BBEFF050ED221
:1039EA0061F404BE00128547F0A4E5F020E709203F
:1039FA005B0123FE24AA5001227C807B8030516621
:103A0A00302163C006C0078AF0E545A4AEF0FFE5A1
:103A1A0056205B011375F009A4ACF0FD12546F74C3
:103A2A00FFBE0001EFFA24C050027A3FD007D00649
:103A3A00E55212DCB2303504B2D5B2D1EA8CF0A428
:103A4A0030E70205F0748025F020D10495F095F056
:0A3A5A00FCEA8BF0A430E70205F04F
:103A6400748025F030D50495F095F0FBC3EC2F203D
:103A74006203C39F9FFFEB2E306103C39E9EFE2013
:103A84003C64200C05123B1E4064123B00405F1254
:103A9400DE2DE51EFD24FB50550E12DE2DED24F621
:103AA400504C1E1F12DE2DED24F150421E0F12DE6B
:103AB4002DED24EC50380F12DE2DED24E7502F1F8E
:103AC4001F0E0E12DE2DED24E250231E0F0F12DE08
:103AD4002DED24DD50180E12DE2DED24D8500F1ECE
:103AE4001E1F1F02DE2D123B004003799E0722E9B0
:103AF400242AFFE82461FE123B1E401DEF2460408F
:103B040018243F5013EE2460400F243F500AEF2442
:103B1400D6FFEE249FFEC322D322532CF8432C0459
:103B2400EE10E706D2E7F404D261FE24D340EAEFB4
:103B340010E706D2E7F404C262FF24D340DBEFB5FA
:103B440006005003CED26070057480FE8062FF24AC
:0D3B5400FD5060903C0A938EF0A4AAF0335F
:103B6100CA33CA33CA33CA33CA33FA903C34938F47
:103B7100F0A433C5F033CA903C5593FB123BD29568
:103B810070500224B412DCB2EA8BF0A430E70205D3
:103B9100F0C3748095F020D50425F025F0FEEA8C61
:103BA100F0A430E70205F0C3748095F030D104250C
:103BB100F025F0FFC3227A01EE6F70097B16BF0278
:103BC100BB7A0380B7BF01047B0080B07B0D0A8004
:103BD100ABE52C540723C3903BDC73800E800E8031
:103BE10024801E8010800A80108012EB22742D9B8D
:103BF10022742D2B22745A9B22745A2B2274879B78
:103C01002274872B2274B39B22FFFFCCAA9280716E
:103C1100665D554E4944403C383533302E2C2A28B8
:103C2100272524232221201F1E1D1C1B1A1A1918A7
:103C31001817178181818282838384858687898A87
:103C41008B8D8F90929496989B9D9FA2A4A7A9ACCF
:103C5100AFB1B4B400010203040405060708090A60
:103C61000A0B0C0D0D0E0F0F10111112131314145A
:103C7100151516161612BD7912BC07E4F5F7C2B276
:103C8100C2B2E5F7D2B264C022203D07123C767081
:103C910003D23D22056D056D12BC077D008DF7C273
:103CA100B2C2B285F71F8DF7C2B2C3E5F79573F5BE
:103CB100188DF7C2B2C2B2E5F79574F5198DF7C246
:103CC100B2C2B2E5F78DF7C2B2C3E5F79576F51A40
:023CD1008DF76D
:103CD300C2B2C2B2E5F79577F51B8DF7C2B2C2B295
:103CE300E5F78DF7C2B2C2B2E5F7F51E8DF7C2B2A2
:103CF300C3E5F7957AF51C8DF7C2B2C2B2E5F78D2D
:103D0300F7C2B2C2B2E5F7D2B2543F30E50244C0C3
:103D1300955EF51D156D156DE51024784001227E25
:103D230000AF55EF30E7011E0512E51FA2E592D55E
:103D3300400EE515951EF515E5149400F514800B5A
:103D4300E515251EF515E43514F5147800E51E6018
:103D53000620D50318F404C39FF5F0E89E30E7016D
:103D6300220513E5F0A42517F517E5F03516F5162A
:103D730022303D03D23D22123C7660F8123C76603D
:103D8300F3E546600A123C7660EA123C7660E5058C
:103D93006D056D056D12BC077D008DF7C2B2C3E5DD
:103DA300F79573F5188DF7C2B2C2B2E5F79574F5BE
:103DB300198DF7C2B2C2B2E5F78DF7C2B2C3E5F708
:103DC3009576F51A8DF7C2B2C2B2E5F79577F51B72
:103DD300D2B2156D156D156D2230742412BE41C219
:103DE3003D75101E123D74203D167902123E484067
:0A3DF3000CA806A907123AF34003DA
:103DFD0012DE2DD510E422200F4030123D2006CFCB
:103E0D00304806200C03204FC6E546790260147930
:103E1D000614600F791614600A79361460057976E8
:103E2D0014701712BE41C23D7896123D74203D0AA2
:103E3D00123E48400312DE2DD8F022532CF8AB1859
:103E4D00E519FC339262123E9ABC002BEB89F053BC
:103E5D00F00784FF24DF401FAB1AE51BFC33926192
:103E6D00123E9AAA4712539ABC000CEB89F053F0FC
:103E7D000784FE24DF5002D32274562F2062029F46
:103E8D009FFF741F2E3061029E9EFEC322500312AF
:103E9D0055F6E920E40122C3EC13FCEB13FBE920FA
:103EAD00E50122C3EC13FCEB13FBE920E60122C371
:103EBD00EC13FCEB13FB2274542F2062029F9FFF27
:103ECD00741D2E3061029E9EFE2279B4203249204F
:103EDD001D46EFB506009260AC06AB074004AC077B
:103EED00AB06903F26EC2304938BF0A4A9F0EC23B2
:033EFD00938BF0B4
:103F0000A429F9903F8693C9904086E52C540793E5
:103F100013E95001F490408EF9E52C54079329756C
:103F2000F0B484A9F022FFFFFFFF7FFF55553FFF4C
:103F300033332AAA24921FFF1C711999174515556E
:103F400013B1124911110FFF0F0F0E380D790CCC60
:103F50000C300BA20B210AAA0A3D09D8097B0924BF
:103F600008D30888084207FF07C107870750071CC6
:103F700006EB06BC06900666063E061805F405D15B
:103F800005B005900572000000000001010101016B
:103F90000101010102020202020202020203030302
:103FA00003030303030304040404040404040405D6
:103FB00005050505050505050606060606060606A9
:103FC000060607070707070707070708080808087E
:103FD0000808080808090909090909090909090A55
:103FE0000A0A0A0A0A0A0A0A0A0B0B0B0B0B0B0B2A
:103FF0000B0B0B0C0C0C0C0C0C0C0C0C0C0C0D0D02
:104000000D0D0D0D0D0D0D0D0D0E0E0E0E0E0E0ED9
:104010000E0E0E0E0F0F0F0F0F0F0F0F0F0F0F0FB4
:10402000101010101010101010101010101111118D
:10403000111111111111111111111212121212126A
:104040001212121212121213131313131313131347
:104050001313131313131414141414141414141426
:104060001414141414151515151515151515151505
:1040700015151515151616161616161616161616E5
:1040800016161616161600FFFF00FF0000FF002E82
:10409000B5875B2D5A88E537607414603EB40258CA
:1040A0007F347E12E5342437400810644B90A3C15E
:1040B000801AF89041E012D500E824FD501179A152
:1040C000E77E0590A20520E70390A20F0F803A2417
:1040D000040F7E2312D4C1D26480627F357E02E554
:1040E000342437401410641090A0FA30081B127763
:1040F000027E1A90A3C0801122700590A10C800945
:10410000909D8A200C03909D9612770280C97F357E
:10411000E5342433402A2404501B7D0F600C7D1E9F
:104120001460077D3C1460027D78ED305D02C3139E
:104130007E2B12D3897E0090A10D12770202DD1230
:104140007E0524FE5005909F688009909D6D200F8C
:1041500003909D7912770280E4E546604A14603C42
:1041600014602E14602014601290A5F8205D419018
:1041700041D97F367E3412D500803C90A5F8305D61
:104180000390A5F4802A90A5F4305D0390A5F080FB
:104190001F90A5F0305D0390A5EC801490A5EC3045
:1041A0005D0390A5E8800990A5E4305D0390A5E04B
:0241B0007F3658
:1041B2007E331277357E3C7422305D02748302D4E2
:1041C200D4305D0890A5D0305BE4800690A5D8205D
:1041D2005BDC90A5D480D70508B28D8DB5BA0910E5
:1041E20006000A10F248922492249224F2480A10FD
:1041F2000600305E5220434F20284CE55864FF6091
:1042020046E54824F640407F3FE55804F9C23D1296
:10421200424A1211AE601AB404047401D23D75F020
:1042220003A4243CB5070A7E3A303D027E36124290
:104232004C0F0F0FD9D7E55975F003A4243EFF1296
:10424200424A0F0F12424A227E3D12DE2D0EBE401E
:10425200F922C248C249305E56202853E55864FF0D
:10426200604DE54824F640471211AE6042D249B48F
:104272000402803B1465597036D248304E31E559FC
:104282006558602B3074281242B7120E67E5BFB42E
:10429200011DE5BD20E618202416205F129006E4D9
:1042A200E0700CA3E024CE400624255002055922DA
:1042B200305FFC80E820113375A7009006E4E070BF
:1042C20028A3E0302402F404305F02F4042404F949
:1042D20024F74015E924FC4003D26C2270012230FD
:1042E2006C097536A7D22ED22FC26C22305E0830EE
:1042F2007405E558B4FF0122C244C24D780075A787
:0B4302000475830712463688188A1ED7
:10430D008E168F17C23EC23BE54824F6500302437A
:10431D00C7D23EE55860F7E8655970F22048EF12B4
:10432D00447C30D13BAE16AF17A818E54670551238
:10433D000920E5CC49604DD244E5CC7033E924CD5C
:10434D00402EE975F038A4ACF0FB12558512558559
:10435D00EBFDF5111243DD304D2CC206C23B8043FF
:10436D00E546705C120920E5CC7005E924CD50506E
:10437D00124F7C75A704758307A8181246368A1E3E
:10438D008E168F178037120E67E5BDA2E0B3923BF4
:10439D005011307428123AF34026A907A806D20608
:1043AD0012CA711243F91243F01244398907880673
:1043BD001E1F90463112D500800630D103124411D4
:1043CD00A81808C3E55898400302430075A70022BA
:1043DD0074562F2062029F9FF9741F2E3061029E2A
:1043ED009EF822E51865586001227D057A00EA12D3
:1043FD00DCB212DDB00A0AED24F240020A0AEA2408
:10440D004C50EB22AE16AF17123EC41E303E021EAC
:10441D001EE51E12D4A2EE2404FEE51212D4A23023
:08442D003E09EE2404FEE51334
:1044350012D4A222E5186558603CC001C000C01224
:10444500C0138518101245B4D013D012D000D00176
:10445500E510303B07C39570500224B412DCB2203E
:104465003B07AE16AF171243DDE5112402FD7A06B0
:1044750012DDB01DDAFA221211AEB40457E87054F9
:10448500120E85E5BD604D78C6A61308A61208A6CE
:104495002C12C81E75A704758307751001125AC220
:1044A50012C8181510125AC21256DC8E628F63128A
:1044B50057648B1C8A1B12C82420320E12456420B7
:1044C5003B08D24D1266FF1244DA78C68613088679
:1044D5001208862C22120E85AABD7C027BB31253CC
:1044E5009A8C128B13AA1DA91F1253DCA91CA81B99
:1044F5001255158C1D8B1FAC12AB13AA19A91A12D4
:1045050053DCA91CA81B1255158C198B1AE56E25B1
:104515001AF9E56D3519F8C3E56E951AFBE56D9544
:1045250019FAC3E554951FFDE56F951DFCE5542566
:104535001FFFE56F351DFEE52C23652C30E206ECEB
:10454500CEFCEDCFFD75A7049005C2E8F0E9F0ECCF
:07455500F0EDF0EAF0EBF0DD
:10455C00EEF0EFF075A70022D23BC3E5649573C56E
:10456C00659574F564E5669575600404600822E54C
:10457C006424E0500822E5642420400122C3E5674E
:10458C009576F567E5689577F566E5699578600940
:10459C0004600122E566F48002E5668562F0A4748D
:1045AC00E025F04002C23B2212C81E75A704758399
:1045BC0007125AC212C8180510125AC2C02C125A2D
:1045CC00DBD02C891002C82430125120064E780002
:1045DC0075A70475830612463630D139123EC4E5F0
:1045EC004624FE500A0E0F90462C12D5008026EA67
:1045FC007007745D12D49E801C75F06484ADF070ED
:10460C000FED75F00A847008E5F00E12D48F80055A
:10461C001EED12D42408C3E55A9850B475A7002295
:10462C00030340A040030340E040D2D1E8C4F5822C
:10463C00E0FA797312468F30D146AF06532CF8ED61
:10464C00BFFF07F40460390FD262BF00331247C3B7
:10465C00402E797612468F30D126E5822403F582DE
:10466C00E0F512E0F513EEA2E713FEED13BEFF0723
:0A467C00F404600C0ED261BE0006CB
:104686001247E0400122C2D122C3E09709FDE0971C
:1046960009FEE097600904700AEE30E7068007EE2F
:1046A60030E703C2D122E546600E14600BF9EDCE69
:1046B600A2E713CE13D9F8FD227C007B44E54660C1
:1046C600207C007BCC1460197C017B981460127CE2
:1046D600037B3014600B7C067B601460047C0C7BCF
:1046E600C08C148B157AE9125371A8471255138C96
:1046F600168B1775C70075C6047510DF75B901E509
:10470600BC20E76FF51385BD1205C605C675B90150
:10471600532CF8C3E5BE9573FBE5BF9574FC05C63F
:1047260075B901E5BC9575FD5005D2621255FEC3FB
:10473600E5159BE5149CE49D40338C198B18C3E565
:10474600BD9576FBE5BE9577FCE5BF9578FD5005F2
:10475600D2611255FEC3E5179BE5169CE49D400DFC
:104766008C1B8B1A12478AE5322428401305C6E5AE
:10477600C68006E5C62404F5C6700205C7D5100135
:0F47860022024702AE19AD181246ACED1247C31E
:10479500AE1BAD1A1246ACEE13ED131247E0123EF6
:1047A500C4E54624FB50080E0F90463102D5001E85
:1047B500E51312D4A2EE2404FEE51202D4A275F08C
:1047C500067FFDA946B9000575F0027FFF84C5F097
:1047D5002F500205F0C5F0FF24DE228547F0A430F6
:1047E500E70205F0E5F0A946B9000280050475F079
:1047F5000384FE24E022E537B4020122E537700286
:10480500D23964027002C239E53724FC799EE7602B
:1048150005640B600C22D27E20081E401C107F1000
:1048250022D27F2008134011107E01227537012204
:104835007537002039037537022275F9FF75FB00BE
:10484500800E75F9FF75FBFF801C2053F512487D1E
:10485500759E85759D2D801412487D759E84759D68
:104865002D800912487D759E83759D09C2AC75988A
:1048750052C26DC26EC26F2212166EC253E4F5F9B2
:10488500F5FB30340215FB22D2A47F3212DE0AC2B8
:10489500A412D98912DD1212DDF3C214C215124811
:1048A5003F74C012DC3D74A312DBFA748F12DBFA7D
:1048B5001248D374C012DC3D75A7049048DD7F1003
:1048C500E49312DBFADFF91248D375A70022E53825
:0548D50012DBFA74CAB9
:1048DA0002DBFAA29494859C808080808081838008
:1048EA00819E8075A60A12489FD269D2ACE5A62499
:1048FA00FA500C306DF712DB8FB4E0F1124935C271
:10490A00ACC26975A6FF22D21EC274C273E4FDF559
:10491A0071F570C22D12483FD2AC12DB8FC5F07010
:10492A0005DDF7C2AC22C5F0B4E0EFF538E4F532A4
:10493A0012DB8AA2E19273A2E2927475A704900430
:10494A00B4F012DB8AC2D1124B1C20690330740BFB
:10495A008D758E748F73E514C4F57D124B9C124BC2
:10496A001C20690330740C8D788E778F76E51425B8
:10497A007DF57D124B9CD2D1124B1CEEF0F55DEF0A
:10498A00F0F55C207303E4FEFF79BCA70609A707CC
:10499A0012DB8A7D0A124B898F71EE60037571FFF3
:1049AA007D14124B89C22DED24F150010F240A50B7
:1049BA0002D22DBFB4027F008F7012DB8AF0540737
:1049CA00C52E54F8252EF52EE571700EE4F571F515
:1049DA0070C22D9004BFF0F0F0F012DB8AE5386067
:1049EA0009D21EC27412AED68005C21E12AED212EF
:1049FA00DB8AB4E1FA75A7049004C412DB8AF012C8
:104A0A00DB8AF0F53A12DB8AF0F53B12DB8AF0F525
:0B4A1A003C12DB8AF0F53D12DB8AF055
:104A2500F53E12DB8AF0F53F12DB8A12DB8AB4E22F
:104A3500FA12DB8AF07E0C12DB8AFF12DB8A12DBAC
:104A45008A12DB8A12DB8A20E1027F00EFF012DB9B
:104A55008ADEE412DB8AB4E3FA12DB8AFF12DB8A10
:104A6500CF60027F7F9004E4EFF0E4F012DBBA90B0
:104A750004D8124B8912DB8AB4EAFAC2AC75A704D2
:104A85009004DAE561F0E560F0E55EF0E57AF0E5E1
:104A950079F0E52EF0E55FF0E57BF0E551F0207467
:104AA50012E4F571F5709004B4F09004BDF0F0F0E7
:104AB500F0F0F075A70078ABA63A08A63B08A63C2F
:104AC500120E7BE5BF253D240C75F0188478AEA643
:104AD500F0186005640260182216E670121816E6D2
:104AE5007004760C181678ACE6904B0F9308F622F6
:104AF5000618E608904B0F930466700D76011806AC
:104B0500E6640D70047601180622001F1D1F1E1F86
:104B15001E1F1F1E1F1E1F12DB8AFC12DB8AFD12C1
:104B2500DB8AFE12DB8AFFECA2E692E7921713FC02
:084B3500ED92E713FDEE92E79B
:104B3D0013FEEF92E7301701F4F513ECA2E713FC27
:104B4D00ED92E713FDEE92E7301701F4F512ECA2AA
:104B5D00E713301701F4F510ED92E7301701F4F576
:104B6D00111255A620D10E8C1C8D1D8E1E8F1F125D
:104B7D00B2DE1255A630170312B2B82212DB8AC369
:104B8D0013FEF012DB8A92E7FFF07C0002547CAC3E
:104B9D001CAD1DAE1EAF1F30170312B2B8ECF0EDF9
:104BAD00F0EEF0EFF022124BBC0202C612BC46C270
:104BBD00101248F07F5A7E0590A3CF12770212DDB6
:104BCD0012D214D215C255122CEC789F768008762D
:104BDD000012BC861232FA7570FE853A71853B72F1
:104BED00853C73853D74853E75853F7612BCE51217
:104BFD0032FA7570C0757B03757A54E4F57FF57ED6
:104C0D0012BCE5751421751348755F01757B007530
:104C1D00750475745275780175776CE4F57DF551F1
:104C2D00757F0190DF5C85836E85826DC23D124C70
:104C3D009A851C1D75A6FF305505C221022EA7129F
:104C4D004C9AE572A2E59275A2E79277D274D2736F
:104C5D00E51275F008A4AEF0FF2075031255E612AB
:104C6D00C76E12C7B7124D1DE51C251D13F57185B5
:054C7D001C1D12BC5ECD
:104C820012BCB6757F02E56A70B57F5A7E2FE54188
:104C920012D38912DD1280A7856E83856D82C2557B
:104CA2007873124CFE7876124CFEE493F570B4B42D
:104CB20002D255A3E493F51CA3E493F512A3203D7D
:104CC2000FA97BE493F57BC399502A20E702055F85
:104CD200A385836E85826D103D16D23DE582240543
:104CE200F582E43583F583E493F52654F0F57222D8
:104CF200E526C480F630E7D8155F80D48601E493B8
:104D0200F6A308C399500A20E70606B60002080671
:104D12002230E70616B6FF0218162230750DE5138B
:104D22002579F513E43514F514800DC3E51395794F
:104D3200F513E5149400F514AE14AF137C007D0A4C
:104D420012547C8E5E8F7A22124DDF851617203D1B
:104D520001227F5A909C831276F07F64E5166404E8
:104D6200700C909C9B12773312DD1202DDED909C49
:104D72008F1276F07F6E7E0890A5C0127702121E07
:104D82000312DD127515B87514047F6E7E20C224DD
:104D9200A815E82404F9C23DE7124E27203D06E695
:0A4DA20012D4D48008E6128460E801
:104DAC00A815F60515EE2406FED514DA851716128D
:104DBC001E5112DD1210000510018D80F878B8120A
:104DCC000E8F86BC0886BD0886BE0886BF124EE6CE
:104DDC0012DEE8120E8FC23D75160078B87F4B7E3E
:104DEC000890A5C01277027E20E5BC12D4D4124ED6
:104DFC001E7E26E5BD12D4D4124E1E7E2CE5BE12AC
:104E0C00D4D4124E1E7E32E5BF12D4D4124E1E02E2
:104E1C00DD12F608080808F618181824D0500524D6
:104E2C00F64001220516D23D2275C70375C6FE1247
:104E3C00766E124EE675C6FC75BC2675BD6475BEE5
:104E4C00A975BF70124EE675C6FB12766E124EE651
:104E5C0075C6FA75BC1475BD1475BE0075BF0C1201
:104E6C004EE675C6F975BC4E75BDBF75BE0075BFF7
:104E7C0019124EE675C6F875BC0A75BD7E75BE0076
:104E8C0075BF01124EE675C6F775BC0175BD23756D
:104E9C00BE4575BF67124EE675C6F675BC0275BD8C
:104EAC00AB75BE0175BF01124EE675C6F512766E76
:104EBC0075BE0275BF0A124EE675C6F412766E7593
:104ECC00BCE1124EE675C6F312766A124EE615C6B2
:104EDC00124EE615C6124EE615C675B90575B90221
:104EEC0022751500127D6775B901E5BC64816003FC
:104EFC001276510515E515242050E975C70375C6C2
:104F0C008075B90505C6E5C6241C50F5124F1E0266
:034F1C007BBDE476
:104F1F00F5C7F5C6742612766F75BD4E124F38124F
:104F2F004F35E4124F3512766F124EE605C6227FCB
:104F3F00357E00E54B12D4407E10E54C12D4407EF6
:104F4F0020E54D12D4407E30E54E12D440227F46EC
:104F5F007E00E56C12D4407E10E56B12D4407E20AB
:104F6F00E56A12D4407E30E57F12D44022207401CE
:104F7F0022D24475A700758307E559C454F024075E
:104F8F00F582E0F51A244C40E7A3E0F512A3E0F513
:104F9F00131209208938120E67E5BDA2E0923BE596
:104FAF001A40069570500224B4F51A203B05D2061C
:104FBF0012CA71E51A1250DFE5152437F51DE435D5
:104FCF0014F51CE5172437F51FE43516F51E85CCAF
:104FDF0012853813AC12AB137A0412536375380170
:104FEF0024FA401A05382402401405382401400ED3
:104FFF000538053824014006053805380538C3E55E
:10500F001A945A500224B4F51AC23BC23CC23D75E1
:10501F001B00A23B823C406D203B2CE51A75F0082B
:10502F00A4951BFBE5F0303D04940180029400FC35
:10503F005008EB24A0FBEC3405FC1250E6125095FF
:0A504F00923B40031250B8203C2CA5
:10505900E51A75F008A4251BF9E4303D010435F083
:10506900FAE994A0FBEA9405FC5004AB01AC0212E6
:1050790050E6125095923C40031250B8E51B253872
:10508900F51B5094203D04D23D808D22E51F251744
:10509900FEE51E35167016EE24914011E51D251505
:1050A900FFE51C35147006EF2491400122D3228EAE
:1050B900027C8A7B3B125371ED2402FE8F027C8AAB
:1050C9007B3B125371ED2439FF02DE2D1256CF803E
:1050D900311256C2804675F008A4ACF0FB75190070
:1050E900C3EB9468F9EC9401FA40080519AC02ABDA
:1050F9000180ED8C108B11531903E51920E0CD12B5
:1051090056C212513AAF05E51924FE50031255E66D
:105119008E168F17E51920E0B81256CF12513AAF03
:1051290005E5191460061460031255E68E148F15EF
:1051390022AC06AB07AA12A9130253DC125227208C
:105149003D4974857F227E0812D4D47E0830173CED
:10515900AC1EAB1FEB2418EC34FC402F125342E574
:105169001B60077F207E0812D4EF7F207E10E51A8E
:0951790012D4EF7F237E17742E7F
:1051820012D4D07F207E1BE51B7011E519C2E012FC
:10519200D4EF227F207E0E740A02D4EFE51975F057
:1051A200058475F005A402D4EF125227203D5E74E7
:1051B200857F227E3A12D4D4301753AC1EAB1FEB3C
:1051C2002418EC34FC4046EC7033EB249C402E7ED9
:1051D2002D125219125585C0E07F2A7E2EEB12D471
:1051E200EF7E39D0E0C2E012D4EF7F347E3712DE98
:1051F2002D1E12DE2D1F12DE2D0E02DE2D7E30122E
:105202005219125585EB7F2A7E3112CE13227F2A44
:105212007E39740A02D4EF7F2912DE5D0FBF34F9A2
:105222000EBE40F322D23D301266120E71E5BDF57C
:105232001C75F00AA4F824E15002781EE4FCFBFE7F
:10524200FFC23D12BE41125293203D44D8F8751D53
:10525200CEE51C146009751D9C146003751D6AC29D
:1052620017EC30E705D2171255F68C018B00E9488E
:105272007003D23D22EE7008EF251D4003D23D227D
:10528200AC06AB077A1C1253711255158C1E8B1F7C
:1052920022203D07123C767003D23D22056D12BCDE
:1052A20007E4F5F7C2B2C2B2ADF7F5F7C2B2C2B2C5
:0252B200E5F71E
:1052B400FAD2B230E4E3ED2FFFE43EFEE56D2408BC
:1052C400F56D12BC07E4F5F7C2B2C2B2ADF7D2B2C3
:1052D400EA30E508EB2DFBEC3400FC22C3EB9DFB2C
:0552E400EC9400FC2227
:0100030055A7
:10DF5C0069FC362E06FD69FC372F071169FD383038
:10DF6C0007FD69FD3931061169FE383107FD68FE80
:10DF7C003732091168FF373008FD68FF372D07115C
:10DF8C006800362909FE680036290C116801372B08
:10DF9C000CFF6801372F0A116802383009FF68023C
:10DFAC00372E08116803372C0AFE6803372E081128
:10DFBC006704373208FE67043633091167053535B7
:10DFCC0005FF6705353303116706362F02FF670619
:10DFDC00362B05116707362B07FF6707352F051101
:10DFEC006708353104FF6708332E0511670931289E
:10DFFC000700670931250A11670A35240B01670AE6
:10E00C003A240A11660A3C210801660B3D1E0B11CD
:10E01C00660B3D1E0C00660B3D200A11660C3B2165
:10E02C000CFF660C39220E11660C37231100660D9D
:10E03C0036240D11660D34260F01660E3226111191
:10E04C00660E32251401660F35251311660F37271E
:10E05C0016016610392918116610392B1502651135
:10E06C00392D11116511372E0C026512332F081141
:10E07C006512312F07026513302C0A1165132D29F7
:10E08C000E0265132A271011651429270E02651438
:10E09C002C290C1165153129080365153726071134
:10E0AC006515321F09036516411B09116516411CC4
:10E0BC0008036416461F081164164D2105046416E6
:10E0CC005922031164166425040563156A2407118B
:10E0DC0063156D23090663156C230D1163156C25EF
:10E0EC00130762146E2B151162146E2F1406621333
:10E0FC006E30161162136E30150761136F311211E9
:10E10C0061126F350F0761126F380D116011723A81
:10E11C000A086011763F0611601079420209600FFF
:10E12C007A3A0533600F7832040A5F0F742C01338E
:10E13C005F0E722B030A5F0E732E08115F0E743084
:10E14C00050C5F0D722C02135E0D6C2B010C5E0D19
:10E15C00622C05315E0D5F2B030D5D0D5E290833BE
:10E16C005D0D5F23030B5D0D5F1B01335D0D5A16B7
:10E17C00020A5D0D521B00115C0D4D26000C5C0E4D
:10E18C00462802335C0E3926040C5C0F2C2B08330A
:10E19C005C0F23320C0F5D0F172E0A335D0F0C2E04
:10E1AC0009105D0F043507335E0FB23C080F5F0F8B
:10E1BC00AB4209335F0EA43E070F5F0EA2430B3335
:10E1CC00600EA746120B600D9F490C73610C9C49A5
:10E1DC000F0C610B97460973610B8B440A0C610A97
:10E1EC008B420B336109843A080C6108823A043380
:10E1FC0061087934030C60086F2F063360086228BD
:10E20C00050C6008572505336008511F040D5F0885
:10E21C004E1B05335F08491B090D5F094120103760
:10E22C005F0938270D0D5F0A302F06335F0B2B3239
:10E23C00070F5F0B282F0A335F0B262E0E0E600C78
:10E24C0023361137600D1F3F160F600D18411277E2
:10E25C00610D0F320A13610D042B0633610D022E72
:10E26C00040E620D043A0231620E0343050D630D78
:10E27C00B1470113630DA94A000B640CA14D0511A4
:10E28C00640C9B44070E650B99490911650A944768
:10E29C00090D65098E49021365088848060D650845
:10E2AC0081400E336407793B130F6407722F187784
:10E2BC0064076D231A106407692911776407651CBC
:0DE2CC00080F63075D180B33630751190D30
:10E2D9000D630746220E336308402B110F6308387C
:10E2E900291837630932271B0D6309312B1477620B
:10E2F9000A372C0F0A620A3C280973620A441E0B6A
:10E309000C620A48150E33620B46190C0A620B4758
:10E31900260D33610B4C280C0B610B54251037610A
:10E329000B5E24170C600B63291A77600A66361492
:10E339000A600A68390B735F0A6C2C100A5F09724C
:10E349002015775F097422120A5F0873300F775F0F
:10E35900087639140A5F077D3816775F0785370F06
:10E36900095F068D3B0D735F058B4410075F048BB6
:10E37900490C735F048E3F0C075F03863604335FD5
:10E389000394280708600299300E1160029E400527
:10E39900076102A34A0C336101AA4810086201B15E
:10E3A90042127762020131150A6202062B13776362
:10E3B900020830110C63020B361277630310331114
:10E3C9000C6403182B147764032223110A640426AE
:10E3D90023107764042226110A64051C2715776423
:10E3E900051D251508640521271277640628270FBE
:10E3F9000764062F1D11776406350F140764063E5E
:10E409000A19776406401216086407431B117763DB
:10E41900074A22120663075228127763075A2713FD
:10E429000662075E2314776206612011076206649B
:10E439001E0E7362066A1E0E076206742110376289
:10E44900057828130661057A2F157761047A332038
:10E459000661047A301B7761037A281B0761037F01
:10E4690023187761028429160661028832177761B9
:10E47900018D371305610193340C7362009A2E09DB
:10E489000562009D2E043362009D370C0663FFA0D0
:10E4990040103763FFA844140564FFAF4612776440
:10E4A900FF014511056500043F12776500053E101F
:10E4B900076600073F117766000B430D07670110D8
:10E4C9003D117367011539120767021A321277670E
:10E4D900021A2C12076702192C107768031B2E0FDA
:10E4E9000668031F2C117768042729100468042E75
:10E4F9002A0F776705322F130467053330127767C0
:10E5090006362D140567063B291677670643231B34
:10E51900046706471E16776607491E150366074CEA
:10E529001B157766074C2217046607522214776574
:10E53900075B26150265066229157765066D291799
:10E549000165067529137765057D281A0265058217
:10E5590028187765047F1F160265048F2A117765CD
:10E5690003953211006602993D157766029C401C9D
:10E57900FF6602A13E1F776701A43F1CFF6701A741
:10E589004314776801AB4710FF6901B1490F7769F7
:10E5990001024911026A0207490D736A020B480C0C
:10E5A900056B030F480B336B03144A0D026B0419F7
:10E5B9004914376B051F491CFE6C06224824776CE9
:10E5C90006233F21FC6C07203023776C0721272184
:10E5D900FC6C07262420776C08292812FC6C082873
:10E5E9002C0F776C0927230CFF6C09251802316C55
:10E5F90009350F05FC6C094C1401116C09561D01F4
:10E60900FC6B095F2003136B086B2108FB6B087413
:10E619002509336B08772507FC6B0778210D336BC8
:10E62900077A1E0AFB6B077F220C336B06832E0ABF
:10E63900FA6B05853C09336B0489410EF96B048C2F
:0DE649003E10376B038D3C0FFA6B038D40C4
:10E6560013776B02904112FA6C01934110776C01AB
:10E66600984410F86C009B471A776D009F461EF879
:10E676006DFFA24519776EFFA14019F86EFFA640FF
:10E6860014776FFEAA4417FA6FFEAF4A127770FE30
:10E69600B34D18FA70FF024B1B7771FF054718FD43
:10E6A60071FF0942177772000E4012FD7200163D87
:10E6B6000C7372011B3510FA7201232E1577720244
:10E6C60029321AF872032C371D7772032F3014F88B
:10E6D600720336210F77710346190DF87103502026
:10E6E6000B33710353290EF87003572B143770033D
:10E6F600612712F870036F2911777002793017F7C6
:10E706007001803722777001843D1FF67000883FC4
:10E71600197770FF8D3F11F670FF933D0C7371FEF4
:10E72600973D0EF571FE9B3E0C3372FD9F4310F62E
:10E7360072FDA448127773FDAB4C13F573FDB14F10
:10E74600167774FD034F14F775FE074C127775FEA6
:10E756000A4510F975FE0E400F7776FF124111F843
:10E7660076001745167776001C4614F67601214288
:10E7760017777602263D17F3760229382177760336
:10E786002A3315F276032B3009737604302A07F004
:10E79600760439220A337604472110F07504512590
:10E7A60012777504552416F1750459210F777504EF
:10E7B6005F2111F0740463231477740468240EF245
:10E7C600740370230933740379270AEF74028030C7
:10E7D6000B33740185360DEF74018B3913377400D2
:10E7E600903D1BF075FF94441E7775FF984823EF04
:10E7F60075FE9B46207776FE9F4221F076FEA13F6E
:10E80600177777FDA44313EF77FDA747157778FDB4
:10E81600AA4915EF78FDAD4C157779FDB04D19EE87
:10E826007AFDB34D1C777AFD024E19F07BFD054F3C
:10E836001B777BFE094F24F37CFE0D531D777CFF6F
:10E84600114619F37CFF173F12777C001F3810EF33
:10E856007C00263613777C012B3115ED7C012F2B9E
:10E8660015777C02332513ED7C02392214777C025E
:10E87600402110EE7C0249210B737B02531F0FEBE4
:10E886007B02601E15777B026A2214EA7B017428DC
:10E8960019777B017B2D1AEA7B00833122777B0077
:10E8A6008A3320EB7BFF91371A777BFE953C1FEA74
:10E8B6007CFE983C26777CFEA74621EC7CFD9939A8
:10E8C60023777CFC9A3B1FEA7DFC9A3F1C777DFBF5
:10E8D6009A401EE87DFB9B3F20777EFA9B3F1FE612
:10E8E6007EFA9C431A777EF99E4717E57FF8A04A81
:10E8F6000E737FF8A34A0AEA80F8A548073380F822
:10E90600A94402EA81F8AE46041182F8B24C00E747
:10E9160082F80351021183F8085304EA83F90E4D75
:10E92600061183F914430CEC84FA1A400E1184FB89
:10E93600203F0AE884FC2540061384FC2B4008E6A9
:10E9460084FD3039073383FD36300EE483FE3C2BDD
:10E95600193783FE402A1EE783FE3D25187783FE7E
:10E96600371B16E783FF3114137783FF35170FE440
:10E9760083FF3E220D738200412C15E58200432C55
:10E986001A77820046251BE782004C201577810006
:10E99600552116E581005E2510778100682718E469
:10E9A60081FF72291E7780FF7A2E22E580FE7E3057
:10E9B600277780FE812B22E680FD85251C7780FD4A
:0DE9C600882618E281FC8A2F187781FC8DCD
:10E9D3003821E181FB903F287781FA924025E0813D
:10E9E300FA943D237782F9973C18E082F99A3F1510
:10E9F3007782F89E4412E083F8A347107783F8A741
:10EA03004A0CDF84F8AA4D133785F7AC5214E2851C
:10EA1300F7AF56107786F7B2580DE087F802560223
:10EA23003387F8055002E388F8094C051188F90C7F
:10EA33004E02E489F91052011189FA155004DF8955
:10EA4300FB1D45041389FB233304DE89FB292306BD
:10EA53003389FC2B1F05DE89FC2F23093389FD3302
:10EA6300280ADC89FD3B23103788FD471E0EDD880D
:10EA7300FD511E0E3388FD53200CDD88FD54210B00
:10EA83003387FD57200DDD87FD5C20093387FD5D4E
:10EA93002403DE87FD5B29013386FD592C04DE86C2
:10EAA300FD5D2C093385FD622F0CDC85FD652D0B87
:10EAB3003385FC672908DF85FC6722093385FC6BF6
:10EAC300210CDD84FC72280A3384FB783005DD8455
:10EAD300FA7C37073384FA7E390ADC84F9813B06F2
:10EAE3003384F8843F05DB84F8873F023384F78A55
:10EAF3003C04DB84F78D390A3384F6903908D985D1
:10EB0300F5923F113785F595430FD985F498440A5B
:10EB13007386F49B440AD986F39C440C3386F39C96
:10EB23004507DA87F29C47063387F19E4C0AD9885A
:10EB3300F1A251103788F1A65516D989F0A7571FAE
:10EB4300778AF0A9541BDA8AF0AA4D12778BF0ACBE
:10EB5300460DDB8BF0AC4906338CEFAB4D05DB8CFC
:10EB6300EFA95002318DEEA85209E28DEEA7530EA4
:10EB7300118EEEA75316E58EEDA44A20118FEDA05A
:10EB83004423E28FEC9C4821118FEB9A4A22E090B8
:10EB9300EB95411D1190EA8E391DDF90EA893621EC
:10EBA3001190E9873223E590E9852C2C118FE87DBC
:10EBB3002A26E08FE8762124118FE8662122E08F50
:10EBC300E856221F118EE947201DE08EE9392116F0
:10EBD300118EE9302518E28EEA2D2917118EEB30BC
:10EBE3003213E18EEB333711118EEC373C10E18E8B
:10EBF300ED393E07138DED3B4203DD8DEE3B3E09C0
:10EC0300338DEE3B310DDE8DEE392812378DEF3823
:10EC13002319DC8DEF382A18778DF0372A12DC8D13
:10EC2300F0382214778DF0361B0EDC8DF1361B0C79
:10EC3300338CF1371F0DDB8CF136250E378CF23414
:10EC4300270CDC8CF22A270D338DF31F2A0CDC8D65
:10EC5300F3173409338DF4143A08E48EF4123A0CA2
:10EC6300338EF4103D11EA8FF50E411A778FF50CB0
:10EC73004917EA90F50A50157790F5054F13E79178
:10EC8300F5B24F107792F5AD5408E492F4AB5A0104
:10EC93003393F4AB5C05E893F4A9500A3394F3A4DB
:10ECA300450CE094F3A041093394F29A3A05E295B6
:10ECB300F29734043395F1913208DC95F19E310DCE
:10ECC3003395F08A320CDA95F0872D0B3395EF806C
:10ECD300250EDE94EF73220C3394EF6C2412DD9433
:10ECE300EF6928157794EE6B2812DF93EE69280EEF
:10ECF3007393EE64270DDF93EE5C260B3392EE578E
:10ED0300270EDB92EE5828123792EE5E2610DB9226
:10ED1300EE64240D7391EE6C2108D991ED722304F6
:10ED23003391ED782904D991EC7C320A3391EB7F4E
:10ED33003A08D891EB833D093391EA883C0CD7918B
:0DED4300E98D3B103791E9903E12D792E820
:10ED50009143137792E794420ED792E7993E073397
:10ED600093E7A03901D993E7A63B0A1194E6A83F9F
:10ED70000CD794E6AB490E1195E6AE4F07D695E653
:10ED8000004D011396E6034601D996E6033E0811AD
:10ED900097E7043D0ED997E70740151198E70C4314
:10EDA00012DA98E812460F1198E918490CDA98E936
:10EDB0001D44081198EA243D05D898EB293A03111F
:10EDC00098EB2C3707D898EC2D38093398ED2E3D69
:10EDD0000ADC98ED2E3E0A3398EE2D3F0BDB98EFC0
:10EDE0002C420C3398F02B430ED998F02B3D113761
:10EDF00098F12D3710D898F130340D7398F23433E0
:10EE00000FD698F237330F7798F339331CD597F331
:10EE10003C32167797F43E2F11D797F440280973A8
:10EE200097F4422109D797F4461F0AB396F44B2171
:10EE300008D796F45325083396F45C2505D796F445
:10EE40006723023395F4722503D695F3782B0231AC
:10EE500095F37B3102D695F27E31063395F1832FFF
:10EE600004D695F18A2F023395F0913201D596F0B0
:10EE70009638061196EF9A3F02D497EF9D450213FC
:10EE800097EE9F4704D497EEA247073398EEA64427
:10EE900008D398EEAA430B3399EEAD440CD499EE07
:10EEA000B1400D339AEE013F11D39AEE054512772A
:10EEB0009BEE064A15D59BEE064712779CEF05425E
:10EEC00012D79CEF063E0F779DEF084111D39DEFBF
:10EED000094619779EF00B4718D39EF00D431C7717
:10EEE0009FF10F4015D69FF1114113779FF2134602
:10EEF0000ED9A0F2174A0B33A0F31C4A08D4A0F491
:10EF000023420333A0F42A3305D3A0F53127071198
:10EF1000A0F5382300D29FF53D2702339FF6442900
:10EF200003D39FF64F2808119EF55E2807D19EF562
:10EF30006C2D04119EF4752F01D09EF47C2D0433AA
:10EF40009EF3822B04D09EF3872E05119EF28B3503
:10EF500007D09EF2903D01119FF1954203D09FF0A2
:10EF600094400333A0F09F3F0BD0A0F0A13D0F379A
:10EF7000A0EFA33C0DD1A1EFA43C0C33A1EFA43C26
:10EF80000AD0A1EEA53D0533A2EEA63C00D1A2EE2B
:10EF9000A8390211A3EEAA3C04D0A3EEAD3F05119F
:10EFA000A4EEB24008D0A4EE03410C11A5EE064138
:10EFB0000AD2A5EE08450711A6EF094A05D2A6EF29
:10EFC000094C0111A7EF0A4807D3A7F00B420B1118
:10EFD000A8F00B420DD4A8F00D461311A9F111466B
:10EFE00014D9A9F1173F1B11A9F21E381ADAA9F397
:10EFF00021381811A9F31F3A17DFA9F41839151190
:10F00000AAF4163A1DDCAAF5183C1A11AAF51C3A06
:10F010001AD9AAF61F391A11ABF6203615D9ABF753
:10F0200021341711ABF8203B19D9ABF81E3F17114B
:10F03000ACF91D4011D9ACF91E3F0E11ACFA1F40BE
:10F040000CD6ACFB22410D11ACFC23450FD6ADFC18
:10F0500023490B11ADFD214A0DD6ADFE2047091104
:10F06000ADFE21450CD6ADFF22430E11AE00224568
:10F070000CD8AE01214B0A11AE0220500DD7AF03C0
:10F080001D4F0B11AF031A5109D9AF04174A0D11C7
:10F09000B00418470BDBB0051A500A11B0061C5516
:10F0A0000ED7B1071C560B11B10719470ED9B1087D
:10F0B000173C0C11B208183D0CDCB2091C490E11AA
:0DF0C000B20A1E4E0AD9B30B1D500B11B33E
:10F0CD000C1A5109D9B30C174F0711B40D17490B71
:10F0DD00DBB40D17480D11B50E19490ADCB50F1922
:10F0ED004F0B11B50F185605DBB61017550711B696
:10F0FD0011174C0ADBB61116430B11B711173F0D43
:10F10D00DDB71219430C11B7131A480BDCB8131ADB
:10F11D00450F11B81419410DDCB81418400B11B975
:10F12D001518430DDBB91618470F11B91618490DEF
:10F13D00DBBA1718470A11BA1717450CDBBB1814A1
:10F14D00460F11BB18134C0EDBBC1912510A11BC22
:10F15D001A125007DBBC1A12470B11BD1A10400DC5
:10F16D00DCBD1B10400A11BE1B124509DCBE1C156F
:10F17D00490B11BE1D184A0ADBBF1D1B4A0811BFE2
:10F18D001E1B480CDBBF1F1A470E11BF1F1A490B60
:10F19D00DBC0201B4B0D11C0211C4910DBC0211DF4
:10F1AD00470F11C1221D4711DBC1231C4B0F11C18C
:10F1BD00231B4B0EDBC22419441111C224193D0F20
:10F1CD00DBC2251B3B1011C2261D3F0DDAC2261EC8
:10F1DD00411011C3271D3F12DAC3271C3D0F11C368
:10F1ED00281B3D10DBC4291C401111C4291C450FDF
:10F1FD00DCC42A1C460E11C42A1B4510DCC52B1974
:10F20D00431111C52C184511DDC62C164A1011C617
:10F21D002D174A11DEC62D18491211C72E19471088
:10F22D00DEC72F1A460E11C72F1C4410DFC7301F23
:10F23D00471111C731214B0CDBC832224D0E11C8BD
:10F24D0032224A10DAC83321471111C83420460F33
:10F25D00D9C83520461111C93521430CDBC93623D8
:10F26D003F0F11C937253D11DBC93725400E11C997
:10F27D0038254211DCC93925431311C939254312EB
:10F28D00DCC93A25431111CA3B24400DDCCA3C248C
:10F29D00411011CA3C23400EDCCA3D22401111CA57
:10F2AD003E20420FDECB3E20451011CB3F204714B0
:10F2BD00DECB4021441211CB40213F10DFCB412248
:10F2CD003C0D11CB42234011DFCC42233E1111CC1A
:10F2DD0043202F0EE0CC4319221211CC43122011E2
:10F2ED00E3CC4311250E11CD43132B10E3CD441266
:10F2FD002D1111CD440F2B0FE3CD44092B1211CE3F
:10F30D004404320FE2CE4401360E11CF44B3370D13
:10F31D00E0CF44B3330E11D04401370EE0D0440595
:10F32D003D0D11D0450A3B0CE3D14512330D11D1E2
:10F33D00451A2D0EE3D1461E2B0F11D1461D2E0F52
:10F34D00E4D1471D300F11D1471E320EE3D24821B3
:10F35D00330F11D248233510E2D24923350F11D284
:10F36D004A20360EE3D24A1D360E11D24B1B3410F5
:10F37D00E3D34B1B320F11D34B1B300EE4D34C1B7D
:10F38D00340D11D34C1B3A0DE5D44D1A3B0E11D44F
:10F39D004D1B360AE6D44E1D340E11D44E1E360DBD
:10F3AD00E5D44F1F360C11D5501F350EE5D5501F26
:10F3BD00340D11D5511E340EE5D5511E370C11D516
:10F3CD00521E390EE5D652203B0F11D653223C0F5B
:10F3DD00E4D65423391111D654243710E3D65524CD
:10F3ED00360F11D655253310E3D65626330D11D6CB
:10F3FD005627350BE2D657273A0C11D658273C0F16
:10F40D00E2D75827391011D75927370FE2D75A2786
:10F41D00381011D75A283B0FE2D75B293C1111D771
:10F42D005C2B3C12E2D75C2D391111D75D2C3910B4
:0DF43D00E3D75E2B3C0F11D75E293B0EE399
:10F44A00D75F27371011D75F26360EE3D760273CE0
:10F45A000E11D761284310E3D76229451111D762EB
:10F46A00293F0FE4D763283A1011D763293A11E4E8
:10F47A00D7642A3E1011D7652C4211E4D7662E4272
:10F48A001011D7662D3F11E4D7672F3A1011D768AC
:10F49A002D3B0CE4D7682E3D0711D7692E4204E4B0
:10F4AA00D76A2E470111D76B2E4702E4D76B2D403E
:10F4BA000513D76C2B3503E4D76C2A2B0711D76DAC
:10F4CA002B2909E5D76D2B300611D76E2A3A04E4A9
:10F4DA00D76F28400611D76F283E08E4D77027381F
:10F4EA000C11D87026320DE6D871252F0911D87162
:10F4FA0024310AE9D87221340811D8721B3A08EA71
:10F50A00D9730D420A11D973104909EADA730C4505
:10F51A000811DA730A3B06E8DB74093D0211DB7451
:10F52A000A4003E9DB740B3C0213DC75103406EA6B
:10F53A00DC7517350333DC761A3F06EADD771C469D
:10F54A000433DD771F4001E8DD7824360731DD78A2
:10F55A002C3206E7DC7933320413DC79373409E7D5
:10F56A00DC7A3A340C33DC7A3C3508E7DC7B3D370D
:10F57A000233DB7C3C3A05E7DB7C3C3D0333DB7D35
:10F58A003B3A04E7DB7D3B320331DA7D3E2D09EA63
:10F59A00DA7E43270D11DA7E4D230AE9DA7E5726F1
:10F5AA000B11D97D5E2C0BE9D97D61300C11D97D07
:10F5BA00632F08EAD87D662F0511D87C683005EAE2
:10F5CA00D87C6D330611D77B733608E9D77B7C3834
:10F5DA000511D77A853A04E8D8798B3B0711D8798F
:10F5EA008E3809E9D8788F371011D878903B0BE814
:10F5FA00D87791420D11D976954A08E7D976984974
:10F60A000411D9759D4008E8DA75A23A0B33DA7508
:10F61A00A53C0AE8DB75A8430031DB74AA4603E976
:10F62A00DC74AF460213DC74004A02EADD75054C4D
:10F63A000333DD75084D00EDDE75084B0533DF76C3
:10F64A00064902EDDF76044A0131E076044902EA0E
:10F65A00E076044C0513E176045006EAE176014DA2
:10F66A000D33E276B1450FEAE276AD3F1077E375E6
:10F67A00AB3F0DEAE375AC430A33E475AE4604EAE0
:10F68A00E475B0400131E575B23908EAE575013C27
:10F69A000611E675054607ECE6760A4B0311E7768E
:10F6AA000F4604EEE777163B0611E778203405EC9F
:10F6BA00E77827350611E7792D3409ECE7793234F2
:10F6CA000B11E77A3B260AECE67A45250B11E67A16
:10F6DA004D230BEAE67A56250711E67A5F270AEAEE
:10F6EA00E579672A0C11E579731F0AEBE578792E1B
:10F6FA000811E578843302EAE5778D3B0313E67651
:10F70A00954104EAE676993F0733E6759A3801EAA5
:10F71A00E67595310531E6748F3202EAE6748E3564
:10F72A000111E773923301EAE77398310413E77220
:0AF73A009D3304EBE872B4370911A7
:00000001FF
